:100000000C94BB060C94FF060C94FF060C94FF06A0
:100010000C94FF060C94FF060C94FF060C94FF064C
:100020000C94FF060C943F190C94FF060C94FF06E9
:100030000C9488330C94FF060C94FF060C94FF0676
:100040000C94FF060C94FF060C940F160C94FF06FC
:100050000C942A0C0C94FF060C94F40B0C94FF06E1
:100060000C94FB1B0C94FF060C941B2F0C94FF06A6
:100070000C942B760C94FF060C942771261C2B1CD9
:10008000301C391C501C671C771C871CA41C901E3C
:10009000671C521D631D921DB01DCD1D271E821EA3
:1000A0006020F220AF212F22982248234F25AC2533
:1000B00019266326AE26FB264C27AE270D28A72837
:1000C00042293C2A3A2F6E2FB12F213039307A3015
:1000D0003131F831F831F831F831F831F831F8319F
:1000E000F831F831F831F831AD31AF31B431CC31CC
:1000F000CE310A0D426174743A00202564204365B4
:100100006C6C732000204C6F77207761726E696E83
:1001100067206C6576656C3A2025642E2564000A9C
:100120000D466F756E6420424C2D4374726C3A20FC
:10013000002564000A0D0A0D2121204D4953534921
:100140004E4720424C2D4354524C3A2025642021E6
:1001500021000A0D3D3D3D3D3D3D3D3D3D3D3D3D8B
:100160003D3D3D3D3D3D3D3D3D3D3D3D3D3D3D3DBF
:100170003D3D3D3D3D3D3D000A0D43616C69627270
:100180006174696E67207072657373757265207330
:10019000656E736F722E2E004F4B0A0D000A0D46CE
:1001A0006C696768742D74696D65202575206D69AB
:1001B0006E2020546F74616C3A2575206D696E0055
:1001C0000A0D436F6E74726F6C3A2000486561646B
:1001D000696E67486F6C64004E6F726D616C2028A9
:1001E0004143432D4D6F646529000A0D3D3D3D3D62
:1001F0003D3D3D3D3D3D3D3D3D3D3D3D3D3D3D3D2F
:100200003D3D3D3D3D3D3D3D3D3D3D3D3D3D3D0A51
:100210000D00416E676C654E69636B2020202020C5
:100220002020416E676C65526F6C6C20202020206E
:1002300020204163634E69636B2020202020202012
:100240002020416363526F6C6C20202020202020EE
:1002500020205961774779726F20202020202020AC
:1002600020204865696768742056616C7565202098
:1002700020204163635A202020202020202020209D
:1002800020204761732020202020202020202020B3
:100290002020436F6D706173732056616C7565200B
:1002A0002020566F6C74616765205B302E31565D7F
:1002B00020205265636569766572204C6576656CB1
:1002C00020204779726F20436F6D70617373202017
:1002D00020204D6F746F722031202020202020209C
:1002E00020204D6F746F722032202020202020208B
:1002F00020204D6F746F722033202020202020207A
:1003000020204D6F746F7220342020202020202068
:1003100020203136202020202020202020202020B6
:1003200020203137202020202020202020202020A5
:100330002020313820202020202020202020202094
:100340002020313920202020202020202020202083
:100350002020536572766F2020202020202020202E
:100360002020486F7665726761732020202020204E
:10037000202043757272656E74205B302E31415DB2
:1003800020204361706163697479205B6D41685D11
:10039000202052656D61696E4361705B6D41685DDF
:1003A0002020323520202020202020202020202026
:1003B0002020323620202020202020202020202015
:1003C0002020323720202020202020202020202004
:1003D00020204932432D4572726F72202020202048
:1003E0002020424C204C696D697420202020202060
:1003F00020204750535F4E69636B2020202020202F
:1004000020204750535F526F6C6C2020202020200A
:10041000202021212120494E434F4D504154494233
:100420004C4520212121002E000A0D20444143206B
:100430006F7220493243204552524F522120436867
:1004400065636B204932432C2033567265662C203D
:1004500044414320616E6420424C2D4374726C0011
:100460005B25695D005B25695D002B204D696B7222
:100470006F4B6F70746572202B0048573A56256495
:100480002E25642053573A25642E25642563005396
:10049000657474696E673A2564202573004861723B
:1004A0006477617265204572726F7220313A2564FB
:1004B000202121004D697373696E6720424C2D43E2
:1004C00074726C3A25642121004D6978657220456B
:1004D00072726F722100493243204552524F5221AD
:1004E0002121004865696768743A20202535690034
:1004F000536574706F696E743A2535690050726582
:1005000073737572653A253569004F666673657455
:100510003A20202535690048656967687420636F53
:100520006E74726F6C0044495341424C454400481C
:10053000656967687420636F6E74726F6C004449FC
:100540005341424C4544006163742E2062656172E0
:10055000696E67004E69636B3A20202020202025B9
:10056000356900526F6C6C3A202020202020253500
:100570006900436F6D706173733A202020253569DF
:10058000004B313A25346920204B323A253469201A
:10059000004B333A25346920204B343A2534692006
:1005A000004B353A25346920204B363A25346920F2
:1005B000004B373A25346920204B383A25346920DE
:1005C000004E693A2534692020526F3A253469205B
:1005D0000047733A253469202047693A2534692059
:1005E0000050313A253469202050323A25346920B0
:1005F0000050333A253469202050343A253469209C
:10060000004779726F202D2053656E736F72004E14
:1006100069636B25346920282533692E25692900F3
:10062000526F6C6C25346920282533692E25692981
:100630000047696572253469202825336929004EF1
:1006400069636B2025346920282533692E25782994
:1006500000526F6C6C2025346920282533692E25C3
:1006600078290059617720202534692028253369AD
:1006700029004E69636B20253469202825336929B8
:10068000282533692900526F6C6C20253469202895
:1006900025336929282533692900596177202025C8
:1006A00034692028253369292825336929004143E5
:1006B00043202D2053656E736F72004E69636B206B
:1006C00025346920282533692900526F6C6C202558
:1006D0003469202825336929005A20202020253418
:1006E0006920282533692900566F6C746167653A63
:1006F0002020202533692E253169560043757272FA
:10070000656E743A2020202533692E253169410019
:10071000506F7765723A20202020202534695700D9
:100720004469736368617267653A202535696D4174
:10073000680052656365697665720052432D5253B5
:1007400053493A202020202534690052432D517509
:10075000616C6974793A202534690052432D4368ED
:10076000616E6E656C733A25346900436F6D70611C
:1007700073730048656164696E673A2020253569A6
:100780000056616C75653A2020202025356900539C
:10079000746172743A2020202025356900506F74EE
:1007A00069313A202025336900506F7469323A204C
:1007B0002025336900506F7469333A20202533694E
:1007C00000506F7469343A202025336900506F74EB
:1007D00069353A202025336900506F7469363A2014
:1007E0002025336900506F7469373A20202533691A
:1007F00000506F7469383A202025336900536572C0
:10080000766F202000536574706F696E7420202508
:10081000336900506F736974696F6E3A20253369CC
:100820000052616E67653A2533692D2533690045AD
:10083000787465726E436F6E74726F6C2020004E18
:10084000693A2534692020526F3A253469200047DF
:10085000733A253469202047693A253469200048D5
:10086000693A253469202043663A253469200042DC
:100870004C2D4374726C204572726F727320002588
:10088000336420253364202533642025336420001D
:1008900025336420253364202533642025336420E8
:1008A00000253364202533642025336420253364F8
:1008B0002000424C2054656D7065726174757265DC
:1008C00000253369202533692025336920253369C4
:1008D00020002533692025336920253369202533FD
:1008E00069200025336920253369202533692025B7
:1008F00033692000424C2D4374726C20666F756E14
:1009000064200020256320202025632020202563EB
:10091000202020256320002025632020202563201F
:10092000202025632020202563200020256320200F
:10093000202D2020202D2020202D2000313000319E
:100940003100313200466C696768742D54696D65F9
:10095000202000546F74616C3A2535756D696E0006
:100960004163743A20202535756D696E00287265E3
:1009700073657429000A0D47656E65726174696E4E
:10098000672064656661756C7420506172616D6585
:1009900074657220536574202564000A0D557369CF
:1009A0006E6720506172616D657465722053657465
:1009B000202564000A0D47656E65726174696E6773
:1009C0002064656661756C74204D69786572205489
:1009D00061626C65000A0D4D697865722D436F6E1A
:1009E0006669673A202725732720282575204D6FD3
:1009F000746F727329000A0D3D3D3D3D3D3D3D3D07
:100A00003D3D3D3D3D3D3D3D3D3D3D3D3D3D3D3D16
:100A10003D3D3D3D3D3D000A0D414343206E6F7419
:100A20002063616C69627261746564210D0A000063
:100A3000008F001E01AD013B02CA025803E6037499
:100A40000402058F051B06A7063307BE074808D218
:100A5000085B09E3096B0AF20A780BFD0B810C04B1
:100A60000D860D070E870E060F840F00107B10F504
:100A7000106E11E5115B12CF124213B313231492BF
:100A800014FE146A15D3153B16A11605176717C86F
:100A90001727188318DE1837198E19E319361A87A5
:100AA0001AD61A231B6E1BB61BFD1B411C831CC3CD
:100AB0001C001D3C1D751DAB1DE01D121E421E6F4E
:100AC0001E9A1EC31EE91E0D1F2E1F4D1F691F8477
:100AD0001F9B1FB01FC31FD31FE11FEC1FF51FFB80
:100AE0001FFF1F002003010000226A000201011500
:100AF0006B01030202A96B02000303066C25326935
:100B00002E25316956002533642563202530336452
:100B10006D00537461747573004552524F523A2000
:100B200025326400253469202532693A253032693E
:100B3000002534696D25630025336920253369203C
:100B40002533692025336900253369202533692041
:100B5000253369202533690054656D7065726174B1
:100B600075726573202020200025634320202020FB
:100B700020002532692E2531695620202533692E23
:100B8000253169410025346957202536696D416852
:100B9000002532756D2F73205361743A256420004F
:100BA00020203344004E6F4678004447505300489D
:100BB0006F6D653A2533646D202533642563004EDF
:100BC0006F204E6176694374726C21000A0D77774D
:100BD000772E4D696B726F4B6F707465722E646502
:100BE0002028632920486953797374656D73204701
:100BF0006D6248000A0D74686520757365206F6624
:100C0000207468697320736F6674776172652069F8
:100C100073206F6E6C79207065726D697474656491
:100C2000200A0D6F6E206F726967696E616C204DCE
:100C3000696B726F4B6F707465722D486172647767
:100C4000617265004143542044534C004A65746905
:100C500020736174656C6C6974005370656B747299
:100C6000756D20736174656C6C697420284C6F77A6
:100C7000207265736F6C7574696F6E2900537065AF
:100C80006B7472756D20736174656C6C6974202867
:100C90003230343829005370656B7472756D20736F
:100CA0006174656C6C6974004D756C746973696707
:100CB0006E616C2050504D000A0D52656365697677
:100CC00065723A2000756E6B6E6F776E2E205573CD
:100CD000696E672050504D2E2E2E006E6F7420735B
:100CE0007570706F727465642062792068617264D7
:100CF0007761726521000A0D3D3D3D3D3D3D3D3D25
:100D00003D3D3D3D3D3D3D3D3D3D3D3D3D3D3D3D13
:100D10003D3D3D3D3D3D3D3D3D3D3D000A0D466C6B
:100D200069676874436F6E74726F6C0A0D48617204
:100D300064776172653A25642E25640A0D536F66E7
:100D400074776172653A5625642E25642563200008
:100D50000A0D3D3D3D3D3D3D3D3D3D3D3D3D3D3D26
:100D60003D3D3D3D3D3D3D3D3D3D3D3D3D3D3D3DB3
:100D70003D3D3D3D3D0011241FBECFEFD0E1DEBF24
:100D8000CDBF11E0A0E0B1E0E8E8F0EF02C00590CF
:100D90000D92A63FB107D9F718E0A6EFB1E001C068
:100DA0001D92A53DB107E1F76AEAE2E0F0E081E2D9
:100DB000809357007491AE014F5F5F4F20EF37EF84
:100DC000DA019FE0F9012F5F3F4F84918D9391509D
:100DD00097FFF8CF773911F40000FECFFA019EE0BB
:100DE000819168276095915097FFFACF888968179D
:100DF00021F0773911F40000FECF0C94C0070C9459
:100E0000000080912006E82FFF27EE0FFF1FE65B12
:100E1000F84F808191818D5E9F4F14F010920301F5
:100E2000808191818A5B9F4FCCF48091030188235C
:100E3000A9F481E080930301809163048F5F809324
:100E40006304853038F088EE93E090932902809314
:100E5000280204C066E970E00E94FA3680916304BB
:100E600099279093F1058093F00508951F93CF93F0
:100E7000DF93182F882389F082EF90E09F938F9360
:100E800084EF92E19F938F93E0912F04F0913004CF
:100E900009950F900F900F900F9080914306823329
:100EA00008F044C084EF91E00E941A17EC0111236E
:100EB00029F0CE010E9423178823D9F3C2E0D0E0A5
:100EC00026E530E080911E0190911F018217930763
:100ED00030F02196255D3F4FC730D10598F38091C2
:100EE00043069927C89F9001C99F300DD89F300DA8
:100EF0001124209300011123D9F068EC70E08C2FAD
:100F00000E94FA36DF93CF938AEF90E09F938F93FE
:100F100084EF92E19F938F93E0912F04F09130043E
:100F200009958DB79EB706968DBF02C080930001CC
:100F3000112311F1809100016AE00E946F77892FDF
:100F400099279F938F93809100010E946F77992733
:100F50009F938F9385E091E09F938F9384EF92E12D
:100F60009F938F93E0912F04F091300409952DB752
:100F70003EB7285F3F4F2DBFDF91CF911F9108955E
:100F8000CFEFD0E1DEBFCDBF8824992414B815B8C7
:100F900007EE13E00253104017FFFCCF189B06C06A
:100FA000199B02C08DE007C08BE005C0199B02C0F1
:100FB00084E101C08AE08093020181E887B93E9A0A
:100FC0008FEF88B98BE184B981E085B98EE38AB966
:100FD00087E48BB9469A84B7877F84BF809160008D
:100FE0008861809360001092600084EC99E0909397
:100FF00029028093280210921C0310921B03109266
:101000004F0710924E0710921E0310921D0310926C
:10101000200310921F0320910201243128F084EC58
:1010200094E0A0E0B0E004C08BE095E0A0E0B0E088
:101030008093960190939701A0939801B0939901A2
:101040002A3011F0243110F0289801C0289A0E940B
:1010500083170E9454170E94FC120E946C330E9456
:10106000B31A81E00E94CF2E0E94CA620E945E7570
:10107000809102018C3010F4299A01C0299878944B
:101080000E94EE2D0E94F56C809170028260809328
:101090007002109273020E941C4284EF91E00E9441
:1010A0001A178C018091700280FD05C0C8010E9452
:1010B00023178823B9F38FE191E09F938F93B4EFC7
:1010C000AB2EB2E1BB2EBF92AF92E0912F04F09114
:1010D0003004099580EA9FE00E941A178C01C0E055
:1010E000D0E00F900F900F900F90ACEEEA2EA6E09C
:1010F000FA2EF0EACF2EF6E0DF2E0E941C428091FD
:10110000700280FD05C0C8010E9423178823B9F32F
:10111000F60180811816ACF40BC00E941C4280912D
:10112000700280FD05C0C8010E9423178823B9F30F
:10113000C8010E942317882321F4F70180818823A6
:1011400064F7F701808187FF18C02196DF93CF9362
:10115000219781E391E09F938F93BF92AF92E091AB
:101160002F04F091300409958091F6018F5F8093F0
:10117000F6018DB79EB706968DBF2196E4E0F0E0AC
:10118000CE0EDF1E88E090E0E80EF91ECC30D105CF
:1011900008F4B3CFC0E0D0E009EE16E0E0EAEE2EAE
:1011A000E6E0FE2EF801838187FD1CC0F7018081F7
:1011B0001816C4F42196DF93CF93219784E391E02E
:1011C0009F938F9384EF92E19F938F93E0912F04ED
:1011D000F0913004099582E0809326028DB79EB786
:1011E00006968DBFF801838180788383219684E001
:1011F00090E0E80EF91E085F1F4FCC30D10590F249
:1012000082E591E09F938F93C4EFD2E1DF93CF9378
:10121000E0912F04F0913004099590911E06809181
:10122000F6010F900F900F900F90981728F480916F
:10123000490480618093490488E791E09F938F93EC
:10124000DF93CF93E0912F04F0913004099588EE5D
:1012500093E00E941A178C010E94B91A0F900F9008
:101260000F900F90C8010E9423178823D9F388E9B3
:1012700091E09F938F93DF93CF93E0912F04F091B0
:101280003004099580E00E94BC37809102010F90E4
:101290000F900F900F908A3011F0843110F0289841
:1012A00001C0289A80ED97E090932902809328024C
:1012B00085E5809365048EE090E00E94802C99275C
:1012C000182F00278FE090E00E94802C080F111D3E
:1012D0001093FC010093FB018AE090E00E94802CB7
:1012E0009927182F00278BE090E00E94802C080F90
:1012F000111D1093FA010093F9010F5F1F4F39F090
:101300008091FB019091FC018F5F9F4F41F41092FF
:10131000FC011092FB011092FA011092F9018091E8
:10132000F9019091FA019F938F938091FB01909125
:10133000FC019F938F938DE991E09F938F93DF93AF
:10134000CF93E0912F04F091300409958DB79EB7AB
:1013500008968DBF80EC91E09F938F93DF93CF939E
:10136000E0912F04F0913004099580912C060F90A4
:101370000F900F900F90E0912F04F091300482FFB6
:1013800007C08CEC91E09F938F93DF93CF9308C0BD
:1013900088ED91E09F938F9384EF92E19F938F93D9
:1013A00009950F900F900F900F900E94D71F88E81B
:1013B00093E1909393018093920181E08093640480
:1013C0000E943607809146060E94C4748AEE91E01E
:1013D0009F938F93DF93CF93E0912F04F09130048C
:1013E000099580ED97E00E941A178C018AEF90E032
:1013F0000E941A17EC0183E08093C8050F900F90AC
:101400000F900F908091FE018111FFCFCE010E94BD
:101410002317882339F084E690E00E941A17EC0124
:101420000E941A7680912C02882309F4D5C18091FC
:101430001001882309F4D0C110922C02809163041A
:10144000882319F00E94010702C00E94F6440E94FE
:101450001C42209102012A3011F0243110F028980A
:1014600001C0289A8091210390914904882339F082
:1014700080912103815080932103977F0AC080913E
:101480006F00806280936F0010924B0710924A07A2
:1014900098609093490480919201909193010197F3
:1014A0009093930180939201809192019091930186
:1014B000892B21F0809171028823C9F180919201DA
:1014C00090919301892BD9F40E94F92E85E090E048
:1014D000909393018093920180910206909103066C
:1014E00001969093030680930206809149048160DF
:1014F000809349048091C90582608093C9058091D9
:101500000801909109018F5F9F4F19F58091180391
:101510008823F9F080E197E29093290280932802D2
:1015200080E890E0909309018093080112C02A306E
:1015300011F0243110F0289801C0289A80912802D7
:1015400090912902892B29F4809149048E7F809300
:10155000490480912C02882309F03EC180910E013C
:10156000882311F00E949A170E943F130E947A0E5E
:10157000C8010E942317882309F42AC10C5E1F4F5B
:101580008091710290914904882339F09260909380
:1015900049048091C90582600CC09D7F90934904E5
:1015A0008091920190919301079728F08091C9054D
:1015B0008D7F8093C9058091920190919301079747
:1015C00028F0809149048E7F809349048091050121
:1015D000882321F081508093050125C080936F04FA
:1015E0001092F9021092F8021092F7021092F6028D
:1015F0001092F5021092F402809108019091090175
:101600008F5F9F4F81F480912103882361F488E9E3
:101610009AE3909329028093280280E09CE09093C3
:101620000901809308018091ED01893C48F08150C7
:101630008093ED01809149048B7F8093490430C0F1
:10164000809140088823E1F0809149048460809370
:10165000490480910801909109018F5F9F4F81F4A7
:1016600080911803882361F088E99AE39093290216
:101670008093280280E098EA909309018093080102
:1016800010920104109200041092FF031092FE03C6
:101690008FEF9FEF90936E0880936D081092ED018D
:1016A00080910001282F332780911E0190911F0106
:1016B00082179307CCF48091ED0280628093ED0253
:1016C00080910801909109018F5F9F4FC1F480E7DD
:1016D00097E1909329028093280280E093E0909311
:1016E0000901809308010BC0809128029091290282
:1016F000892B29F48091ED028F7D8093ED020E9469
:10170000D66684E08093270280911803882329F409
:101710005AEA852E55E0952E12C08091FD018F5F0B
:101720008093FD01813359F41092FD018091F701FE
:101730009091F80101969093F8018093F701089435
:10174000811C911CF2E78F16FBE09F0609F040C058
:10175000882499242091FB013091FC012F5F3F4F99
:101760003093FC012093FB018091F9019091FA01E3
:1017700001969093FA018093F901832F9927682F9E
:101780008EE090E00E94862C8091FB019091FC01FC
:101790009070682F8FE090E00E94862C8091F90174
:1017A0009091FA01892F9927682F8AE090E00E9492
:1017B000862C8091F9019091FA019070682F8BE04E
:1017C00090E00E94862C84E190E00E941A178C0120
:1017D0000E9426670E94166D80912702882309F0D7
:1017E00011CE0E94EB620ECE1F920F920FB60F9297
:1017F00011248F939F93EF93FF9380910701882388
:10180000E1F48091180290911902019690931902C7
:1018100080931802FC01E25EFA4FE081ED3019F08E
:101820008A3A910539F4109219021092180281E057
:1018300080930701E093C60004C010921902109231
:101840001802FF91EF919F918F910F900FBE0F9013
:101850001F9018951F920F920FB60F9211242F937D
:101860003F934F935F936F937F938F939F93AF9328
:10187000BF93CF93EF93FF9390E08091FE0181306F
:1018800029F48091C6008093CE00CCC08091FE01E7
:10189000823029F48091C60080937204C3C0809185
:1018A000C6008093100250911E025A3A10F0909395
:1018B0001F02809110028D3009F065C080911F02D7
:1018C000823009F060C090931F02852F99278E58AF
:1018D0009B4FFC013297408120911A0230911B02EC
:1018E000241B3109DC0111978C91281B3109C90196
:1018F0009F7090931B0280931A0246E096958795FD
:101900004A95E1F7982F935C90931C022F733070E7
:10191000235C20931D028081981729F48C9128174D
:1019200011F491E006C090E080910D028F5F8093EA
:101930000D02C0910F02CC2309F074C0992309F461
:1019400071C081E080930F02580F50930C025150E8
:10195000E52FFF27EE58FB4F8DE0808380917404C4
:10196000823509F05FC00E94D71F88E190E02CE02B
:101970000FB6F894A895809360000FBE2093600086
:10198000C09326024FC020911F02822F99278130D9
:101990009105F9F0823091051CF4892B21F040C0AB
:1019A000029711F13DC080911002833239F4809189
:1019B0000F02882319F481E080931F0280911002A6
:1019C0008093720481E080931E0280911002992717
:1019D00022C02F5F20931F02E52FFF27EE58FB4FF9
:1019E00080911002808309C0E52FFF27EE58FB4F3E
:1019F0008091100280835A3A20F45F5F50931E0258
:101A000002C010921F022091100280911A02909140
:101A10001B02820F911D90931B0280931A0202C039
:101A200010921F02FF91EF91CF91BF91AF919F91C3
:101A30008F917F916F915F914F913F912F910F9077
:101A40000FBE0F901F901895AC01A0E0B0E09D0173
:101A5000A817B90748F4EEE1F5E08191280F311D90
:101A60001196A417B507C8F33F70FD01E25EFA4F67
:101A7000C90156E0969587955A95E1F7835C808376
:101A80001196FD01E25EFA4F2F733070822F835C56
:101A90008083A15EBA4F8DE08C93109207018091F4
:101AA0001E058093C6000895A0E0B0E0EAE5FDE0E1
:101AB0000C94E8772C859D850E85BB2483E280936A
:101AC0001E059F5990931F052093200533E0E32EB8
:101AD000F12C002309F49EC0CF84D888BE016D5E2E
:101AE0007F4FA989BA890150109709F493C01097C4
:101AF000B9F0F601EB0DF11DB3949081119791F4BB
:101B0000002349F1FB016E5F7F4FDB01C080D18074
:101B10006E5F7F4F0D90BC91A02DBB24015002C081
:101B200090E019C01097B9F0F601EB0DF11DB394D8
:101B30004081119791F4002341F1FB016E5F7F4FCB
:101B4000DB01C080D1806E5F7F4F0D90BC91A02DD6
:101B5000BB24015002C040E018C01097B1F0F6015C
:101B6000EB0DF11DB3941081119781F4002371F0F6
:101B7000FB013296DB01CD90DC90BF016E5F7F4FA1
:101B8000A081B181BB24015001C010E0F701E25EE9
:101B9000FA4F892F86958695835C80830894E11C93
:101BA000F11CF701E25EFA4F892F9927837090703C
:101BB00024E0880F991F2A95E1F755279A0194E0B0
:101BC000369527959A95E1F7822B835C808308945C
:101BD000E11CF11CF701E25EFA4F4F705070440FA8
:101BE000551F440F551F812F992726E096958795FD
:101BF0002A95E1F7842B835C80830894E11CF11C17
:101C0000F701E25EFA4F1F73135C10830894E11C26
:101C1000F11C6ACFC7010E94240DE9E00C940478FE
:101C2000A3E07A2F40910C024650442309F458C097
:101C3000E72FFF27EE58FB4F80818D537F5FE72F03
:101C4000FF27EE58FB4F20812D537F5FE72FFF27A3
:101C5000EE58FB4F30813D537F5FE72FFF27EE5853
:101C6000FB4F60816D537F5F9927880F991F880F05
:101C7000991F522F52955F70582B822F99278F7082
:101C80009070F4E0880F991FFA95E1F7232F2695BD
:101C90002695282B832F992783709070E6E0880F74
:101CA000991FEA95E1F7682B41504F3FC9F0EA2FA1
:101CB000FF27EE58FB4F5083AF5F41504F3F81F0FD
:101CC000EA2FFF27EE58FB4F2083AF5F41504F3F75
:101CD00039F0EA2FFF27EE58FB4F6083AF5FA5CFA7
:101CE00085E794E090930B0280930A02A350A0939F
:101CF00009020895A2E0B0E0E0E8FEE00C94EE777F
:101D000080910F02882309F46BC40E94100E809109
:101D10007304823609F025C38091740499278037B3
:101D2000910509F4C1C081379105C4F48A36910543
:101D300009F48DC28B36910544F48B34910571F111
:101D40008636910509F46CC10CC38D36910509F4F2
:101D50007BC08E36910509F45FC003C384379105BB
:101D6000D1F1853791054CF48137910509F4A3C071
:101D70008337910509F4F1C0F4C28737910509F45E
:101D800028C2883791052CF48537910509F4E4C100
:101D9000E8C28937910509F47AC1E3C2E0910A02E9
:101DA000F0910B02808191819093340380933303EF
:101DB0002091310330913203821B930B845E9D4F3F
:101DC00068E671E00E948F77845B904090933003C7
:101DD00080932F03C6C280910C02A0910A02B09199
:101DE0000B02853140F080E1EDE4F4E00D900192CA
:101DF0008A95E1F70DC08D919D910D90BC91A02D1C
:101E000080934D0490934E04A0934F04B0935004DC
:101E100080EF809307024BC0809107018823E1F394
:101E20008DE490E09F938F9383E996E09F938F9347
:101E300081E08F938F938EE48F930E94540D8DB722
:101E40009EB707968DBF8DC2A0910A02B0910B027A
:101E50001C91113081F48DE4E3E9F6E00D900192DC
:101E60008A95E1F70E943D2D1983809149048F7E68
:101E70008093490401C01982809107018823E1F30E
:101E800081E090E09F938F93CE0101969F938F9373
:101E900081E08F938F938DE48F930E94540DADB7A3
:101EA000BEB71796ADBF5DC281E0809312028FEF7F
:101EB0008093050156C2E0910A02F0910B02E08185
:101EC0008E2F8A508A3058F48983882311F481E058
:101ED00003C0863010F085E0898361E00EC08E2F4C
:101EE00084518A3070F48983882311F481E003C01F
:101EF000863010F085E0898360E089810E94B12DF1
:101F000012C0E983EF3F19F40E94A22D89838981D1
:101F1000882311F481E003C0863010F085E08983C6
:101F200089810E94952C809107018823E1F383E742
:101F300090E09F938F938FE196E09F938F9381E042
:101F400090E09F938F93CE0101969F938F9382E0B1
:101F50008F9381E08F9381E572C120910A023091C5
:101F60000B02D9018C918150853008F040C0F901F5
:101F700081818535E1F52F5F3F4F83E7EFE1F6E0A3
:101F8000D9010D9001928A95E1F7F90182910E94A1
:101F9000D92C809160069927AA27BB27BC01CD01C7
:101FA00024EC39E040E050E00E945077DC01CB01A6
:101FB0008093D5019093D601A093D701B093D80117
:101FC000809161069927AA27BB27BC01CD010E94F9
:101FD0005077DC01CB018093D1019093D201A09383
:101FE000D301B093D4010E94A22D898301C019822C
:101FF000809107018823E1F381E090E09F938F9324
:10200000CE0101969F938F9381E08F938F9383E509
:102010008F930E94540D8DB79EB707968DBF26C033
:10202000E0910A02F0910B02E0818E2F8150853001
:1020300018F48E2F0E94952C0E94A22D89838091E6
:1020400007018823E1F381E090E09F938F93CE0115
:1020500001969F938F9381E08F938F9386E48F9364
:102060000E94540DADB7BEB71796ADBF809118034F
:10207000882329F46EE670E089810E94FA3680E0B8
:102080000E943607809146060E94C4746AC1E0919E
:102090000A02F0910B028081992787FD9095909319
:1020A0006507809364078181992787FD90959093B8
:1020B0006707809366078281992787FD90959093A3
:1020C0006907809368078381992787FD909590938E
:1020D0006B0780936A078481992787FD9095909379
:1020E0006D0780936C078581992787FD9095909364
:1020F0006F0780936E078681992787FD909590934F
:102100007107809370078781992787FD9095909339
:102110007307809372078085992787FD9095909328
:102120007507809374078185992787FD9095909313
:102130007707809376078285992787FD90959093FE
:102140007907809378078385992787FD90959093E9
:102150007B0780937A0705C1E0910A02F0910B0298
:1021600080810E94C5328A83882319F481E08983A3
:1021700001C01982809107018823E1F388E090E093
:102180009F938F9381EE96E09F938F9321E030E0B1
:102190003F932F9380910A0290910B029F938F930C
:1021A0003F932F93CE0102969F938F933F932F934C
:1021B000CE01820F931F9F938F9384E08F9381E0D2
:1021C0008F9385E58F930E94540DEDB7FEB77396FC
:1021D0003CC080910902893008F4C3C020910A02F2
:1021E00030910B022F5F3F4F88E0A1EEB6E0F9017E
:1021F00001900D928A95E1F7D9018E910E941B32D0
:102200008A83882319F481E0898301C0198280912F
:1022100007018823E1F321E030E03F932F93CE01C3
:1022200002969F938F933F932F93CE01820F931F1C
:102230009F938F9382E08F9381E08F9387E58F93B5
:102240000E94540DEDB7FEB73B96EDBF8AC00E94C9
:1022500077748983823019F0843009F082C0F89451
:102260008091C1008F738093C1008091C9008F73EA
:102270008093C9008091C100877E8093C1008091C6
:10228000C900877E8093C9008091C80087FF03C082
:102290008091CE00F9CF8091C00087FF03C080916C
:1022A000C600F9CFE0910A02F0910B0280818823E9
:1022B00059F581E08093FE011092CD0080E490E01A
:1022C0008093CC008091CD008093C5008091CC009C
:1022D0008093C4008091CA008F7D8093CA00809152
:1022E000CA008F7E8093CA008091C9008B7F809343
:1022F000C9008091CA0084608093CA008091CA009E
:1023000082608093CA0003C082E08093FE018091C6
:10231000CA00877F8093CA008091C200877F809324
:10232000C2008091C9008E7F8093C9008091C10056
:1023300088618093C1008091C90088618093C90041
:102340008091C10080688093C1008091C90080683D
:102350008093C90010926E0010926F00109270006E
:1023600078948091740499278436910509F4CDC03E
:1023700085369105ACF48136910509F481C0823629
:1023800091052CF48B34910509F45DC021C182368E
:10239000910509F482C08336910509F491C018C1F2
:1023A0008C36910509F4FFC08D3691054CF48736C3
:1023B000910509F40AC18836910509F4C4C008C121
:1023C0008437910529F08637910509F4FAC000C1D8
:1023D00080910C02A0910A02B0910B02803140F072
:1023E00080E1EDE4F4E00D9001928A95E1F70DC0F3
:1023F0008D919D910D90BC91A02D80934D04909353
:102400004E04A0934F04B093500480910701882399
:10241000E1F31F92809104018F9384E58F930E94D2
:10242000540D8AEF809307028FEF8093050180EAB5
:102430009FE00E941A17909300028093FF010F9073
:102440000F900F90C5C0E0910A02F0910B028081BD
:102450009181909334038093330320913103309121
:102460003203821B930B845E9D4F68E671E00E94ED
:102470008F77845B90409093300380932F03A8C0A4
:10248000E0910A02F0910B02808180930601803274
:1024900098F08FE1809306010FC0A0910A02B091DD
:1024A0000B028BE0E5E6F4E00D9001928A95E1F7EE
:1024B00080916E0480930A068FEF8093050188C097
:1024C0008091030290910402892B89F4E0910A0221
:1024D000F0910B02E081EE2351F08AE0E89FC00109
:1024E00011240E941A179093400480933F04E091B6
:1024F0000A02F0910B0290818AE0989FC00111249A
:10250000909304028093030215C08FEF809305011E
:10251000E0910A02F0910B0290818AE0989FC0013D
:1025200011249093060280930502892B19F081E013
:102530008093140280EA9FE00E941A179093000291
:102540008093FF0145C08FEF80930501E0910A025F
:10255000F0910B02908197FD08C082E080931102F8
:1025600010920202109201021AC0909580916902A5
:10257000892B8093690291818AE0989FC001112480
:10258000909302028093010284E08093110280EA1A
:102590009FE00E941A17909300028093FF0181E050
:1025A0008093150215C08FEF80930501E0910A0218
:1025B000F0910B02808180936A0281E08093160281
:1025C00007C081E08093130203C081E0809317026B
:1025D00010920F0210920B0210920A02109209023E
:1025E000E3E0CE5F0C940A78982F8091C00085FFBD
:1025F000FCCF9093C60008950F931F9388E18093BA
:10260000C1008091C00082608093C0008091C100B1
:1026100080688093C1008091C10080648093C10074
:1026200000E010E00093C5008AE290E08093C400CF
:1026300080910502909106020E941A17909342041D
:10264000809341048CED90E00E941A1790937104DE
:10265000809370041092430482E5809344041092A6
:1026600047048BE0809345041092460410930B02BC
:1026700000930A02109209021F910F910895A0E1A0
:10268000B0E0E5E4F3E10C94EB7780910701882357
:1026900009F4C1C28091FF01909100020E942317AA
:1026A000882361F010920202109201021092060239
:1026B000109205021092040210920302809101020E
:1026C00090910202892B41F080911C0590911D058B
:1026D0000E942317882329F480911502882309F486
:1026E00060C080910701882309F45BC080911102CA
:1026F00001E211E08430A8F00E94EB1F80E590E039
:102700009F938F931F930F9381E08F938F9388E410
:102710008F930E94540D2DB73EB7295F3F4F2DBFB9
:1027200034C010926B0282E194E09F938F9380EE0D
:102730009FE19F938F93E0912F04F09130040995CE
:1027400084E190E09F938F931F930F9381E090E03B
:102750009F938F9381E192E09F938F9382E08F9379
:1027600081E08F9388E48F930E94540D8091110231
:10277000982F8F5F809311022DB73EB7215F3F4F97
:102780002DBF943010F010921102809101029091AF
:1027900002020E941A1790931D0580931C05109247
:1027A000150280911602882351F180910701882338
:1027B00031F10E94EB1F80E590E09F938F9381E2BF
:1027C00091E09F938F9321E030E03F932F9380E23D
:1027D00091E09F938F933F932F938AE692E09F938C
:1027E0008F9383E08F9381E08F938CE48F930E948B
:1027F000540D109216028DB79EB70F968DBF809123
:1028000013028823D1F0809107018823B1F08AE078
:1028100090E09F938F9383E494E09F938F9381E064
:102820008F938F9386E58F930E94540D109213021D
:102830002DB73EB7295F3F4F2DBF809117028823E8
:10284000D9F0809107018823B9F08BE090E09F9345
:102850008F9385E694E09F938F9381E08F9380918F
:1028600004018F9387E48F930E94540D10921702F6
:102870008DB79EB707968DBF8091700490917104BB
:102880000E942317882309F461C0809107018823DF
:1028900009F45CC080913B069927880F991F880F27
:1028A000991F7C010027F7FC0095102F809175037C
:1028B00090917603A0917703B0917803BC01CD018C
:1028C000A80197010E94C47730935E0420935D04B1
:1028D00080916D0390916E03A0916F03B09170038E
:1028E000BC01CD01A80197010E94C4773093600418
:1028F00020935F048091020380936104809101031F
:102900008093620488E090E09F938F938DE594E03C
:102910009F938F9381E08F9383E08F938BE68F93C8
:102920000E94540D809163042DB73EB7295F3F4F3D
:102930002DBF853018F086E08093630483E690E035
:102940000E941A179093710480937004809105027D
:1029500090910602892B41F08091410490914204AC
:102960000E942317882321F480911402882339F1CF
:1029700080910701882319F10E94E83582E490E0F4
:102980009F938F9388EC95E09F938F9381E08F9333
:102990008F9384E48F930E94540D109214028DB78C
:1029A0009EB707968DBF8091050290910602009711
:1029B00031F00E941A179093420480934104809151
:1029C000030290910402892B09F4B8C080913F045E
:1029D000909140040E942317882309F4AFC080918E
:1029E0000701882309F4AAC080913B069927880F24
:1029F000991F880F991F7C010027F7FC0095102F65
:102A00008091750390917603A0917703B09178033C
:102A1000BC01CD01A80197010E94C4773093320414
:102A20002093310480916D0390916E03A0916F0308
:102A3000B0917003BC01CD01A80197010E94C47739
:102A400030933404209333042091260830912708D2
:102A50004091280850912908DA01C90163E0880FE4
:102A6000991FAA1FBB1F6A95D1F7820F931FA41F3E
:102A7000B51F820F931FA41FB51F2091960130919F
:102A800097014091980150919901BC01CD010E949C
:102A9000C477309336042093350480913D039091A0
:102AA0003E03A0913F03B091400339E0B595A7954F
:102AB000979587953A95D1F780933704809139039C
:102AC00090913A03A0913B03B0913C0329E0B59566
:102AD000A795979587952A95D1F78093380480918B
:102AE000450390914603A0914703B091480309E044
:102AF000B595A795979587950A95D1F78093390451
:102B00008EE090E09F938F9381E394E09F938F9367
:102B100081E08F938F9383E48F930E94540D809173
:102B20000302909104020E941A179093400480932C
:102B30003F042DB73EB7295F3F4F2DBF809106015F
:102B40008F3F71F1992714E0880F991F1A95E1F7CB
:102B50008E5E9D4F40E150E0BC01CE0101960E9487
:102B60007E7680E190E09F938F93CE0101969F93B4
:102B70008F9381E090E09F938F9386E091E09F9305
:102B80008F9382E08F9381E08F9381E48F930E94F3
:102B9000540D8FEF809306018DB79EB70B968DBFB6
:102BA00080910A068823D1F0809107018823B1F033
:102BB00081E090E09F938F938AE096E09F938F93BC
:102BC00081E08F938F9382E48F930E94540D109233
:102BD0000A062DB73EB7295F3F4F2DBF80911202E5
:102BE0008823C9F0809107018823A9F084E390E04D
:102BF0009F938F938AE497E09F938F9381E08F93C5
:102C00008F9380E58F930E94540D109212028DB71E
:102C10009EB707968DBFE6E0C05F0C9407781F92C1
:102C20000F920FB60F9211242F933F935F936F93E0
:102C30007F938F939F93AF93BF93EF93FF9320E086
:102C400080912702882329F0809127028150809368
:102C5000270280911204882319F081508093120476
:102C600080912F02815080932F028F3F09F05BC02B
:102C700089E080932F0280912D0290912E0201967F
:102C800090932E0280932D0280910F018F5F8170AF
:102C900080930F01882319F481E080932C023499EA
:102CA00003C081E080933002809128029091290234
:102CB000892B21F180912802909129020B9750F0E5
:102CC00080912802909129020A979093290280937B
:102CD000280204C010922902109228028091280232
:102CE00090912902209108013091090182239323B8
:102CF000892B11F021E008C020E006C08FEF9FEF84
:102D0000909309018093080180910201222331F000
:102D10008A3011F45A9A07C0479A05C08A3011F4D4
:102D20005A9801C0479880913002882309F472C0F4
:102D30002091ED01222309F06DC080912C0683FFC4
:102D400069C086B19927FC01E071F07084FF14C05E
:102D500080912A0290912B02019690932B028093EE
:102D60002A0280912A0290912B02895E934008F4F6
:102D700051C0209330024EC080912A0290912B02C4
:102D8000892B09F443C080912A0290912B028A5624
:102D90009140E0F580912A0290912B0269E270E067
:102DA0000E947B7780912A0290912B02860F971FB9
:102DB00090932B0280932A0280912A0290912B02F9
:102DC0000B9750F080912A0290912B020A979093D2
:102DD00034038093330304C0F0933403E09333034C
:102DE0008091330390913403209131033091320369
:102DF000821B930B845E9D4F68E671E00E948F7783
:102E0000845B90409093300380932F0310922B02A9
:102E100010922A02FF91EF91BF91AF919F918F91F4
:102E20007F916F915F913F912F910F900FBE0F9007
:102E30001F90189520912D0230912E02280F391FD6
:102E4000C9010196089520912D0230912E02821B16
:102E5000930B892F99278695807490700895CF934E
:102E6000DF930E941A17EC01CE010E9423178823DA
:102E7000D9F3DF91CF910895CF93DF930E941A1772
:102E8000EC0109C080911001882329F09093100172
:102E90008FEC80937A00CE010E942317982F88230D
:102EA00089F3DF91CF9108959FB7F8945F983E9A88
:102EB000469A8091B0008F708093B0008091B000EE
:102EC00083608093B0008091B1008B738093B100D8
:102ED0008091B1008B608093B1001092B2008FEFAF
:102EE0008093B3008091B00080688093B00080919F
:102EF00070008A7F80937000809170008260809360
:102F000070009FBF08958AE090E00E941A17909386
:102F100036028093350282E085BD83EA84BD17BC0A
:102F200084EB88BD86E086BD80916E0081608093D1
:102F30006E000895A0E0B0E0E0EAF7E10C94EA77D3
:102F400080915606E82FFF27E456FE4F9681D080E9
:102F500080910E01A92FBB27A7FDB095CB2FDB2FAA
:102F6000813009F0C9C020917503309176034091FA
:102F7000770350917803BD01CE010E94507797FFEF
:102F800004C061587F4F8F4F9F4F7B018C0167E0DA
:102F900015950795F794E7946A95D1F78D2D9927A4
:102FA00087FD9095A92FB92F20916D0330916E0365
:102FB00040916F0350917003BC01CD010E94507786
:102FC00097FF04C061587F4F8F4F9F4F57E09595F3
:102FD0008795779567955A95D1F7F801E701C61B54
:102FE000D70BE80BF90B80914D069927AA27BB2731
:102FF000BC01CD019E01AF010E94507797FF04C034
:1030000061507E4F8F4F9F4FFC01EB0149E0F595DA
:10301000E795D795C7954A95D1F78091C101992732
:1030200036E0880F991F3A95E1F740910C015091D5
:103030000D01209155063327841B950BB9010E9481
:103040008F7780910C0190910D01860F971F9093BF
:103050000D0180930C0180910C0190910D0197FD61
:103060000F9624E0959587952A95E1F79093230292
:10307000809322028091840680FF07C08091220203
:10308000909123028C0F9D1F06C080912202909187
:1030900023028C1B9D0B909323028093220280912C
:1030A0004E06282F3327220F331F220F331F809104
:1030B000220290912302821793077CF080914F06A1
:1030C000282F3327220F331F220F331F8091220214
:1030D000909123022817390724F430932302209378
:1030E000220280910201843108F4C2C080910E0155
:1030F0008F5F80930E01BEC020916D0330916E03EF
:1031000040916F0350917003BD01CE010E94507732
:1031100097FF04C061587F4F8F4F9F4F7B018C01F9
:10312000C7E015950795F794E794CA95D1F78D2DCB
:10313000992787FD9095A92FB92F2091750330917C
:1031400076034091770350917803BC01CD010E9432
:1031500050779B01AC0197FF04C021583F4F4F4F60
:103160005F4FB7E05595479537952795BA95D1F7B5
:103170002E0D3F1D401F511F809151069927AA27F0
:10318000BB27BC01CD010E94507797FF04C061505E
:103190007E4F8F4F9F4FFC01EB01A9E0F595E7951E
:1031A000D795C795AA95D1F78091C001992776E068
:1031B000880F991F7A95E1F740910A0150910B0110
:1031C000209155063327841B950BB9010E948F77F8
:1031D00080910A0190910B01860F971F90930B012C
:1031E00080930A0180910A0190910B0197FD0F963F
:1031F00064E0959587956A95E1F790932102809315
:1032000020028091840681FF07C080912002909166
:1032100021028C0F9D1F06C08091200290912102F7
:103220008C1B9D0B9093210280932002809152066B
:10323000282F3327220F331F220F331F80912002A4
:1032400090912102821793077CF080915306282FDA
:103250003327220F331F220F331F809120029091BA
:1032600021022817390724F43093210220932002E9
:1032700010920E01E7E0CDB7DEB70C9406781F92EE
:103280000F920FB60F9211242F933F934F935F939A
:103290008F939F93EF93FF9380910201909131025E
:1032A000843108F04CC0992309F01CC18091B00012
:1032B00086FF24C08091B0008F7B8093B000809106
:1032C00022029091230287559E4F9093250280936E
:1032D000240225E08D3D920718F08CED95E005C0A5
:1032E0008757914030F487E791E0909325028093CF
:1032F00024028091240290912502BAC08091B000EE
:1033000080648093B00080915406282F33278DED80
:1033100096E0289FA001299F500D389F500D112441
:10332000CA012091320230913302821B930B909399
:1033300025028093240281E080930E01D0C099235E
:1033400009F0D0C08091B00086FF97C08091B00096
:103350008F7B8093B000E0913402EE23F1F48091F2
:103360005406282F33278DED96E0289FA001299F32
:10337000500D389F500D1124CA0120913202309116
:103380003302821B930B90932502809324021092A8
:10339000330210923202469AA2C089EA93E09093D7
:1033A0002502809324028E2F992783309105D9F02E
:1033B0008430910534F48130910549F0029761F031
:1033C00020C08430910591F0059799F01AC0809142
:1033D00022029091230204C0809120029091210248
:1033E00087559E4F1DC08091E50705C08091BB07A2
:1033F00002C08091F0079927880F991F880F991FA5
:10340000EFCFFF27EE0FFF1FE65BF84F20813181E2
:10341000220F331F8091240290912502820F931F67
:10342000909325028093240280912402909125029A
:1034300055E08D3D950718F08CED95E005C0875758
:10344000914030F487E791E0909325028093240225
:1034500020912402309125022C5B304030932502CC
:10346000209324028091320290913302820F931FA5
:10347000909333028093320232C08091B000806416
:103480008093B0008CEB90E090932502809324020F
:10349000809132029091330284549F4F9093330273
:1034A0008093320280912602882321F080912103AB
:1034B000833320F480912602823011F4469801C0B3
:1034C000469A809134028F5F809334029091540623
:1034D000981728F481E080930E011092340281E065
:1034E00080933102209124023091250241E02F3750
:1034F000340730F08FEF8093B3002F5F30400FC060
:103500002F3F3105C9F0C0F0A9014F5F50404F3740
:10351000510550F480E88093B30020583040309338
:1035200025022093240212C08FEF8093B3005093A2
:103530002502409324020AC0809124028093B300A4
:10354000109225021092240210923102FF91EF9105
:103550009F918F915F914F913F912F910F900FBE4F
:103560000F901F90189510927C008FEC80937A003A
:103570000895CF93DF9310923B0283E090E00E9486
:10358000802CC82FDD27C531D10508F02A97C7BD8B
:1035900084E690E00E943C178091140190911501FF
:1035A0008052934010F4C0E0D0E0CA3FD105F8F457
:1035B000C7BD82E390E00E943C1787E294E09F93AE
:1035C0008F9384EF92E19F938F93E0912F04F0917A
:1035D0003004099580911401909115010F900F907E
:1035E0000F900F908052934010F02196DECFC09341
:1035F0001B066C2F83E090E00E94862C80912C06A5
:1036000080FF0AC080911B068A508B3E28F0809173
:103610004804806480934804C7BD8CE291E00E9416
:103620003C17DF91CF910895EF92FF921F93CF93B4
:1036300010E080ED97E00E941A177C01CCE813306F
:1036400019F4CB3008F0C9E010E080914B02909162
:103650004C028C5F934024F48091130181500AC086
:1036600080914B0290914C028750944034F08091AD
:1036700013018F5F8093130101C011E08091490213
:1036800090914A028C5F934024F480911201815002
:103690000AC08091490290914A028750944034F0C8
:1036A000809112018F5F8093120101C01F5F809192
:1036B0004702909148028C5F934024F4809111015D
:1036C00081500AC0809147029091480287509440EF
:1036D000C4F0809111018F5F8093110113C089E2C2
:1036E00094E09F938F9384EF92E19F938F93E09167
:1036F0002F04F091300409950F900F900F900F90C8
:103700005FC01F5F82E180937602809170028E7F9E
:103710008093700285EA8093BC00809113018A3007
:1037200040F4809148048160809348048AE080934B
:10373000130180911301863F40F08091480481601D
:103740008093480485EF80931301809112018A30A1
:1037500040F4809148048260809348048AE080931A
:10376000120180911201863F40F0809148048260EE
:103770008093480485EF80931201809111018A3073
:1037800040F4809148048460809348048AE08093E8
:10379000110180911101863F40F0809148048460BE
:1037A0008093480485EF80931101809176028823ED
:1037B00039F0C7010E942317882309F090CFF5CF75
:1037C000109210018FEC80937A0080911001882371
:1037D000E1F3CA3020F48AE090E00E943C17C15027
:1037E00009F02DCF86E490E00E943C17CF911F9105
:1037F000FF90EF9008951F920F920FB60F92112431
:10380000AF92BF92CF92DF92EF92FF920F931F93EE
:103810002F933F934F935F936F937F938F939F93D8
:10382000AF93BF93EF93FF9380915402282F3327D8
:10383000442755278F5F80935402F90122313105C7
:1038400008F08CC3E25CFF4F0C94167880917800EE
:103850009091790046C080917800909179002CC1B8
:10386000809178009091790090935702809356024E
:1038700057C180917E0390917F0320917800309111
:103880007900821B930B90930C0680930B0680911A
:103890000B0690910C0690936102809360025EC1CA
:1038A000809178009091790020918003309181037C
:1038B000821B930B90931A06809319068091190628
:1038C00090911A06909363028093620249C380919B
:1038D0005A0290915B022091780030917900820F1A
:1038E000931F90935B0280935A0281E03AC38091C8
:1038F0005802909159022091780030917900820FFE
:10390000931F909359028093580284E02AC38091B8
:103910001E0190911F019C01220F331F280F391F98
:10392000809178009091790063E070E00E947B774D
:10393000260F371F369527953695279530931F010B
:1039400020931E0185E00DC380917800909179004D
:1039500040917A0350917B03841B950B9093420214
:10396000809341028091410290914202029704F1BA
:1039700022E04E3E520784F4209155022B5F2093A3
:10398000550225508091EE029091EF02845F9140A4
:1039900018F4215F2093550280915502853684F1F9
:1039A0004F5F5F4F50937B0340937A03845626C04A
:1039B00080914102909142028F5F9F4F0CF532E05F
:1039C00047325307ECF020915502255020935502C1
:1039D0002B5F8091EE029091EF02845F914018F48A
:1039E0002F5020935502809155028C394CF4415050
:1039F000504050937B0340937A038C598093550237
:103A000081E08093400280917800909179009093BA
:103A100012068093110680914102909142029C010E
:103A2000442737FD4095542F8091350390913603FC
:103A3000A0913703B0913803820F931FA41FB51FC5
:103A40008093350390933603A0933703B0933803E4
:103A5000209135033091360340913703509138035C
:103A600057FF04C021503C4F4F4F5F4F0AE0559520
:103A70004795379527950A95D1F780913503909111
:103A80003603A0913703B0913803821B930BA40B2C
:103A9000B50B8093350390933603A0933703B0930F
:103AA00038032EC1809158029091590220917800DC
:103AB00030917900820F931F90935902809358029E
:103AC0001092530250C2809102018A3071F48091A9
:103AD0007800909179002091560230915702820F20
:103AE000931F01969695879517C040915602509165
:103AF0005702843158F02091780030917900240FDA
:103B0000351F8FEF97E0821B930B06C080917800E2
:103B100090917900840F951F9093480280934702FB
:103B200086E01FC280917E0390917F0320917800F0
:103B300030917900821B930B90930C0680930B06B7
:103B400080910B0690910C062091600230916102E9
:103B5000820F931F909346028093450287E001C233
:103B600080917800909179002091800330918103B9
:103B7000821B930B90931A06809319068091190665
:103B800090911A062091620230916302820F931F76
:103B90009093440280934302E3C120915A023091F2
:103BA0005B028091780090917900280F391F309343
:103BB0005B0220935A02809102018A3019F4220F8D
:103BC000331F04C0220F331F220F331F30935B02B9
:103BD00020935A0220915A0230915B02C90137FDAD
:103BE0000796A3E095958795AA95E1F790934C02E7
:103BF00080934B0280915C0290915D02820F931F33
:103C000097FD01969595879590935D0280935C0250
:103C100020918A0330918B03821B930B90931D019B
:103C200080931C01209151023091520280911C011D
:103C300090911D01280F391F37FF02C02F5F3F4FA2
:103C40003595279530935202209351024ECE209104
:103C50005802309159028091780090917900280F94
:103C6000391F3093590220935802809102018A3003
:103C700019F4220F331F04C0220F331F220F331FEA
:103C800030935902209358022091580230915902E2
:103C9000C90137FD079663E0959587956A95E1F729
:103CA00090934A028093490280915E0290915F0254
:103CB000820F931F97FD01969595879590935F02CC
:103CC00080935E022091880330918903821B930BBD
:103CD00090931B0180931A0120914F023091500262
:103CE00080911A0190911B01280F391F37FF02C0E4
:103CF0002F5F3F4F359527953093500220934F0209
:103D000083E02FC11092540281E0809310018091D2
:103D100037029091380201969093380280933702CF
:103D2000809178009091790090931501809314010F
:103D30008091140190911501AA27BB27A0906402DD
:103D4000B0906502C0906602D0906702A80EB91EBE
:103D5000CA1EDB1EA0926402B0926502C092660287
:103D6000D0926702809168028F5F809368028231EF
:103D700008F4F6C08091160190911701A0911801E6
:103D8000B09119017C018D0123E0EE0CFF1C001F96
:103D9000111F2A95D1F7E81AF90A0A0B1B0BEA0C36
:103DA000FB1C0C1D1D1D80913B02992787FD9095E2
:103DB000A92FB92FBC01CD0126EC34E240E050E040
:103DC0000E945077DC01CB01E81AF90A0A0B1B0BA1
:103DD000D801C7010496A11DB11DB7FF05C0D801C8
:103DE000C7010B96A11DB11D13E0B595A795979539
:103DF00087951A95D1F78093160190931701A09398
:103E00001801B093190180911306909114067C015A
:103E10000027F7FC0095102F809116019091170153
:103E2000A0911801B0911901E81AF90A0A0B1B0BAD
:103E3000E0921303F09214030093150310931603FA
:103E400020913C0230913D0240913E0250913F0250
:103E500057FF04C0215F3F4F4F4F5F4FF4E0559530
:103E6000479537952795FA95D1F780913C02909127
:103E70003D02A0913E02B0913F02821B930BA40B26
:103E8000B50B80933C0290933D02A0933E02B09309
:103E90003F0280913C0290913D02A0913E02B09180
:103EA0003F028E0D9F1DA01FB11F80933C02909377
:103EB0003D02A0933E02B0933F028091390290915F
:103EC0003A02AC01E5E0440F551FEA95E1F7481BC3
:103ED000590B80913C0290913D02A0913E02B0911D
:103EE0003F02B7FF03C00F96A11DB11D74E0B59549
:103EF000A795979587957A95D1F7209113033091DF
:103F00001403281B390B63E0220F331F6A95E1F776
:103F1000240F351F37FF02C0215E3F4F45E0359526
:103F200027954A95E1F730933A0220933902D6015A
:103F3000C501D7FE03C00196A11DB11DB595A7957A
:103F4000979587958093640290936502A09366028B
:103F5000B093670289E08093680202C01092540215
:103F600082E0809353028091530280937C00809181
:103F70005402882319F08FEC80937A00FF91EF911F
:103F8000BF91AF919F918F917F916F915F914F9171
:103F90003F912F911F910F91FF90EF90DF90CF9065
:103FA000BF90AF900F900FBE0F901F90189590E2AA
:103FB000E1E2F1E08FE49193815087FFFCCF089517
:103FC00090916B02E1E2F1E0E90FF11D80839F5FC8
:103FD00090936B020895EF92FF920F931F93CF93EC
:103FE000DF932091690220FF0AC080916A02882332
:103FF00011F0815002C08091200180936A0221FF5C
:104000000CC090916A0280912001981719F41092C7
:104010006A0203C09F5F90936A02822F992780FFF4
:1040200004C081FF02C010926A020E94D71F8091D3
:104030006A02282F332750EEE52E5FE1F52EC0915E
:104040002F04D09130048A3098F481E180936B0280
:104050003F932F9380E694E09F938F93FF92EF928C
:10406000FE0109952DB73EB72A5F3F4F2DBF11C006
:1040700080E180936B023F932F9385E694E09F93BA
:104080008F93FF92EF92FE0109958DB79EB706962A
:104090008DBF20916A02822F9927AA27BB27FC0196
:1040A000429710F00C949C2AE05BFF4F40EEE42E08
:1040B0004FE1F42EC0912F04D09130040C94167867
:1040C00010926B028AE694E09F938F9300EE1FE1BB
:1040D000FF92EF92FE01099584E180936B020F90AD
:1040E0000F900F900F9081E690E09F938F9382E561
:1040F00090E09F938F931F921F92809102016AE03C
:104100000E946F77892F99279F938F938091020147
:104110000E946F7799279F938F938AE794E09F93EC
:104120008F93FF92EF92E0912F04F0913004099564
:1041300088E280936B022DB73EB7225F3F4F2DBFC1
:1041400084E996E09F938F930E94A22D99279F93D5
:104150008F938FE894E09F938F93FF92EF92E0917B
:104160002F04F091300409958DB79EB708968DBF46
:1041700090914804992351F08CE380936B02892F2E
:1041800099279F938F938DE994E081C69091710256
:10419000992371F08CE380936B02892F99279F9369
:1041A0008F9384EB94E09F938F931F930F9391C011
:1041B0008091490484FF07C08CE380936B0289ECF3
:1041C00094E00C942E2A809192019091930106978D
:1041D00010F00C94A52A8CE380936B0286ED94E09A
:1041E0000C942E2A80912C0630EEE32E3FE1F32E24
:1041F000C0912F04D091300480FF74C010926B02E4
:104200008091130390911403A0911503B0911603AC
:10421000BC01CD0125E030E040E050E00E94C477D1
:104220003F932F9383EE94E09F938F93FF92EF92AF
:10423000FE01099584E180936B022DB73EB72A5F9A
:104240003F4F2DBF80910F0390911003A091110358
:10425000B0911203BC01CD0125E030E040E050E018
:104260000E94C4773F932F9380EF94E09F938F93A6
:10427000FF92EF92E0912F04F0913004099588E2CB
:1042800080936B028DB79EB706968DBF8091140107
:10429000909115019F938F938DEF94E09F938F934F
:1042A000FF92EF92E0912F04F091300409958CE396
:1042B00080936B022DB73EB72A5F3F4F2DBF87B566
:1042C00099279F938F938AE095E09F938F93FF9216
:1042D000EF92E0912F04F091300409958DB79EB7CD
:1042E000069633C710926B0287E195E09F938F93F8
:1042F000FF92EF92FE01099584E180936B020F908B
:104300000F900F900F9086E295E09F938F93FF920E
:10431000EF92E0912F04F0913004099588E28093A8
:104320006B020F900F900F900F908FE295E09F938C
:104330008F93FF92EF92E0912F04F0913004099552
:104340008CE380936B020F900F900F900F908EE391
:1043500095E09F938F93FF92EF920C94322A1092E4
:104360006B0287E495E09F938F9300EE1FE1FF922D
:10437000EF92FE01099584E180936B020F900F90FC
:104380000F900F908091750390917603A091770321
:10439000B0917803B7FF04C081509C4FAF4FBF4F1F
:1043A0002AE0B595A795979587952A95D1F7BF935C
:1043B000AF939F938F9384E595E09F938F931F9383
:1043C0000F93E0912F04F0913004099588E28093D7
:1043D0006B022DB73EB7285F3F4F2DBF80916D0315
:1043E00090916E03A0916F03B0917003B7FF04C06A
:1043F00081509C4FAF4FBF4FCAE0B595A795979599
:104400008795CA95D1F7BF93AF939F938F9383E618
:1044100095E09F938F931F930F93E0912F04F0915A
:10442000300409958CE380936B028DB79EB7089694
:104430008DBF80913303909134039F938F9382E7D4
:1044400095E09F938F931F930F93E0912F04F0912A
:10445000300409952DB73EB72A5F3F4F11C7109220
:104460006B0280914E0790914F079F938F9380919D
:104470004C0790914D079F938F9381E895E09F9310
:104480008F93FF92EF92FE01099584E180936B0276
:104490008DB79EB708968DBF8091520790915307B4
:1044A0009F938F9380915007909151079F938F9383
:1044B00081E995E09F938F93FF92EF92E0912F0413
:1044C000F0913004099588E280936B022DB73EB7D6
:1044D000285F3F4F2DBF80915607909157079F93BC
:1044E0008F9380915407909155079F938F9381EA02
:1044F00095E09F938F93FF92EF92E0912F04F091BC
:10450000300409958CE380936B028DB79EB70896B3
:104510008DBF80915A0790915B079F938F938091F5
:104520005807909159079F938F9381EB95E0A2C014
:1045300010926B0280912106E82FFF27EE0FFF1FDC
:10454000E65BF84F808191819F938F938091200645
:10455000E82FFF27EE0FFF1FE65BF84F8081918168
:104560009F938F9381EC95E09F938F93FF92EF92AF
:10457000FE01099584E180936B028DB79EB7089682
:104580008DBF80912306E82FFF27EE0FFF1FE65B0C
:10459000F84F808191819F938F9380912206E82F1D
:1045A000FF27EE0FFF1FE65BF84F8081918188584F
:1045B0009F4F9F938F9381ED95E09F938F93FF92F1
:1045C000EF92E0912F04F0913004099588E28093F6
:1045D0006B022DB73EB7285F3F4F2DBF8091250658
:1045E000E82FFF27EE0FFF1FE65BF84F80819181D8
:1045F00082599F4F9F938F9380912406E82FFF2726
:10460000EE0FFF1FE65BF84F8081918182599F4F2B
:104610009F938F9381EE95E09F938F93FF92EF92FC
:10462000E0912F04F091300409958CE380936B02A4
:104630008DB79EB708968DBF80912706E82FFF277C
:10464000EE0FFF1FE65BF84F8081918182599F4FEB
:104650009F938F9380912606E82FFF27EE0FFF1F71
:10466000E65BF84F8081918182599F4F9F938F9392
:1046700081EF95E09F938F93FF92EF92E0912F044B
:10468000F091300409952DB73EB7285F3F4FF8C52C
:1046900010926B0281E096E09F938F9300EE1FE1F2
:1046A000FF92EF92FE010995809102010F900F9009
:1046B0000F900F908A3009F09DC084E180936B02C7
:1046C00080918A0390918B039C0197FF02C0295F20
:1046D0003F4F287F821B930B9F938F9380918A0378
:1046E00090918B0397FD0796A3E095958795AA95E2
:1046F000E1F79F938F9320918A0330918B0337FFCB
:1047000002C0295F3F4FF3E035952795FA95E1F711
:1047100080914B0290914C02821B930B9F938F933D
:104720008FE096E09F938F931F930F93E0912F0458
:10473000F0913004099588E280936B028DB79EB7A3
:104740000A968DBF80918803909189039C0197FF01
:1047500002C0295F3F4F287F821B930B9F938F934B
:10476000809188039091890397FD0796E3E09595E2
:104770008795EA95E1F79F938F9320918803309175
:10478000890337FF02C0295F3F4F73E035952795B6
:104790007A95E1F78091490290914A02821B930B2E
:1047A0009F938F9380E296E09F938F931F930F9335
:1047B000E0912F04F091300409958CE380936B0213
:1047C0002DB73EB7265F3F4F2DBF80918603909156
:1047D00087039F938F938091860390918703209105
:1047E000470230914802821B930B9F938F9381E382
:1047F00096E0A7C38B3019F0843108F4ADC084E192
:1048000080936B0280918A0390918B039C0197FFA8
:1048100002C0215F3F4F207F821B930B97FD0196C3
:10482000959587959F938F9380918A0390918B03A1
:1048300097FD0F9654E0959587955A95E1F79F93CC
:104840008F9320918A0330918B0337FF02C0295F39
:104850003F4F43E0359527954A95E1F780914B020C
:1048600090914C02821B930B9F938F938FE396E062
:104870009F938F931F930F93E0912F04F091300437
:10488000099588E280936B022DB73EB7265F3F4FB4
:104890002DBF80918803909189039C0197FF02C0EE
:1048A000215F3F4F207F821B930B97FD01969595CB
:1048B00087959F938F93809188039091890397FDAB
:1048C0000F96C4E095958795CA95E1F79F938F93CE
:1048D000209188033091890337FF02C0295F3F4F41
:1048E000B3E035952795BA95E1F78091490290910B
:1048F0004A02821B930B9F938F9381E596E09F93CF
:104900008F931F930F93E0912F04F091300409953A
:104910008CE380936B028DB79EB70A968DBF809112
:1049200086039091870397FD0196959587959F93B0
:104930008F93809186039091870320914702309155
:104940004802821B930B9F938F9383E696E09F937D
:104950008F931F930F9392CE8D3009F0F6C584E1AB
:1049600080936B028091130199279F938F9380917D
:104970008A0390918B0397FD0F96F4E095958795A8
:10498000FA95E1F79F938F9320918A0330918B03DF
:1049900037FF02C0295F3F4FE3E035952795EA9541
:1049A000E1F780914B0290914C02821B930B9F93F5
:1049B0008F9382E796E09F938F931F930F93E091DD
:1049C0002F04F0913004099588E280936B028DB733
:1049D0009EB70A968DBF8091120199279F938F935E
:1049E000809188039091890397FD0F9674E09595C7
:1049F00087957A95E1F79F938F9320918803309163
:104A0000890337FF02C0295F3F4F63E03595279543
:104A10006A95E1F78091490290914A02821B930BBB
:104A20009F938F9386E896E09F938F931F930F93A6
:104A3000E0912F04F091300409958CE380936B0290
:104A40002DB73EB7265F3F4F2DBF809111019927AB
:104A50009F938F93809186039091870397FD019692
:104A6000959587959F938F93809186039091870367
:104A70002091470230914802821B930B9F938F93A2
:104A80008AE996E09F938F931F930F93E0912F04F1
:104A9000F091300409958DB79EB70A9656C31092CF
:104AA0006B028EEA96E09F938F93FF92EF92FE0146
:104AB000099584E180936B020F900F900F900F90F7
:104AC00080918003909181039F938F938091430203
:104AD000909144029F938F938BEB96E09F938F93DB
:104AE000FF92EF92E0912F04F0913004099588E253
:104AF00080936B022DB73EB7285F3F4F2DBF80914B
:104B00007E0390917F039F938F93809145029091B4
:104B100046029F938F938AEC96E09F938F93FF9228
:104B2000EF92E0912F04F091300409958CE380938B
:104B30006B028DB79EB708968DBF80917A039091D6
:104B40007B039F938F9380914102909142029F93A8
:104B50008F9389ED96E08ECD10926B0280911E01AD
:104B600090911F016AE070E00E948F779F938F936E
:104B700080911E0190911F016AE070E00E948F7782
:104B80007F936F9388EE96E09F938F93FF92EF92BF
:104B9000FE01099584E180936B028DB79EB708965C
:104BA0008DBF80919F089091A0086AE070E00E94FC
:104BB0007B779F938F9380919F089091A0086AE0E4
:104BC00070E00E947B777F936F938CEF96E09F93CA
:104BD0008F93FF92EF92E0912F04F09130040995AA
:104BE00088E280936B022DB73EB7285F3F4F2DBF01
:104BF0008091A1089091A2089F938F9380E197E004
:104C00009F938F93FF92EF92E0912F04F0913004E5
:104C100009958CE380936B028DB79EB706968DBF86
:104C20008091A3089091A4089F938F9380E297E0CE
:104C30002EC110926B0282E397E09F938F93FF92B5
:104C4000EF92FE01099584E180936B020F900F9023
:104C50000F900F9080914A0790914B079F938F93ED
:104C60008BE397E09F938F93FF92EF92E0912F0455
:104C7000F0913004099588E280936B028DB79EB75E
:104C800006968DBF8091210399279F938F938BE484
:104C900097E09F938F93FF92EF92E0912F04F09112
:104CA000300409958CE380936B022DB73EB72A5FE1
:104CB0003F4F2DBF80914907992701979F938F936D
:104CC0008BE597E002CB10926B028BE697E09F9307
:104CD0008F93FF92EF92FE01099584E180936B021E
:104CE0000F900F900F900F9080912F0390913003B1
:104CF0009F938F9383E797E09F938F93FF92EF9219
:104D0000E0912F04F0913004099588E280936B02C2
:104D10002DB73EB72A5F3F4F2DBF8091330390914F
:104D200034039F938F9381E897E09F938F93FF9233
:104D3000EF92E0912F04F091300409958CE3809379
:104D40006B028DB79EB706968DBF8091310390910F
:104D500032039F938F938FE897E099C010926B0274
:104D60008091220399279F938F938DE997E09F93DA
:104D70008F93FF92EF92FE01099584E180936B027D
:104D80008DB79EB706968DBF8091230399279F9379
:104D90008F9389EA97E09F938F93FF92EF92E09130
:104DA0002F04F0913004099588E280936B022DB7AF
:104DB0003EB72A5F3F4F2DBF8091240399279F93D1
:104DC0008F9385EB97E09F938F93FF92EF92E09103
:104DD0002F04F091300409958CE380936B028DB71A
:104DE0009EB706968DBF8091250399279F938F9339
:104DF00081EC97E04CC010926B02809126039927BA
:104E00009F938F938DEC97E09F938F93FF92EF92F8
:104E1000FE01099584E180936B028DB79EB70696DB
:104E20008DBF8091270399279F938F9389ED97E0FA
:104E30009F938F93FF92EF92E0912F04F0913004B3
:104E4000099588E280936B022DB73EB72A5F3F4FEA
:104E50002DBF8091280399279F938F9385EE97E02C
:104E60009F938F93FF92EF92E0912F04F091300483
:104E700009958CE380936B028DB79EB706968DBF24
:104E80008091290399279F938F9381EF97E09F93B8
:104E90008F93FF92EF92D9CA10926B028DEF97E039
:104EA0009F938F9300EE1FE1FF92EF92FE01099511
:104EB00084E180936B020F900F900F900F90809180
:104EC000C10199279F938F9385E098E09F938F93DB
:104ED000FF92EF92E0912F04F0913004099588E25F
:104EE00080936B028DB79EB706968DBF809122028C
:104EF0009091230297FD03969595879595958795B3
:104F00009F938F9383E198E09F938F931F930F93C9
:104F1000E0912F04F091300409958CE380936B02AB
:104F20002DB73EB72A5F3F4F2DBF80914F0699277F
:104F30009F938F9380914E0699279F938F9381E241
:104F400098E09F938F931F930F93E0912F04F0911C
:104F5000300409958DB79EB70896F7C010926B0282
:104F60008FE298E09F938F93FF92EF92FE01099555
:104F700084E180936B020F900F900F900F908091BF
:104F80006904992787FD90959F938F93809168047A
:104F9000992787FD90959F938F938FE398E09F9338
:104FA0008F93FF92EF92E0912F04F09130040995D6
:104FB00088E280936B022DB73EB7285F3F4F2DBF2D
:104FC00080916A04992787FD90959F938F93809194
:104FD0006B0499279F938F938FE498E09F938F930F
:104FE000FF92EF92E0912F04F091300409958CE349
:104FF00080936B028DB79EB708968DBF80916F042A
:1050000099279F938F9380916C04992787FD9095A2
:105010009F938F938FE598E02DCB10926B028FE6D4
:1050200098E09F938F93FF92EF92FE01099584E1A0
:1050300080936B020F900F900F900F908091040758
:1050400099278F7790709F938F938091FC06992773
:105050008F7790709F938F938091F40699278F7725
:1050600090709F938F938091EC0699278F77907023
:105070009F938F938FE798E09F938F93FF92EF9288
:10508000E0912F04F0913004099588E280936B023F
:105090008DB79EB70C968DBF8091240799278F7787
:1050A00090709F938F9380911C0799278F779070B2
:1050B0009F938F938091140799278F7790709F9378
:1050C0008F9380910C0799278F7790709F938F9380
:1050D00080E998E09F938F93FF92EF92E0912F04E5
:1050E000F091300409958CE380936B022DB73EB7A5
:1050F000245F3F4F2DBF8091440799278F77907091
:105100009F938F9380913C0799278F7790709F93FF
:105110008F938091340799278F7790709F938F9307
:1051200080912C0799278F7790709F938F9381EAB6
:1051300098E09F938F93FF92EF92E0912F04F0916C
:10514000300409958DB79EB70C968DBFFEC11092A5
:105150006B0282EB98E09F938F93FF92EF92FE0198
:10516000099584E180936B020F900F900F900F9040
:1051700080910807992787FD90959F938F93809141
:105180000007992787FD90959F938F938091F8064C
:10519000992787FD90959F938F938091F00699278B
:1051A00087FD90959F938F9381EC98E09F938F93C9
:1051B000FF92EF92E0912F04F0913004099588E27C
:1051C00080936B022DB73EB7245F3F4F2DBF809178
:1051D0002807992787FD90959F938F9380912007AB
:1051E000992787FD90959F938F9380911807992712
:1051F00087FD90959F938F9380911007992787FD46
:1052000090959F938F9382ED98E09F938F93FF9259
:10521000EF92E0912F04F091300409958CE3809394
:105220006B028DB79EB70C968DBF8091480799276A
:1052300087FD90959F938F9380914007992787FDD5
:1052400090959F938F9380913807992787FD90952C
:105250009F938F9380913007992787FD90959F9317
:105260008F9383EE98E09F938F93FF92EF92E0915C
:105270002F04F091300409952DB73EB7245F3F4FBE
:105280002DBF63C110926B0284EF98E09F938F93C0
:1052900000EE1FE1FF92EF92FE01099584E18093F9
:1052A0006B020F900F900F900F9080910407881F52
:1052B0008827881F97E0899FC00111248D969F93AE
:1052C0008F938091FC06881F8827881F96E0899F0E
:1052D000C00111248D969F938F938091F406881FAF
:1052E0008827881F95E0899FC00111248D969F9380
:1052F0008F938091EC06881F8827881F9927880F35
:10530000991F880F991F8D969F938F9383E099E043
:105310009F938F93FF92EF92E0912F04F0913004CE
:10532000099588E280936B028DB79EB70C968DBF6E
:1053300080912407881F8827881F9BE0899FC001D0
:1053400011248D969F938F9380911C07881F882727
:10535000881F9AE0899FC00111248D969F938F9397
:1053600080911407881F8827881F99E0899FC001B2
:1053700011248D969F938F9380910C07881F882707
:10538000881F992723E0880F991F2A95E1F78D96AA
:105390009F938F9387E199E09F938F93FF92EF9272
:1053A000E0912F04F091300409958CE380936B0217
:1053B0002DB73EB7245F3F4F2DBF80912C07881F2C
:1053C0008827881F9CE0899FC00111248D969F9398
:1053D0008F938BE299E09F938F93FF92EF92E091EE
:1053E0002F04F09130040995809134072DB73EB712
:1053F0002A5F3F4F2DBF87FF12C080E480936B026E
:105400008CE399E09F938F93FF92EF92E0912F04AA
:10541000F091300409950F900F900F900F908091AC
:105420003C0787FF12C084E480936B028FE399E00E
:105430009F938F931F930F93E0912F04F09130046B
:1054400009950F900F900F900F908091440787FF60
:105450007CC088E480936B0282E499E09F938F93F1
:105460001F930F93E0912F04F091300409950F9052
:105470000F900F900F9069C010926B0285E499E035
:105480009F938F93FF92EF92FE01099584E18093A1
:105490006B020F900F900F900F908091F9019091F7
:1054A000FA019F938F9383E599E09F938F93FF92E7
:1054B000EF92E0912F04F0913004099588E28093F7
:1054C0006B028DB79EB706968DBF8091FB019091C0
:1054D000FC019F938F9380E699E09F938F93FF92B7
:1054E000EF92E0912F04F0913004099589E48093C4
:1054F0006B022DB73EB72A5F3F4F2DBF8DE699E077
:105500009F938F93FF92EF92E0912F04F0913004DC
:105510000995809169020F900F900F900F9083FF73
:1055200014C01092FC011092FB0160E070E08EE06C
:1055300090E00E94902C09C080912001281719F456
:1055400021502093200110926A0210926902E6E035
:10555000CDB7DEB70C9407784AEA20E030E0261792
:10556000370740F4FC018191480F2F5F3F4F26170A
:105570003707C8F3842F99270895AC019AEA20E0F1
:1055800030E02617370750F4DA01A20FB31F0E944C
:105590001C78802D980F2F5F3F4FF3CF892F9927CD
:1055A000089581E08093220682E08093210683E0C3
:1055B0008093200684E08093230685E08093240670
:1055C00086E08093250687E08093260688E0809316
:1055D000270689E0809328068AE0809329068BE0DD
:1055E00080932A068CE080932B06089595E590938E
:1055F0001F0680910201843170F08AE080933F069B
:10560000109263068BE180933B068EE480936006E4
:10561000809361060DC083E080933F0680E2809313
:1056200063068EE180933B0690936006909361063B
:105630008AE680932C0683E08093850681E0809340
:1056400046061092820610927F0668E06093390643
:1056500086EE80933A0680E880933C065EE15093A4
:105660002D068FEF80932F069FE090933006509386
:105670002E06109232066093330680E4809334063F
:105680001092350690933106109248061092490602
:1056900010924A0610924B0610926506109266060A
:1056A000109267061092680638E730934C0648E27D
:1056B00040934D0672E07093840690934E0627EF58
:1056C00020934F0685E0809354068DE7809357061C
:1056D0008093580680935906309350069AE590932C
:1056E000510610925206209353064093550610928D
:1056F00056068FE58093690683EF80936B068AEAEE
:1057000080936D0680936E0684E180936A06809391
:105710006C0682E380935A0690935B0680935C0646
:10572000109283068EEF80936F0624E62093700616
:105730009093710690937206909373068BE4809316
:10574000740680937506809376061092770686E03D
:10575000809378066093790690937A0650937B063F
:1057600020937C0620937D0670937E06109280061F
:105770001092810681E2809343068DE28093440675
:10578000909345060895CF93DF930E94F62A8EE00A
:105790008093360620E1209337063CE030933806AC
:1057A00090E590933D0686E980933E0690934006EF
:1057B0008093410686E08093420680E2809347060C
:1057C0008AE580935D0690935E0681E080935F0694
:1057D0002093620684E680936406A6E8B6E0E1E7DB
:1057E000F1E0ED01019009923A95E1F763E770E08D
:1057F000CD01875690400E94AC2A80939206DF919B
:10580000CF910895CF93DF930E94F62A8AE0809388
:10581000360680E18093370626E0209338069AE525
:1058200090933D0688E780933E06909340068093D0
:1058300041062093420620E22093470690935D069E
:1058400080E580935E068CE380935F06209362067A
:105850008BE480936406A6E8B6E08CE0E8E7F1E02C
:10586000ED01019009928A95E1F763E770E0CD01BF
:10587000875690400E94AC2A80939206DF91CF9188
:105880000895CF93DF930E94F62A88E0809336062E
:1058900030E13093370626E02093380694E6909363
:1058A0003D0688E780933E0690934006809341062C
:1058B00020934206309347068AE580935D0680E593
:1058C00080935E0696E490935F0680E28093620682
:1058D00090936406A6E8B6E08CE0E0E8F1E0ED0124
:1058E000019009928A95E1F763E770E0CD01875650
:1058F00090400E94AC2A80939206DF91CF91089548
:10590000DC010E941C78802D99270895DC01062E69
:105910000E942E780895DC010E942978CF01089515
:10592000DC010B010E943A780895FF920F931F93B8
:10593000CF93DF93982F8150853008F093E084E770
:10594000F82E9F9D80011124E801609763E770E0C5
:10595000CE010E94BD2A982FD801AD59BF4F0E9499
:105960001C78802D891731F4DE010E941C78802D6F
:10597000853519F080E090E00AC0EFE1F6E0DE0145
:105980001F2C0E9424780E94176781E090E0E5E0D8
:10599000CDB7DEB70C940878863010F085E003C0F0
:1059A000882309F481E0A2E0B0E0082E0E942E785E
:1059B00008951F93CF93DF93182FCFE1D6E0809106
:1059C0001F06853591F5163010F015E002C0112341
:1059D00061F163E770E08FE196E00E94AC2A80936A
:1059E000920684E7189FD00111245097FE01182ECB
:1059F0000E943F78E0E2F6E0A0E5B0E02CE030E085
:105A0000122E0E943F78B90180E296E00E94AC2AF3
:105A1000ACE5B0E0082E0E942E78812F0E94CC2C9D
:105A20000E94176781E090E002C080E090E0DF9183
:105A3000CF911F9108956DE470E088EE93E00E948D
:105A4000BD2AA5E3B4E00E941C78902D981739F484
:105A5000A8EEB3E00E941C78802D813019F080E020
:105A600090E00895E3E9F6E0A8EEB3E08EE4182EA6
:105A70000E94247881E090E00895CF93DF93C3E9FA
:105A8000D6E080919306813089F46DE470E0CE0118
:105A90000E94AC2A8093E006A8EEB3E08EE4FE01FB
:105AA000182E0E943F7881E090E002C080E090E0F4
:105AB000DF91CF910895CF93DF9381E08093930698
:105AC000E3E9F6E08FE0158616861786108A815086
:105AD000349687FFF8CF80E48093A0068093A106D8
:105AE0001092A2068093A3068093A40690EC909354
:105AF000A5061092A6068093A7068093A80610928A
:105B0000A9069093AA069093AB068093AC061092D8
:105B1000AD068093AE069093AF06A4E9B6E087E0A9
:105B2000EAE8F1E0ED01019009928A95E1F76DE470
:105B300070E0CD0101970E94AC2A8093E006DF91CE
:105B4000CF910895A2E0B0E00E941C78802D8630AD
:105B500030F083E0A2E0B0E0082E0E942E78992772
:105B600008951F93CF93C82F162F863010F0C5E0ED
:105B700003C0882309F4C1E08C2F99278230910556
:105B800041F08330910544F4019731F40E94C32B16
:105B900005C00E94022C02C00E94412C1123B1F0CA
:105BA0006CE070E080E590E00E94BD2AACE5B0E0DA
:105BB0000E941C78902D981749F4E0E2F6E0A0E5E9
:105BC000B0E08CE0182E0E94247802C00E94D12AF6
:105BD0008C2F0E94D92CCF911F910895DF92EF92C4
:105BE000FF920F931F93CF93FF24DF2CEF2C81E0C4
:105BF00090E00E94802C853539F031E0E32E65E598
:105C000081E090E00E94862C6CE070E080E590E0FE
:105C10000E94BD2AC82FACE5B0E00E941C78802D00
:105C20008C1711F421E0D22EC1E001E010E0EE204B
:105C300029F48C2F0E94952C8823B1F591E0F92E40
:105C40001F930F9385E799E09F938F9384EF92E1E1
:105C50009F938F93E0912F04F091300409958DB7B5
:105C60009EB706968DBF0230110549F0033011052D
:105C70004CF40130110531F40E94C32B05C00E9481
:105C8000022C02C00E94412CDD2049F0E0E2F6E047
:105C9000A0E5B0E08CE0182E0E94247802C00E949B
:105CA000D12A8C2F0E94D92CCF5F0F5F1F4FC63097
:105CB00008F4BDCFFF2019F083E00E94CC2C0E9495
:105CC000A22DC82F0E94952C8C2F99279F938F93DC
:105CD0008BE999E09F938F9304EF12E11F930F9349
:105CE000E0912F04F091300409958DB79EB7069688
:105CF0008DBFEE2021F40E941B2D882399F484EBA4
:105D000099E09F938F931F930F93E0912F04F0914D
:105D1000300409950E945B2D0E943D2D0F900F903D
:105D20000F900F9010921E0690E0E0EAF6E0CFE0B0
:105D30008081349618160CF49F5FC150C7FFF8CFCE
:105D400090931E06892F99279F938F9384E996E05D
:105D50009F938F9385ED99E09F938F931F930F935C
:105D6000E0912F04F091300409958DB79EB7089605
:105D70008DBF86EF99E09F938F931F930F93E091D0
:105D80002F04F091300409950F900F900F900F9011
:105D9000CF911F910F91FF90EF90DF900895982F72
:105DA0002FB7F8943998389A88B1836088B9809170
:105DB000B9008C7F8093B9008AE28093B80010927A
:105DC00076021092740210927302992379F0E9EE30
:105DD000F6E08BE010821182128213821482158207
:105DE000168217828150389687FFF4CF78942FBFA0
:105DF00008951092760284E98093BC0080E8809335
:105E0000BC001092BD001092BA001092BB0010921C
:105E1000B9001092B8001092720280E00E94CF2E5A
:105E20001092BB0085E88093BC0080917002826074
:105E30008093700208951F920F920FB60F92112453
:105E40002F933F934F935F938F939F93EF93FF9382
:105E500080917602282F3327442755278F5F809320
:105E60007602F9012731310508F0C2C2EE59FF4F21
:105E70000C94167881E08093720209C080917402BC
:105E80008C3090F4809174028F5F809374028091C3
:105E90007402E82FFF27EE0FFF1FEE0FFF1FED56D6
:105EA000F94F8585181654F7809174028C3070F084
:105EB00010926F0210926E021092740285E080932D
:105EC000760280917302880F8D5A04C0809174020B
:105ED000880F8E5A8093BB0085E87FC28091740240
:105EE000E82FFF2783E0EE0FFF1F8A95E1F7E751C8
:105EF000F94F81818093BB0085E88093BC0080913D
:105F00007402E82FFF27EE0FFF1FEE0FFF1FEE0FAB
:105F1000FF1FE751F94F808180FF91C0809174028B
:105F2000E82FFF27EE0FFF1FEE0FFF1FEE0FFF1FE3
:105F3000E751F94F8281882329F080911E0687302E
:105F400008F46CC280916E0290916F02892B09F067
:105F500065C280916C0290916D02892B09F05EC23E
:105F60006EC08091740221E030E002C0220F331F26
:105F70008A95E2F780916C0290916D022823392373
:105F8000232B79F080917402E82FFF27EE0FFF1F7B
:105F9000EE0FFF1FEE0FFF1FE751F94F80E18483E3
:105FA0000DC080917402E82FFF27EE0FFF1FEE0F48
:105FB000FF1FEE0FFF1FE751F94F1482809174020B
:105FC000E82FFF2753E0EE0FFF1F5A95E1F7E75147
:105FD000F94F8481282F332743E0220F331F4A953E
:105FE000E1F780917402E82FFF2793E0EE0FFF1F87
:105FF0009A95E1F7E751F94F82818770822B809360
:10600000BB0085E88093BC002091740281E090E0A1
:1060100002C0880F991F2A95E2F720916E023091F5
:106020006F0282239323892B51F081EE96E09093A7
:106030007A028093790288E080937B02EFC184E04A
:1060400089C1E0917902F0917A0281918093BB003D
:1060500085E88093BC00F0937A02E0937902809106
:106060007B02815080937B02882309F4D7C183E0AF
:1060700071C18091B900803351F5809177028823F6
:1060800029F4809174028F5F80937702809174026B
:10609000E82FFF2783E0EE0FFF1F8A95E1F7E75116
:1060A000F94F838199278F7790708F3791057CF412
:1060B00080917402E82FFF27EE0FFF1FEE0FFF1FE6
:1060C000EE0FFF1FE751F94F83818F5F838310929B
:1060D000760284E98093BC008AE090E0909393017B
:1060E00080939201809174028F5F8093740210926A
:1060F00076026DC18091B9008034C9F1809173023C
:10610000E82FFF27EE0FFF1FEE0FFF1FEE0FFF1F01
:10611000E751F94F83818F778383809173028F5F7B
:1061200080937302809173028C30A0F010927302FE
:1061300010926D0210926C02809178028F5F8093B2
:1061400078028C3038F010927802809170028D7F46
:10615000809370028091700281608093700210922F
:10616000760284E98093BC001092720273C0809121
:106170007302E82FFF27EE0FFF1FEE0FFF1FEE0F3A
:10618000FF1FE751F94F83818068838380917302F9
:10619000E82FFF27EE0FFF1FEE0FFF1FEE0FFF1F71
:1061A000E751F94F808180FF2FC080917302E82F63
:1061B000FF2753E0EE0FFF1F5A95E1F7E751F94F24
:1061C00084819927009751F04097D9F581EE96E0A8
:1061D00090937A028093790288E031C080917302B3
:1061E000992743E0880F991F4A95E1F78251994F0B
:1061F00090937A0280937902909173028091780251
:106200009817E1F483E01BC080917302992733E073
:10621000880F991F3A95E1F78251994F90937A022E
:10622000809379028091700281FD06C09091730283
:1062300080917802981711F482E001C081E0809388
:106240007B0280917B02813011F485E801C085ECEE
:106250008093BC0080917702809371021092770244
:10626000DDC0E0917902F0917A028091BB008083D9
:106270008091790290917A02019690937A028093AC
:10628000790280917B02815080937B02823010F0F2
:1062900085EC5DC0813011F485E859C080917002B1
:1062A00081FF2DC08091ED0280FD1DC080917302A1
:1062B000E82FFF2723E0EE0FFF1F2A95E1F7E751B4
:1062C000F94F86818A3F79F480917302E82FFF2786
:1062D00093E0EE0FFF1F9A95E1F7E751F94F8081A8
:1062E000816080830CC080917302E82FFF2783E0D8
:1062F000EE0FFF1F8A95E1F7E751F94F1082809169
:1063000073028F5F80937302809173028C30A0F0D0
:106310001092730210926D0210926C0280917802BA
:106320008F5F809378028C3038F0109278028091E1
:1063300070028D7F809370021092760284E98093C0
:10634000BC008091700281608093700265C0809370
:10635000BC0086E08093760261C088E9BBCD809165
:106360007502880F805FB6CD8091750299278130C4
:10637000910561F0823091051CF4892B21F04EC00B
:10638000029739F04BC080911301A4CD8091120186
:10639000A1CD809111019ECD80E89CCD1092760216
:1063A00084E98093BC00109272028AE090E090939E
:1063B00093018093920180917502823088F48091DC
:1063C00075028F5F8093750282E1809376028091DF
:1063D00070028E7F8093700285EA8093BC001EC09D
:1063E000109275028091700281608093700216C0D5
:1063F0001092760284E98093BC00809170028160E3
:10640000809370028AE090E09093930180939201D0
:10641000109274021092730210927202FF91EF9127
:106420009F918F915F914F913F912F910F900FBE50
:106430000F901F9018951F93CF93DF93182F809183
:106440001803882321F480910702882319F081E042
:1064500090E097C01D3008F092C01123B1F0E12FF9
:10646000FF2723E0EE0FFF1F2A95E1F7E751F94FD1
:1064700035978081359688230CF081C038978081CC
:1064800080FD03C083E090E07CC08091E106823013
:1064900019F084E090E075C067E070E081EE96E06E
:1064A0000E94AC2A9091E806891719F085E090E0E7
:1064B00068C080ED97E00E941A17EC01809170028D
:1064C00080FD05C0CE010E9423178823B9F3112354
:1064D00019F48FEF90E00BC0212F3327215030406B
:1064E00081E090E002C0880F991F2A95E2F790930F
:1064F0006F0280936E02A1E0B0E0E9EEF6E040E0CA
:1065000050E06BE0CD01042E02C0880F991F0A9461
:10651000E2F720916E0230916F0282239323892B40
:1065200011F01182128261504F5F5F4F389667FF02
:10653000E9CF1092740210927602809170028E7FE1
:106540008093700285EA8093BC008091700280FD88
:1065500005C0CE010E9423178823B9F380916E02F3
:1065600090916F02892B29F0CE010E942317882376
:1065700011F380916E0290916F02009711F082E00A
:1065800090E0DF91CF911F9108950F931F93CF93C8
:10659000DF93982F80911803882321F480910702BC
:1065A000882319F081E090E092C09D30A0F49923F7
:1065B00019F486E090E08BC0C92FDD27FE0133E09F
:1065C000EE0FFF1F3A95E1F7E751F94F35978081BC
:1065D000359687FD03C082E090E079C038978081CE
:1065E00080FD03C083E090E072C080ED97E00E94E0
:1065F0001A178C018091700280FD05C0C8010E94AD
:1066000023178823B9F3219721E030E0C90102C0A4
:10661000880F991FCA95E2F790936D0280936C02E0
:10662000D901E9EEF6E040E050E06BE0CD01042E48
:1066300002C0880F991F0A94E2F720916C023091F2
:106640006D0282239323892B11F0118212826150F3
:106650004F5F5F4F389667FFE9CF10927302109239
:10666000E1061092E80610927602809170028E7F09
:106670008093700285EA8093BC008091700280FD57
:1066800005C0C8010E9423178823B9F380916C02CA
:1066900090916D02892B29F0C8010E94231788234D
:1066A00011F38091E106823019F084E090E00FC090
:1066B00067E070E081EE96E00E94AC2A9091E806D7
:1066C000891719F085E090E002C080E090E0DF914A
:1066D000CF911F910F91089589E1AEE7B7E0EAE409
:1066E000F7E011821082329611961C921E92129639
:1066F000815087FFF6CF1092870310928603109285
:1067000089031092880310928B0310928A030895D4
:106710001F920F920FB60F9211240F931F932F9376
:106720003F934F935F936F937F938F939F93AF9319
:10673000BF93CF93DF93EF93FF938091850682FD04
:10674000CFC0409186005091870080917D0290914A
:106750007E02481B590B8091860090918700909390
:106760007E0280937D02CA018D549440A0917F02E5
:10677000B0918002835F9A4178F480917F02809388
:106780004907149714F01092940181E090E09093DF
:10679000800280937F0207C2AD30B1050CF003C2C6
:1067A000CA018B5F9040845B914008F074C0425DE9
:1067B0005140FD01EA0FFB1FE65BF84F808191819C
:1067C000FA01E81BF90BCF01F7FF03C09095819503
:1067D0009F4F06975CF480912103883C20F48091C0
:1067E0002103865F01C088EC80932103FD01EA0F3D
:1067F000FB1FE65BF84F808191819C01220F331FC4
:10680000280F391F240F351F37FF02C02D5F3F4F60
:10681000E901D595C795D595C795CA0101968C17FD
:106820009D0714F4219706C041505040C417D50766
:106830000CF4219680912103833CE0F08D010A0F36
:106840001B1FF801E65BF84F808191819E01281B98
:10685000390BC90163E070E00E948F77CB01880F8C
:10686000991F860F971F0258184FD80111969C93B5
:106870008E9307C0AA0FBB1FA258B84F11961C9247
:106880001E92E0917F02F0918002EE0FFF1FE65B07
:10689000F84FD183C08320917F02309180022F5F17
:1068A0003F4F3093800220937F0280910201843118
:1068B00008F079C12530310511F45D9A01C05D9869
:1068C00080917F02909180028630910511F45C9A4C
:1068D00001C05C98079711F45B9A65C15B9863C12E
:1068E00040918600509187008091810290918202B0
:1068F000481B590B809186009091870090938202EB
:1069000080938102CA018D5494406091EB02835FB1
:106910009A4108F07AC060937C0280917C028430B6
:1069200008F453C09091490780917C02981709F0B0
:106930004CC05091EC025B3008F43FC010929401BF
:106940001092EB0240E05F31C0F0E42FFF27EE0F22
:10695000FF1F9F0129543D4FDF01A65BB84F8D916A
:106960009C91D9018D939C93DF01A258B84F8D91D2
:106970009C91EF52FD4F91838083E42FFF27EE0F10
:10698000FF1F9F01265B384FDF01AD57BD4F8D9133
:106990009C91D90111969C938E93DF01A356BD4F14
:1069A0008D919C91E258F84F91838083842F8F5F63
:1069B000482F8D3040F28093EB028091EC028F3FA4
:1069C000B9F08F5F8093EC0213C08091EC028536A2
:1069D00020F08AE08093EC0202C01092EC028091D9
:1069E00002018A3011F0843110F0289A01C02898F1
:1069F00081E08093EB0280911803882309F0D3C0D3
:106A000080917C0280934907CEC06D3008F0A3C00E
:106A1000CA018B5F9040845B914008F07EC0425D6C
:106A20005140E62FFF27EE0FFF1FED57FD4F8081EE
:106A30009181FA01E81BF90BCF0105960B97B0F491
:106A40008091EC028A3120F080912103865F05C09D
:106A50008B3028F0809121038E5F809321038091F9
:106A60002103893C18F088EC80932103E62FFF274F
:106A7000EE0FFF1FED57FD4F808191819C01220F8A
:106A8000331F280F391F240F351F37FF02C02D5F1A
:106A90003F4FE901D595C795D595C795CA01019690
:106AA0008C179D0714F4219706C041505040C4171D
:106AB000D5070CF42196809121038E3BD8F0E62F68
:106AC000FF27EE0FFF1FDF01AD57BD4F8D919C914A
:106AD0009E01281B390BC90163E070E00E948F778B
:106AE000CB01880F991F860F971FE356FD4F9183A7
:106AF000808308C0E62FFF27EE0FFF1FE356FD4FF0
:106B0000118210828091EB02E82FFF27EE0FFF1F0A
:106B1000ED57FD4FD183C08309C0809102018A30B7
:106B200011F0843110F0289A01C028988091020158
:106B3000843188F48091EB02853011F45D9A05C0B0
:106B40005D98863011F45C9A05C05C98873011F42A
:106B50005B9A01C05B988091EB02843120F48F5FD7
:106B60008093EB0220C08431F1F4809102018A30DD
:106B700011F0843110F0289A01C028988EE180939A
:106B8000EB022CE0CEE7D7E0A7EBB2E0EAE4F7E0D7
:106B90008D919D91918380833296198218822296DD
:106BA000215027FFF5CFFF91EF91DF91CF91BF915A
:106BB000AF919F918F917F916F915F914F913F9195
:106BC0002F911F910F910F900FBE0F901F9018954E
:106BD000EF92FF920F931F9380913B069927880FA6
:106BE000991F880F991F7C010027F7FC0095102F33
:106BF0008091750390917603A0917703B09178030B
:106C0000BC01CD01A80197010E94C4773093CB0548
:106C10002093CA0580916D0390916E03A0916F033C
:106C2000B0917003BC01CD01A80197010E94C47707
:106C30003093CD052093CC058091170890911808CA
:106C400097FD039695958795959587959093CF0594
:106C50008093CE0580912A0890912B0897FD03968A
:106C600095958795959587959093D1058093D005B7
:106C700080918603909187032091470230914802CA
:106C8000821B930B9093D3058093D20580911303BD
:106C900090911403A0911503B0911603BC01CD018E
:106CA00025E030E040E050E00E94C4773093D50505
:106CB0002093D40580914102909142029093D70590
:106CC0008093D60580913303909134039093DB0534
:106CD0008093DA0580911E0190911F019093DD054C
:106CE0008093DC058091210399279093DF058093A1
:106CF000DE058091260890912708A0912808B09180
:106D00002908209196013091970140919801509166
:106D10009901BC01CD010E94C4773093E105209315
:106D2000E0058091EA0699279093E3058093E205B8
:106D30008091F20699279093E5058093E405809170
:106D4000FA0699279093E7058093E605809102075C
:106D500099279093E9058093E8058091220290910C
:106D600023029093F3058093F20580919F08909100
:106D7000A0089093F7058093F6058091A308909161
:106D8000A4089093F9058093F8058091A508909147
:106D9000A6089093FB058093FA058091A708992790
:106DA000909305068093040680910004909101045D
:106DB00090930706809306068091FE039091FF034F
:106DC000909309068093080680914804882321F453
:106DD00080914904882321F08091C905816003C016
:106DE0008091C9058E7F8093C9051F910F91FF90F7
:106DF000EF9008951F93CF93DF93182FEB018091AD
:106E000018038823A1F411501F3F89F0D093290261
:106E1000C09328028091280290912902892BD1F7F2
:106E2000CE018C0F9D1F0E942F17115078F7DF9114
:106E3000CF911F910895CF93DF93809102018D3000
:106E400011F40E94141B10927A0080914B029091D1
:106E50004C029093D1078093D00780914902909182
:106E60004A029093BF078093BE078091470290919A
:106E700048029093200880931F082091430230918C
:106E80004402C901880F991F880F991F820F931F11
:106E9000820F931F90931808809317082091450242
:106EA00030914602C901880F991F880F991F820FE0
:106EB000931F820F931F90932B0880932A088FECC7
:106EC00080937A00A2E2B3E0C4E2D6E097E0899131
:106ED000E82FFF27EE0FFF1FE65BF84F0190F081D0
:106EE000E02DE259FF4F1E161F061CF0E0E0F0E017
:106EF00005C0EF3FF10514F0EFEFF0E08C91282F83
:106F00003327E217F30714F4815004C02E173F070C
:106F100014F48F5F8C939150119697FFD8CF809186
:106F200060069927AA27BB27BC01CD0124EC39E0D4
:106F300040E050E00E945077DC01CB018093D50106
:106F40009093D601A093D701B093D80180916106A8
:106F50009927AA27BB27BC01CD010E945077DC01ED
:106F6000CB018093D1019093D201A093D301B09330
:106F7000D401DF91CF910895A0E0B0E0E2ECF7E317
:106F80000C94E577882EC0E0D0E07E016E0110926F
:106F90004804469AD0938103C0938003D0937F0323
:106FA000C0937E03D0937B03C0937A03D0938B036B
:106FB000C0938A03D0938903C0938803D093870337
:106FC000C09386031092BE011092BD0110923B0245
:106FD0000E941B3784E690E00E943C170E941B37FA
:106FE00080912C0680FF10C08091140190911501B2
:106FF000875B934038F480911401909115018E5E67
:10700000924010F40E94B91A0FE18AE090E00E94C9
:107010003C178091470290914802C80FD91F809178
:107020004B0290914C02E80EF91E8091490290911A
:107030004A02C80ED91E015007FFE7CF9701205F13
:107040003F4F369527953695279530938B032093A0
:107050008A03C60140969695879596958795909355
:107060008903809388036096F5E0D695C795FA95D5
:10707000E1F7D0938703C0938603909385038093B1
:1070800084033093830320938203882009F441C052
:10709000809117089091180897FF03C090958195EB
:1070A0009F4F6CE070E00E948F779B01709381038B
:1070B0006093800380912A0890912B0897FF03C06A
:1070C000909581959F4F6CE070E00E948F77709350
:1070D0007F0360937E038091110690911206909336
:1070E0007B0380937A03B90184E090E00E94902CA6
:1070F00060917E0370917F0386E090E00E94902C67
:1071000060917A0370917B0388E090E00E94902C5C
:1071100065C084E090E00E948B2C90938103809363
:10712000800386E090E00E948B2C90937F038093F5
:107130007E0388E090E00E948B2C9C0190937B035F
:1071400080937A03809180039091810381509840CD
:1071500050F480917E0390917F038150984018F401
:1071600021503440D8F187E19AE09F938F9384EFC8
:1071700092E19F938F93E0912F04F0913004099551
:10718000809117089091180897FF03C090958195FA
:107190009F4F6CE070E00E948F7770938103609343
:1071A000800380912A0890912B0897FF03C0909547
:1071B00081959F4F6CE070E00E948F7770937F0302
:1071C00060937E03809111069091120690937B0349
:1071D00080937A030F900F900F900F901092D10729
:1071E0001092D0071092BF071092BE07109220088D
:1071F00010921F0884E690E00E943C1780914302A1
:10720000909144029C01220F331F220F331F280F3D
:10721000391F280F391F30931808209317088091C1
:107220004502909146028C01000F111F000F111FA3
:10723000080F191F080F191F10932B0800932A0815
:1072400080913B06C82EDD24EE24FF24442737FD21
:107250004095542FC701B6010E9450774B015C0145
:10726000609375037093760380937703909378030C
:107270009801442737FD4095542FC701B6010E945D
:107280005077DC01CB0180936D0390936E03A09344
:107290006F03B09370038092510390925203A092B7
:1072A0005303B09254038093490390934A03A093ED
:1072B0004B03B0934C031092450310924603109277
:1072C0004703109248038091160190911701A091F5
:1072D0001801B0911901909314068093130610922F
:1072E0003A0210923902109235031092360310922E
:1072F00037031092380380913303909134039093B5
:107300003203809331030E94A06282E390E0909365
:10731000290280932802809160069927AA27BB271B
:10732000BC01CD0124EC39E040E050E00E945077F0
:10733000DC01CB018856954CAF4FBF4F8093D501F0
:107340009093D601A093D701B093D80180916106A4
:107350009927AA27BB27BC01CD010E945077DC01E9
:10736000CB018856954CAF4FBF4F8093D10190937E
:10737000D201A093D301B093D40110929B0110923B
:107380009A018091330390913403AA2797FDA09529
:10739000BA2F209196013091970140919801509118
:1073A0009901BC01CD010E945077DC01CB01809393
:1073B000260890932708A0932808B09329081092D4
:1073C0002C0310922B0381E0809301010E94176728
:1073D0008091ED0284608093ED028FEF80939A0894
:1073E00010929B0880E280939C08C2E2D3E0A4E262
:1073F000B6E007E08D91E82FFF27EE0FFF1FE65B59
:10740000F84F8081918182598993015007FFF2CF13
:1074100084E68093210380912602882311F0469A06
:10742000579A80918A0390918B0380569940815C92
:107430009B4228F0809148048160809348048091A9
:1074400088039091890380569940815C9B4228F083
:1074500080914804826080934804809186039091D3
:1074600087038C5291408957954028F080914804B9
:1074700084608093480480918003909181038C52B2
:107480009140835C914028F080914804886080930B
:10749000480480917E0390917F038C529140835CDD
:1074A000914028F080914804806180934804809145
:1074B0007A0390917B03805092408355914028F04D
:1074C00080914804806280934804ECE0CDB7DEB739
:1074D0000C940178A3E1B0E0E0E7FAE30C94DF77E5
:1074E0008091860390918703209147023091480252
:1074F000821B930B9093200880931F088091510268
:107500009091520297FD07969C0113E035952795BF
:107510001A95E1F73093D1072093D00780914F025D
:107520009091500297FD0796B3E095958795BA958F
:10753000E1F79093BF078093BE073093DD07209358
:10754000DC079093D5078093D4078091170890911A
:107550001808AC01440F551F480F591F20914302D2
:1075600030914402C901880F991F880F991F820F1B
:10757000931F820F931F480F591F57FF02C04D5F83
:107580005F4F5595479555954795509318084093EB
:10759000170880912A0890912B08AC01440F551FC1
:1075A000480F591F2091450230914602C901880FAA
:1075B000991F880F991F820F931F820F931F480FE7
:1075C000591F57FF02C04D5F5F4F55954795559521
:1075D000479550932B0840932A08209143023091FD
:1075E0004402C901880F991F880F991F820F931FAA
:1075F000820F931F9C01442737FD4095542F8091A3
:10760000650390916603A0916703B0916803820FB0
:10761000931FA41FB51F8093650390936603A093E7
:107620006703B09368032091450230914602C90177
:10763000880F991F880F991F820F931F820F931F26
:107640009C01442737FD4095542F80916103909110
:107650006203A0916303B0916403820F931FA41F80
:10766000B51F8093610390936203A0936303B0936B
:1076700064038091E8079091E907209143023091DB
:107680004402820F931F9093E9078093E80780914B
:107690002208909123082091450230914602820FE2
:1076A000931F909323088093220880917C039091EC
:1076B0007D03019690937D0380937C038091110656
:1076C0009091120620917A0330917B03821B930BD9
:1076D0009C01442737FD4095542F80915D03909184
:1076E0005E03A0915F03B0916003820F931FA41FFC
:1076F000B51F80935D0390935E03A0935F03B093E7
:1077000060038FEC80937A001092100120914D035A
:1077100030914E0340914F035091500329873A878F
:107720004B875C8729543B46414050402CF028E46D
:107730003BE641E050E00DC089859A85AB85BC856C
:10774000885B9449AE4FBF4F4CF428EB34E94EEFC1
:107750005FEF2D833E834F83588708C089859A85C4
:10776000AB85BC858D839E83AF83B88720915503FD
:107770003091560340915703509158032D873E870F
:107780004F87588B29543B46414050402CF028E409
:107790003BE641E050E00DC08D859E85AF85B88900
:1077A000885B9449AE4FBF4F4CF428EB34E94EEF61
:1077B0005FEF29833A834B835C8308C08D859E8568
:1077C000AF85B88989839A83AB83BC83A0911F0856
:1077D000B0912008BB8BAA8BFD01CF01AA2797FD92
:1077E000A095BA2FA0904503B0904603C0904703E0
:1077F000D0904803A80EB91ECA1EDB1EA0924503F6
:10780000B0924603C0924703D0924803E090260806
:10781000F09027080091280810912908E80EF91E19
:107820000A1F1B1FE0922608F092270800932808E1
:1078300010932908F0910803F98BFF2309F098C1F0
:1078400080910703882309F093C180912C0686FF5D
:107850008FC18091BE079091BF07AA2797FDA09581
:10786000BA2FBC01CD0129813A814B815C810E94F4
:1078700050779B01AC0197FF04C02150384F4F4F08
:107880005F4FBBE05595479537952795BA95D1F74A
:107890008091BD01682E772488249924CA01B901FA
:1078A000A40193010E945077DC01CB0180939903DE
:1078B00090939A03A0939B03B0939C03B7FF04C0DB
:1078C0008150904FAF4FBF4F1C012D01ACE055943C
:1078D000479437942794AA95D1F720929903309230
:1078E0009A0340929B0350929C038091D007909101
:1078F000D107AA2797FDA095BA2FBC01CD012D81F4
:107900003E814F8158850E94507797FF04C0615097
:10791000784F8F4F9F4FFBE09595879577956795AB
:10792000FA95D1F7A40193010E945077DC01CB01B5
:1079300080939D0390939E03A0939F03B093A00315
:10794000B7FF04C08150904FAF4FBF4F9C01AD01B6
:10795000ECE05595479537952795EA95D1F7209313
:107960009D0330939E0340939F035093A003809107
:10797000990390919A039093B4078093B3078091F1
:107980009D0390919E039093B8078093B7072219A7
:1079900033094409550920939D0330939E03409376
:1079A0009F035093A003E20EF31E041F151FE092E5
:1079B0002608F09227080093280810932908809140
:1079C000BC018823B1F457FF04C02F5F3F4F4F4FD6
:1079D0005F4F5595479537952795A21AB30AC40A64
:1079E000D50AA0924503B0924603C0924703D092B5
:1079F00048032A893B8979010027F7FC0095102F5D
:107A000080919D0390919E03A0919F03B091A0034C
:107A1000E80EF91E0A1F1B1FC801B70129813A8110
:107A20004B815C810E9450779B01AC0197FF04C0A1
:107A30002150384F4F4F5F4F6BE055954795379525
:107A400027956A95D1F78091BE01A82EBB24CC243E
:107A5000DD24CA01B901A60195010E945077DC011D
:107A6000CB018093910390939203A0939303B093DF
:107A70009403B7FF04C08150904FAF4FBF4F3C01FC
:107A80004D013CE095948794779467943A95D1F7AB
:107A90006092910370929203809293039092940368
:107AA000C801B7012D813E814F8158850E945077D2
:107AB00097FF04C06150784F8F4F9F4F2BE09595F3
:107AC0008795779567952A95D1F7A60195010E942C
:107AD0005077DC01CB018093950390939603A0939C
:107AE0009703B0939803B7FF04C08150904FAF4FF6
:107AF000BF4FAC01BD018CE07595679557954795D3
:107B00008A95D1F74093950350939603609397031A
:107B1000709398032A893B8937FF03C030952195DC
:107B20003F4F21343105E4F1D401C30197FE07C072
:107B3000B095A095909581959F4FAF4FBF4F8138DD
:107B40009105A105B10584F4DB01CA0177FF07C0E7
:107B5000B095A095909581959F4FAF4FBF4F8138BD
:107B60009105A105B105E4F081E080932D0318C0D3
:107B70001092B8071092B7071092B4071092B3078B
:107B80001092950310929603109297031092980307
:107B90001092910310929203109293031092940307
:107BA0008091950390919603A0919703B0919803CB
:107BB000BC01CD0124E630E040E050E00E94C477F3
:107BC000E0909103F0909203E21AF30AF092CE074C
:107BD000E092CD078091910390919203A09193033D
:107BE000B0919403BC01CD0124E630E040E050E0C8
:107BF0000E94C477DA01C901209195033091960360
:107C00008C01021B130B1093C2070093C1078091D4
:107C1000960190919701A0919801B0919901BC01B2
:107C2000CD0128E631E040E050E00E9450772091FD
:107C300026083091270840912808509129082617D6
:107C400037074807590764F0261B370B480B590BB9
:107C5000209326083093270840932808509329083A
:107C60002091260830912708409128085091290832
:107C700057FF0CC0260F371F481F591F2093260897
:107C80003093270840932808509329086091BE0735
:107C90007091BF076E0D7F1D9B01442737FD4095F6
:107CA000542F8091490390914A03A0914B03B091C6
:107CB0004C03820F931FA41FB51F80934903909319
:107CC0004A03A0934B03B0934C0380910D03909112
:107CD0000E03681B790BCB01AA2797FDA095BA2F3D
:107CE00029853A854B855C85820F931FA41FB51F9C
:107CF00080934D0390934E03A0934F03B093500392
:107D0000C090D101D090D201E090D301F090D40185
:107D1000C816D906EA06FB06C4F488EA91E6A0E094
:107D2000B0E08C199D09AE09BF0980934D03909373
:107D30004E03A0934F03B093500380934903909355
:107D40004A03A0934B03B0934C0322273327A90186
:107D50002C193D094E095F0980914D0390914E0306
:107D6000A0914F03B091500382179307A407B50762
:107D7000B4F4D701C601885A9146A040B040809320
:107D80004D0390934E03A0934F03B0935003809301
:107D9000490390934A03A0934B03B0934C03609123
:107DA000D0077091D107600F711F9B01442737FDE9
:107DB0004095542F8091510390915203A091530309
:107DC000B0915403820F931FA41FB51F80935103DA
:107DD00090935203A0935303B093540380910B03E9
:107DE00090910C03681B790BCB01AA2797FDA095F6
:107DF000BA2F2D853E854F855889820F931FA41F6A
:107E0000B51F8093550390935603A0935703B093E7
:107E10005803E090D501F090D6010091D701109160
:107E2000D801E816F9060A071B07C4F488EA91E6A8
:107E3000A0E0B0E08E199F09A00BB10B8093550311
:107E400090935603A0935703B09358038093510324
:107E500090935203A0935303B093540322273327E4
:107E6000A9012E193F09400B510B809155039091A8
:107E70005603A0915703B091580382179307A407A4
:107E8000B507B4F4D801C701885A9146A040B04064
:107E90008093550390935603A0935703B0935803D0
:107EA0008093510390935203A0935303B0935403D0
:107EB0008091450390914603A0914703B0914803F8
:107EC0008093590390935A03A0935B03B0935C0390
:107ED0008091550390915603A0915703B091580398
:107EE0008093750390937603A0937703B093780300
:107EF00080914D0390914E03A0914F03B091500398
:107F000080936D0390936E03A0936F03B0937003FF
:107F10008091510390915203A0915303B091540367
:107F20008093710390937203A0937303B0937403CF
:107F30008091490390914A03A0914B03B0914C0367
:107F40008093690390936A03A0936B03B0936C03CF
:107F500080911C0190911D0197FD079603E0959576
:107F600087950A95E1F79093D1078093D007809188
:107F70001A0190911B0197FD079613E0959587953F
:107F80001A95E1F79093BF078093BE0780914B024B
:107F900090914C020F9734F488E19CEF9093D107B5
:107FA0008093D00780914B0290914C02079734F454
:107FB00080E398EF9093D1078093D007209102013E
:107FC0002A30A9F480914B0290914C02835F934038
:107FD00034F088EE93E09093D1078093D00780919E
:107FE0004B0290914C028A5F9340DCF014C0809168
:107FF0004B0290914C02815D974034F088EE93E003
:108000009093D1078093D00780914B0290914C02BE
:10801000805E974034F080ED97E09093D107809395
:10802000D0078091490290914A020F9734F488E179
:108030009CEF9093BF078093BE0780914902909177
:108040004A02079734F480E398EF9093BF07809338
:10805000BE072A30A9F48091490290914A02835FB9
:10806000934034F088EE93E09093BF078093BE076F
:108070008091490290914A028A5F9340DCF014C0DB
:108080008091490290914A02815D974034F088EED8
:1080900093E09093BF078093BE078091490290912F
:1080A0004A02805E974034F080ED97E09093BF07DE
:1080B0008093BE076091C801662309F4AFC0409168
:1080C0001C0150911D018091A1039091A203481BB6
:1080D000590B5093A8034093A70320911C013091A2
:1080E0001D01280F391F37FF02C02F5F3F4F359505
:1080F00027953093A2032093A103413851051CF02A
:1081000080E890E005C040585F4F34F480E89FEF6E
:108110009093A8038093A70340911A0150911B01EB
:108120008091A3039091A403481B590B5093A6037D
:108130004093A50320911A0130911B01280F391F8C
:1081400037FF02C02F5F3F4F359527953093A4032B
:108150002093A303413851051CF080E890E005C04E
:1081600040585F4F34F480E89FEF9093A6038093CC
:10817000A503462F55278091A7039091A803849FBC
:10818000B001859F700D949F700D11249B0177FFA6
:1081900002C0215F3F4FF4E035952795FA95E1F74E
:1081A0008091D0079091D107820F931F9093D107B0
:1081B0008093D0078091A5039091A603849FD0015E
:1081C000859FB00D949FB00D1124AD019D01B7FFA7
:1081D00002C0215F3F4FE4E035952795EA95E1F72E
:1081E0008091BE079091BF07820F931F9093BF07A6
:1081F0008093BE0780911C0190911D01860F971FEF
:1082000090931D0180931C0180911A0190911B0194
:10821000840F951F90931B0180931A010091D4073E
:108220001091D5078091B3079091B40710161106ED
:108230005CF59C0197FF04C022273327281B390BCC
:10824000C901AA2797FDA095BA2F2091BC01332719
:1082500044275527BC01CD010E9450779B01AC01FA
:1082600097FF04C0215C3F4F4F4F5F4F76E055951D
:108270004795379527957A95D1F78091CD079091BD
:10828000CE07820F931F27C097FF03C0909581955B
:108290009F4FAA2797FDA095BA2F2091BC013327A5
:1082A00044275527BC01CD010E9450779B01AC01AA
:1082B00097FF04C0215C3F4F4F4F5F4F66E05595DD
:1082C0004795379527956A95D1F78091CD0790917D
:1082D000CE07821B930B9093CE078093CD07E0903F
:1082E000DC07F090DD078091B7079091B8071E1466
:1082F0001F045CF59C0197FF04C022273327281B2D
:10830000390BC901AA2797FDA095BA2F2091BC016E
:10831000332744275527BC01CD010E9450779B018C
:10832000AC0197FF04C0215C3F4F4F4F5F4F96E079
:1083300055954795379527959A95D1F78091C1071F
:108340009091C207820F931F27C097FF03C090959B
:1083500081959F4FAA2797FDA095BA2F2091BC0128
:10836000332744275527BC01CD010E9450779B013C
:10837000AC0197FF04C0215C3F4F4F4F5F4F86E039
:1083800055954795379527958A95D1F78091C107DF
:108390009091C207821B930B9093C2078093C107F1
:1083A00080912C0687FF44C0B989BB2309F040C0E7
:1083B000809107038823E1F5E1E0EE16E1E0FE0697
:1083C0004CF08091D0079091D1078E0D9F1D805069
:1083D00091400DC0F0E0EF16FFEFFF0664F48091CE
:1083E000D0079091D1078E0D9F1D80509F4F909385
:1083F000D1078093D00721E0013012074CF0809123
:10840000BE079091BF07800F911F805091400CC014
:108410003FEF0030130764F48091BE079091BF07CF
:10842000800F911F80509F4F9093BF078093BE078E
:10843000E2E1CD5E0C94FB7780911803882301F56F
:108440008091ED028C7F8093ED02ADE4B4E0E9EE23
:10845000F6E09BE080910702882309F48C938D91CC
:10846000818312829150389697FFF4CF8091070252
:10847000882359F08091070281508093070205C03C
:108480008091ED0281608093ED02809172028823D9
:1084900019F010927202089580937402809376020C
:1084A000809170028E7F8093700285EA8093BC0079
:1084B0000895CF93DF93A2E2B3E0C4E2D6E057E0A1
:1084C0008991E82FFF27EE0FFF1FE65BF84F019021
:1084D000F081E02DE259FF4FEF3FF10521F01CF054
:1084E000EFEFF0E004C0F7FF02C0E0E0F0E04C91F5
:1084F000242F3327E217F307A9F0CF01821B930B38
:1085000097FD03969595879595958795242F280F28
:108510002C93822F9927E817F90714F4215001C0F2
:108520002F5F2C935150119657FFCACF80912E0682
:10853000883F38F0EFEFF0E0E81BF109EE5DFC4F0B
:1085400080818093CE018091CE01882329F08436EA
:1085500018F084E68093CE0180913006883F38F091
:10856000EFEFF0E0E81BF109EE5DFC4F80818093B6
:10857000CC018091CC01882329F0843618F084E660
:108580008093CC0180913D06883F38F0EFEFF0E01A
:10859000E81BF109EE5DFC4F80818093C70180915B
:1085A000C7018B3010F48AE002C08F3F11F4809332
:1085B000C70180916A06883F38F0EFEFF0E0E81BD2
:1085C000F109EE5DFC4F80818093EA078091EA0714
:1085D000823010F481E002C08F3F11F48093EA07EB
:1085E00080916C06883F38F0EFEFF0E0E81BF1096E
:1085F000EE5DFC4F808180931A0880911A088230CA
:1086000010F481E002C08F3F11F480931A0880912A
:108610005706883F38F0EFEFF0E0E81BF109EE5D18
:10862000FC4F80818093E50780915806883F38F0A1
:10863000EFEFF0E0E81BF109EE5DFC4F80818093E5
:10864000BB0780915906883F38F0EFEFF0E0E81B58
:10865000F109EE5DFC4F80818093F00790912F0629
:10866000983F18F49093CD0109C0EFEFF0E0E91BBB
:10867000F109EE5DFC4F80818093CD01983F18F4A5
:108680009093CD0109C0EFEFF0E0E91BF109EE5D39
:10869000FC4F80818093CD0180913206883F38F075
:1086A000EFEFF0E0E81BF109EE5DFC4F8081809375
:1086B000CB0180913406883F38F0EFEFF0E0E81B03
:1086C000F109EE5DFC4F80818093C90180913C06E9
:1086D000883F38F0EFEFF0E0E81BF109EE5DFC4F6A
:1086E00080818093CA0180913E06883F38F0EFEF89
:1086F000F0E0E81BF109EE5DFC4F80818093C6013C
:1087000080913F06883F38F0EFEFF0E0E81BF10979
:10871000EE5DFC4F80818093C80180914006883FC8
:1087200038F0EFEFF0E0E81BF109EE5DFC4F8081DF
:108730008093C50180914106883F38F0EFEFF0E06B
:10874000E81BF109EE5DFC4F80818093C4018091AC
:108750004706883F38F0EFEFF0E0E81BF109EE5DE7
:10876000FC4F80818093C20180914806883F38F099
:10877000EFEFF0E0E81BF109EE5DFC4F80818093A4
:10878000020380914906883F38F0EFEFF0E0E81BE4
:10879000F109EE5DFC4F80818093010380914A06D0
:1087A000883F38F0EFEFF0E0E81BF109EE5DFC4F99
:1087B00080818093000380914B06883F38F0EFEF73
:1087C000F0E0E81BF109EE5DFC4F80818093FF0231
:1087D00080916506883F38F0EFEFF0E0E81BF10983
:1087E000EE5DFC4F80818093FE0280916606883F9B
:1087F00038F0EFEFF0E0E81BF109EE5DFC4F80810F
:108800008093FD0280916706883F38F0EFEFF0E03B
:10881000E81BF109EE5DFC4F80818093FC028091A2
:108820006806883F38F0EFEFF0E0E81BF109EE5DF5
:10883000FC4F80818093FB0280914C06883F38F08A
:10884000EFEFF0E0E81BF109EE5DFC4F80818093D3
:10885000C10180915006883F38F0EFEFF0E0E81B4F
:10886000F109EE5DFC4F80818093C00180915A0632
:10887000883F38F0EFEFF0E0E81BF109EE5DFC4FC8
:1088800080818093BF0180915D06883F38F0EFEFD3
:10889000F0E0E81BF109EE5DFC4F80818093BE01A2
:1088A00080915E06883F38F0EFEFF0E0E81BF109B9
:1088B000EE5DFC4F80818093BD0180915F06883F13
:1088C00038F0EFEFF0E0E81BF109EE5DFC4F80813E
:1088D0008093BC0180916406883F38F0EFEFF0E0B0
:1088E000E81BF109EE5DFC4F80818093BB01809114
:1088F0007F06883F38F0EFEFF0E0E81BF109EE5D0E
:10890000FC4F808180932D088091C201282F33274E
:108910002F5F3F4F8CE398E2B9010E948F777093ED
:10892000D0016093CF0180913A0680931B0880911B
:1089300039068093D60790918106933320F181E028
:108940008093FA02983F58F0EFEFF0E0E91BF1094D
:10895000EE5DFC4F8081823310F41092FA02809118
:108960006D0890916E0897FF08C08091FA028823E5
:1089700021F080914804806803C0809148048F777B
:108980008093480402C01092FA0280916D08909181
:108990006E0897FF1DC0809118038823C9F080914D
:1089A000FA028823A9F080910801909109018F5F54
:1089B0009F4F71F488E99AE39093290280932802EB
:1089C00080E094EA90930901809308011092FA02E2
:1089D0008091FA02882339F08091BE01823D18F41B
:1089E000825E8093BE01DF91CF910895A8E1B0E04F
:1089F000ECEFF4E40C94DF770E946A3A30910201C4
:108A00003C3010F4299A01C02998E0901903F090A5
:108A10001A03FA82E9828091D60799270A96E81606
:108A2000F90614F49A83898380912103843608F02F
:108A30005CC08091BD039091BE03009731F0019717
:108A40009093BE038093BD0307C0109218038091DA
:108A5000ED028F7E8093ED023A3011F0343110F048
:108A6000289A01C028988091EE029091EF02895EC9
:108A70009340C0F180914406282F33273A832983FD
:108A80008091ED0280618093ED0280912006A82FF5
:108A9000BB27AA0FBB1FFD01E258F84F11821082BD
:108AA00080912106282F3327220F331FC9018258B6
:108AB000984FFC0111821082A65BB84F11961C9250
:108AC0001E92265B384FD90111961C921E928091FE
:108AD0002306E82FFF27EE0FFF1FE65BF84F1182FA
:108AE0001082C9C210921803C6C2809121038D382A
:108AF00008F4C1C28091ED028F7E8093ED029091C7
:108B0000450682E3989FC00111249093BE03809391
:108B1000BD03E981FA81B9978CF08091180388230D
:108B200069F08091EE029091EF02FFEF8F3F9F0777
:108B300029F001969093EF028093EE028091EE026D
:108B40009091EF028F3F910509F038F510923D03A7
:108B500010923E0310923F0310924003109239038B
:108B600010923A0310923B0310923C031092A90317
:108B70001092AA031092AB031092AC03109245031B
:108B80001092460310924703109248038A3F9105C2
:108B900049F481E08093C30305C08091ED028260B7
:108BA0008093ED0280912206E82FFF27EE0FFF1F32
:108BB000E65BF84F80819181813591050CF441C1CC
:108BC00020911803222309F03CC180912306E82F4D
:108BD000FF27EE0FFF1FE65BF84F808191818C34F9
:108BE00091050CF406C18091BF038F5F8093BF0392
:108BF000893C08F426C13C3010F4299801C0299A18
:108C0000109218031092BF031092EF021092EE021E
:108C100030912006E32FFF27EE0FFF1FE65BF84F92
:108C20008081918187349105B4F480912106E82FE9
:108C3000FF27EE0FFF1FE65BF84F808191810190C7
:108C4000F081E02DF7FF03C0F095E195FF4FE73489
:108C5000F1050CF478C041E020912106A22FBB273A
:108C6000AA0FBB1FA65BB84F8D919C9111978734BB
:108C7000910544F0E32FFF27EE0FFF1FE65BF84F4F
:108C8000808191818D919C918734910574F08091C0
:108C90002006E82FFF27EE0FFF1FE65BF84F8081CD
:108CA0009181873491050CF042E0E22FFF27EE0F0F
:108CB000FF1FE65BF84F808191818634910574F443
:108CC00080912006E82FFF27EE0FFF1FE65BF84F8D
:108CD00080819181873491050CF043E0E22FFF27DA
:108CE000EE0FFF1FE65BF84F808191818A5B9F4FFB
:108CF00074F480912006E82FFF27EE0FFF1FE65B3C
:108D0000F84F80819181873491050CF044E0E22F87
:108D1000FF27EE0FFF1FE65BF84F808191818A5B92
:108D20009F4F74F480912006E82FFF27EE0FFF1F5E
:108D3000E65BF84F80819181863491050CF445E023
:108D4000842F0E94CC2C80912106E82FFF27EE0F64
:108D5000FF1FE65BF84F808191810190F081E02D4B
:108D6000F7FF03C0F095E195FF4F7E97BCF480912B
:108D70002006E82FFF27EE0FFF1FE65BF84F8081EC
:108D800091818A5B9F4F54F481E08093630488EE65
:108D900093E0909329028093280253C00E94A22D51
:108DA0000E94952C80E00E943607809146060E9422
:108DB000C47480912C0680FF10C0809114019091A2
:108DC0001501875B934038F480911401909115014F
:108DD0008E5E924010F40E94B91A1092260280E032
:108DE0000E94BC3781E08093C20380932602579A89
:108DF0001FC080819181855B9F4F0CF58091BF03DF
:108E00008F5F8093BF03893CE0F03C3010F42998D9
:108E100001C0299A109218031092BF031092EF021A
:108E20001092EE0281E00E94BC3781E08093C20381
:108E30000E94A22D68E770E00E94FA3602C02093DB
:108E4000BF0380912206E82FFF27EE0FFF1FE65B8E
:108E5000F84F808191818B5A9F4F0CF00CC130915B
:108E60001803E0912306332309F0DAC0FF27EE0F41
:108E7000FF1FE65BF84F80819181855B9F4F0CF06F
:108E8000CCC020918206E22FFF27EE0FFF1FE65B8A
:108E9000F84F80819181855B9F4F1CF0222309F060
:108EA000BCC08091C0038F5F8093C003893C08F4ED
:108EB000E2C03093C00380914804882309F0A6C023
:108EC0008091C203882309F4A1C081E090E09093CF
:108ED000EF028093EE0281E0809318031092A903C1
:108EE0001092AA031092AB031092AC0310924503A8
:108EF00010924603109247031092480310924103C8
:108F000010924203109243031092440380913B0657
:108F1000E82EFF2400271127809117089091180848
:108F20009C01442737FD4095542FC801B7010E948A
:108F30005077DC01CB018093550390935603A093A7
:108F40005703B093580380912A0890912B089C01F5
:108F5000442737FD4095542FC801B7010E94507730
:108F6000DC01CB0180934D0390934E03A0934F03FC
:108F7000B09350038091750390917603A09177038D
:108F8000B09178038093510390935203A0935303BD
:108F9000B093540380916D0390916E03A0916F0381
:108FA000B09170038093490390934A03A0934B03BD
:108FB000B0934C0310923D0310923E0310923F0376
:108FC000109240031092390310923A0310923B031F
:108FD00010923C038091ED0288608093ED029091A5
:108FE00080068FE0989F9001112480913303909127
:108FF0003403820F931F68E671E00E948F7797FD1C
:109000000196959587958093790335C08CED95E011
:1090100090932902809328022EC01092C0032BC087
:10902000FF27EE0FFF1FE65BF84F808191818C34A4
:109030009105FCF020918206E22FFF27EE0FFF1F23
:10904000E65BF84F80819181855B9F4F14F022236E
:1090500081F48091C1038F5F8093C103893C58F0F4
:10906000109218031092C1031092EF021092EE02B8
:1090700002C01092C10380919401815080939401A9
:10908000809194018F3F21F08091ED0284FF72C3A3
:109090000E9459428091CC039091CD039C01220FF4
:1090A000331F280F391FC0902006AC2DBB27AA0FF5
:1090B000BB1FFD01E65BF84FB09036064B2D5527E0
:1090C00080819181849FF001859FF00D949FF00D28
:1090D00011242E0F3F1F37FF02C02D5F3F4FB901F4
:1090E0007595679575956795A258B84F8091370625
:1090F000082F11278D919C91809F7001819FF00C0A
:10910000909FF00C11246E0D7F1D7093CD03609322
:10911000CC038091CE039091CF039C01220F331F8B
:10912000280F391FD0902106AD2DBB27AA0FBB1FDA
:10913000FD01E65BF84F80819181849FF001859F5E
:10914000F00D949FF00D11242E0F3F1F37FF02C02A
:109150002D5F3F4FA9015595479555954795A258C5
:10916000B84F8D919C91809F7001819FF00C909FD2
:10917000F00C11244E0D5F1D5093CF034093CE038E
:109180008091FA02882309F448C0CB0177FD039649
:10919000DC01B595A795B595A795CA0157FD03962E
:1091A000FC01F595E795F595E7958091EE01682F1F
:1091B000772767FD70956A9F90016B9F300D7A9FAE
:1091C000300D112480910404482F552747FD5095F8
:1091D0004E9FC0014F9F900D5E9F900D1124280F50
:1091E000391F37FF02C0295F3F4F03E035952795B0
:1091F0000A95E1F73093200320931F036E9F90019F
:109200006F9F300D7E9F300D11244A9FC0014B9FF0
:10921000900D5A9F900D11243FC080918006E82F39
:10922000FF27E456FE4F86818093EE019081909354
:109230000404A82FBB27A7FDB095A69F9001A79F68
:10924000300DB69F300D1124E92FFF27E7FDF09573
:10925000E49FC001E59F900DF49F900D1124280F0D
:10926000391F37FF02C0295F3F4F13E0359527951F
:109270001A95E1F73093200320931F03A49F9001D8
:10928000A59F300DB49F300D1124E69FC001E79FCC
:10929000900DF69F900D1124281B390B37FF02C04B
:1092A000295F3F4FF3E035952795FA95E1F7309325
:1092B0001E0320931D0380912306E82FFF27EE0F46
:1092C000FF1FE65BF84F80819181909581959F4FBC
:1092D00090931C0380931B038330910514F0029735
:1092E00005C00FEF8E3F900734F4029690931C0355
:1092F00080931B0304C010921C0310921B038091E7
:109300000004909101042091FC033091FD03820F31
:10931000931F00911F0310912003081B190B10933A
:10932000200300931F038091FE039091FF0320917F
:10933000FA033091FB03820F931F80901D039090DE
:109340001E03881A990A90921E0380921D03809131
:109350002206E82FFF27EE0FFF1FE65BF84FE080A5
:10936000F18028E730E0E20EF31EF0921A03E0925B
:1093700019038091C7019927AA2797FDA095BA2FB5
:10938000BC01CD010E94F876DC01CB0120E030E089
:1093900040E251E4BC01CD010E949976DC01CB0191
:1093A000BC01CD010E94DB76DC01CB018093240857
:1093B0008091C6018093F3078091C5019927AA2760
:1093C00097FDA095BA2FBC01CD010E94F876DC0173
:1093D000CB0120E030E040E251E4BC01CD010E942D
:1093E0009976DC01CB01BC01CD010E94DB76DC016A
:1093F000CB018093C7078091C4018093DE078091E1
:109400006F0480FF59C080912D08813808F454C042
:1094100080916804992787FD90952B2D3327829F93
:10942000A001839F500D929F500D1124040F151F12
:109430001093200300931F0380916904992787FDEF
:109440009095829FB001839F700D929F700D1124A3
:10945000860E971E90921E0380921D0380916A04CF
:10946000282F332727FD309580911B0390911C03F3
:10947000820F931F90931C0380931B0380916C04B5
:10948000282F332727FD3095809131069927289F73
:10949000D001299FB00D389FB00D1124B0939B01CE
:1094A000A0939A0180916B0499278E159F0524F44F
:1094B00090931A03809319038091190390911A03D2
:1094C00097FF04C010921A031092190380912C0682
:1094D00082FF02C01092F30740911F0350912003B6
:1094E000CA0157FD03969C0135952795359527951B
:1094F00037FF03C0309521953F4F8091F202909144
:10950000F30282179307B4F4CA0157FF03C0909582
:1095100081959F4F97FD039695958795959587958E
:109520009093F3028093F2028536910544F084E62D
:1095300090E001C001979093F3028093F202409172
:109540001D0350911E03CA0157FD03969C013595DA
:1095500027953595279537FF03C0309521953F4FC7
:109560008091F0029091F10282179307B4F4CA013E
:1095700057FF03C0909581959F4F97FD0396959552
:109580008795959587959093F1028093F0028536A3
:10959000910544F084E690E001C001979093F102B8
:1095A0008093F0028091ED0284FF08C01092F302D4
:1095B0001092F2021092F1021092F002ED2DFF27AC
:1095C000EE0FFF1FE65BF84F40915B06242F332719
:1095D000808191812817390744F48091830682FFA6
:1095E00004C081E08093060313C0ED2DFF27EE0F2A
:1095F000FF1FE65BF84F842F992720915C06821BA2
:109600009109208131812817390714F4109206033B
:1096100040912106E42FFF27EE0FFF1FE65BF84F76
:1096200050915B06852F992722273327281B390B5A
:10963000808191818217930744F48091830683FF90
:1096400004C081E08093050316C080910503882340
:1096500091F0E42FFF27EE0FFF1FE65BF84F80919C
:109660005C069927851B9109208131818217930718
:1096700014F410920503EC2DFF27EE0FFF1FE65B9D
:10968000F84F40915B06242F332780819181281762
:10969000390744F48091830680FF04C081E0809301
:1096A000030317C080910303882399F0EC2DFF2753
:1096B000EE0FFF1FE65BF84F842F992720915C0681
:1096C000821B9109208131812817390714F41092E7
:1096D000030340912006E42FFF27EE0FFF1FE65BF8
:1096E000F84F50915B06852F992722273327281B97
:1096F000390B808191818217930744F4809183060E
:1097000081FF04C081E08093040316C080910403AC
:10971000882391F0E42FFF27EE0FFF1FE65BF84F41
:1097200080915C069927851B9109208131818217E0
:10973000930714F41092040380910603882319F40C
:1097400080910503811181E08093070380910303D9
:10975000882321F480910403882351F081E08093D1
:10976000080310920703109206031092050302C02B
:109770008093080380910703882321F480910803D4
:10978000882369F080915A069927E981FA818E171A
:109790009F0714F49A83898381E080932D0380913D
:1097A000ED0284FF1AC010921C0310921B0310924A
:1097B000200310921F0310921E0310921D039AE5BE
:1097C0009093240888E78093F3079093C7078093CA
:1097D000DE0710920703109208038091E107909131
:1097E000E207A091E307B091E4072091750330915F
:1097F00076034091770350917803820F931FA41F43
:10980000B51F8093E1079093E207A093E307B0931D
:10981000E4078091EB079091EC07A091ED07B091E0
:10982000EE0720906D0330906E0340906F035090D0
:109830007003820D931DA41DB51D8093EB079093BB
:10984000EC07A093ED07B093EE078091D8079091B5
:10985000D907A091DA07B091DB07E0907103F0908F
:1098600072030091730310917403EB82FC820D83E9
:109870001E838E0D9F1DA01FB11F8093D80790934C
:10988000D907A093DA07B093DB078091C8079091BE
:10989000C907A091CA07B091CB07E0906903F09087
:1098A0006A0300916B0310916C03EF82F8860987BD
:1098B0001A878E0D9F1DA01FB11F8093C80790931C
:1098C000C907A093CA07B093CB07F0900803FB86A3
:1098D000FF2029F480910703882309F460C01092C7
:1098E000650310926603109267031092680310924A
:1098F000610310926203109263031092640310924A
:10990000E1071092E2071092E3071092E407109229
:10991000EB071092EC071092ED071092EE071092F1
:10992000D8071092D9071092DA071092DB0710922D
:10993000C8071092C9071092CA071092CB078091EE
:10994000550390915603A0915703B091580380930B
:10995000510390935203A0935303B0935403809107
:109960004D0390914E03A0914F03B091500380930B
:10997000490390934A03A0934B03B0934C03109276
:1099800038021092370210920C0310920B031092BF
:109990000E0310920D030B85002309F0F2C1809194
:1099A0000703882309F0EDC18091110690911206FA
:1099B000815092402CF480911803882309F4E1C16E
:1099C00090909A08A0903B06609117087091180833
:1099D000788F6F8B80912A0890912B089A8B898BB6
:1099E0009FEF991609F4D9C0BB24CC24DD24CA0109
:1099F000B901A60195010E94C47779018A01EF8916
:109A0000F88DCF01AA2797FDA095BA2FE81AF90A79
:109A10000A0B1B0BC201B101A60195010E94C4777C
:109A200059016A0129893A89C901AA2797FDA09598
:109A3000BA2FA81AB90ACA0ADB0A292C332427FC30
:109A40003094432C532CC801B701A20191010E940C
:109A5000507797FF04C061507E4F8F4F9F4F3B015F
:109A60004C0109E095948794779467940A95D1F70F
:109A7000C601B501A20191010E94507797FF04C071
:109A800061507E4F8F4F9F4F5B016C0119E0D59461
:109A9000C794B794A7941A95D1F78091F202909148
:109AA000F302813491053CF48091F0029091F1022F
:109AB00081349105D4F0D401C30197FE03C001960F
:109AC000A11DB11D3C014D01959487947794679435
:109AD000D601C501D7FE03C00196A11DB11D5C01D1
:109AE0006D01D594C794B794A79480912306E82F6D
:109AF000FF27EE0FFF1FE65BF84F808191810190F9
:109B0000F081E02DF7FF03C0F095E195FF4F7A97C4
:109B1000A4F0C401B30123E030E040E050E00E9433
:109B2000C47739014A01C601B50123E030E040E0C5
:109B300050E00E94C47759016A0180919C08282F47
:109B4000332727FD3095432F532F2615370548051A
:109B5000590514F439014A01992787FD909590958C
:109B600081959F4FAA2797FDA095BA2F6816790671
:109B70008A069B0614F43C014D012A153B054C0551
:109B80005D0514F459016A01A816B906CA06DB0678
:109B90000CF0CFC05C016D01CCC0EA2CFF24002783
:109BA0001127CA01B901A80197010E94C4773901A0
:109BB0004A014F89588DCA01AA2797FDA095BA2F4F
:109BC000681A790A8A0A9B0AC201B101A8019701A1
:109BD0000E94C47759016A0169897A89CB01AA2751
:109BE00097FDA095BA2FA81AB90ACA0ADB0AD401B0
:109BF000C30197FE03C00F96A11DB11D3C014D018D
:109C0000F4E09594879477946794FA95D1F7D60108
:109C1000C501D7FE03C00F96A11DB11D5C016D01EA
:109C2000E4E0D594C794B794A794EA95D1F78091CE
:109C3000F2029091F302813491053CF48091F0029C
:109C40009091F10281349105A4F0C401B30123E0A5
:109C500030E040E050E00E94C47739014A01C6017B
:109C6000B50123E030E040E050E00E94C4775901A4
:109C70006A0180912306E82FFF27EE0FFF1FE65BA6
:109C8000F84F808191810190F081E02DF7FF03C0B2
:109C9000F095E195FF4F7A97A4F0C401B30123E05A
:109CA00030E040E050E00E94C47739014A01C6012B
:109CB000B50123E030E040E050E00E94C477590154
:109CC0006A0171E267167104810491042CF070E25C
:109CD000672E712C812C912C80EE68168FEF780600
:109CE0008FEF88068FEF980644F460EE662E6FEFD4
:109CF000762E6FEF862E6FEF962E91E2A916B104A5
:109D0000C104D1042CF050E2A52EB12CC12CD12CD1
:109D1000A0EEAA16AFEFBA06AFEFCA06AFEFDA06AB
:109D200044F440EEA42E4FEFB42E4FEFC42E4FEF6D
:109D3000D42E8091550390915603A0915703B09172
:109D4000580386199709A809B90980935503909378
:109D50005603A0935703B093580380914D039091FD
:109D60004E03A0914F03B09150038A199B09AC098F
:109D7000BD0980934D0390934E03A0934F03B0937E
:109D8000500380913702909138028F3F910509F07E
:109D900008F4C4C5BB85BB2309F04EC580910703F9
:109DA000882309F049C580912D03882309F044C513
:109DB000E0916306EC87EE2309F43EC58091E1074C
:109DC0009091E207A091E307B091E407B7FF04C0C8
:109DD00081509F4FAF4FBF4FE92EFA2E0B2F112707
:109DE00007FD1A95E092E107F092E2070093E3077E
:109DF0001093E4078091EB079091EC07A091ED0799
:109E0000B091EE07B7FF04C081509F4FAF4FBF4FD7
:109E1000892F9A2FAB2FBB27A7FDBA958D879E87D9
:109E2000AF87B88B8093EB079093EC07A093ED0777
:109E3000B093EE0780913B06A82EBB24CC24DD24F2
:109E40002091650330916603409167035091680348
:109E5000C601B5010E94507797FF04C061507F4F43
:109E60008F4F9F4F672E782E892E992487FC9A94C6
:109E70006092650370926603809267039092680314
:109E80002091610330916203409163035091640318
:109E9000C601B5010E94507797FF04C061507F4F03
:109EA0008F4F9F4F272E382E492E552447FC5A940A
:109EB00020926103309262034092630350926403E4
:109EC00080915D0390915E03A0915F03B091600368
:109ED000B7FF04C081509F4FAF4FBF4F892F9A2FBC
:109EE000AB2FBB27A7FDBA9580935D0390935E03CC
:109EF000A0935F03B0936003D801C7018619970947
:109F0000A809B9098093B5039093B603A093B7034A
:109F1000B093B80320916206E22EFF240027112798
:109F2000BC01CD01A80197010E94C47759016A01C3
:109F30002093C4033093C5034093C6035093C703D3
:109F40008D859E85AF85B88982199309A409B509C5
:109F50008093B9039093BA03A093BB03B093BC035F
:109F6000BC01CD01A80197010E94C4772093C803CA
:109F70003093C9034093CA035093CB03D601C50164
:109F8000D7FE04C081509F4FAF4FBF4F892F9A2FEC
:109F9000AB2FBB27A7FDBA9590930C0380930B03BF
:109FA00057FF04C021503F4F4F4F5F4FBB2757FD16
:109FB000BA95A52F942F832F90930E0380930D03B2
:109FC0008091F2029091F30281349105DCF480914A
:109FD000F0029091F10281349105A4F4809123065E
:109FE000E82FFF27EE0FFF1FE65BF84F808191817E
:109FF0000190F081E02DF7FF03C0F095E195FF4F50
:10A000007A97E4F080919A088F3FC1F480910B0316
:10A0100090910C0397FD01969595879590930C036D
:10A0200080930B0380910D0390910E0397FD019691
:10A030009595879590930E0380930D038091D80793
:10A040009091D907A091DA07B091DB07B7FF04C060
:10A0500081509F4FAF4FBF4F892F9A2FAB2FBB27F8
:10A06000A7FDBA958093D8079093D907A093DA07F4
:10A07000B093DB078091C8079091C907A091CA07E8
:10A08000B091CB07B7FF04C081509F4FAF4FBF4F78
:10A09000892F9A2FAB2FBB27A7FDBA958093C807AE
:10A0A0009093C907A093CA07B093CB07809175031B
:10A0B00090917603A0917703B09178032B813C8136
:10A0C0004D815E81281B390B4A0B5B0B2093AD033E
:10A0D0003093AE034093AF035093B00380916D0370
:10A0E00090916E03A0916F03B0917003EF80F8849C
:10A0F00009851A85E81AF90A0A0B1B0BE092B103CD
:10A10000F092B2030093B3031093B4032093B5030A
:10A110003093B6034093B7035093B803E092B9036A
:10A12000F092BA030093BB031093BC0380915103D8
:10A1300090915203A0915303B0915403821B930B4F
:10A14000A40BB50B8093510390935203A093530338
:10A15000B09354038091490390914A03A0914B031B
:10A16000B0914C038E199F09A00BB10B809349034A
:10A1700090934A03A0934B03B0934C03FC85FF23B9
:10A18000E1F020912B0330912C03213831054CF064
:10A190008091860390918703019690938703809323
:10A1A000860320583F4F4CF480918603909187039B
:10A1B0000197909387038093860310922C0310924B
:10A1C0002B0381E090E09093D1038093D003E09043
:10A1D000B503F090B6030091B7031091B803D8010E
:10A1E000C70117FF07C088279927DC018E199F092F
:10A1F000A00BB10B81509240A040B04034F084E0FD
:10A2000090E09093D1038093D0038091D6039091F6
:10A21000D703A091D803B091D9032091E1073091E1
:10A22000E2074091E3075091E407821B930BA40BD4
:10A23000B50B815E914BAF4FBF4F8F539C49A040F0
:10A24000B04028F080919B0889310CF4FFC041E0B8
:10A25000E41640E1F40640E0040740E014070CF483
:10A2600073C08091D203882309F46AC0D801C70162
:10A2700017FF07C088279927DC018E199F09A00BBB
:10A28000B10B9C01AD01B7FF04C021503E4F4F4FB1
:10A290005F4FF9E05595479537952795FA95D1F792
:10A2A0008091D0039091D103820F931F9093D1039B
:10A2B0008093D003D801C70117FF03C00796A11DE3
:10A2C000B11DE3E0B595A79597958795EA95D1F7E8
:10A2D0008093C4039093C503A093C603B093C703B0
:10A2E00089589341A040B04064F088E893E1A0E031
:10A2F000B0E08093C4039093C503A093C603B093CA
:10A30000C7032091C4033091C5034091C603509107
:10A31000C70357FF04C021503F4F4F4F5F4F232FBC
:10A32000342F452F552747FD5A9580910B03909167
:10A330000C03820F931F90930C0380930B0306C0B2
:10A3400081E08093D20302C01092D20360E0E6164F
:10A3500060EFF6066FEF06076FEF16070CF073C09D
:10A360008091D303882309F46AC0D801C70117FF7D
:10A3700007C088279927DC018E199F09A00BB10B14
:10A380009C01AD01B7FF04C021503E4F4F4F5F4FBE
:10A3900069E055954795379527956A95D1F780914E
:10A3A000D0039091D103820F931F9093D103809398
:10A3B000D003D801C70117FF03C00796A11DB11D27
:10A3C00023E0B595A795979587952A95D1F7809322
:10A3D000C4039093C503A093C603B093C7038857E3
:10A3E0009C4EAF4FBF4F64F488E79CEEAFEFBFEFDA
:10A3F0008093C4039093C503A093C603B093C7038F
:10A400002091C4033091C5034091C6035091C70306
:10A4100057FF04C021503F4F4F4F5F4F232F342F22
:10A42000452F552747FD5A9580910B0390910C03BA
:10A43000820F931F90930C0380930B0311C081E054
:10A440008093D3030DC01092D3030AC01092D1039E
:10A450001092D00388EE93E09093DA018093D901B3
:10A460008C85282F33278091D0039091D103281712
:10A47000390724F43093D1032093D00310919B0823
:10A48000112379F0212F332727FD30958091D003B8
:10A490009091D1032817390724F43093D1032093E6
:10A4A000D0034091B5035091B6036091B70370910A
:10A4B000B803413851056105710574F080918A0334
:10A4C00090918B032091D0033091D103820F931F81
:10A4D00090938B0380938A0340585F4F6F4F7F4F59
:10A4E00074F480918A0390918B032091D003309172
:10A4F000D103821B930B90938B0380938A0381E09B
:10A5000090E09093D1038093D003C090B903D09092
:10A51000BA03E090BB03F090BC03D701C601F7FE7D
:10A5200007C088279927DC018C199D09AE09BF094E
:10A5300081509240A040B04034F084E090E090938D
:10A54000D1038093D0038091DA039091DB03A09133
:10A55000DC03B091DD032091EB073091EC074091D3
:10A56000ED075091EE07821B930BA40BB50B815E98
:10A57000914BAF4FBF4F8F539C49A040B04018F054
:10A5800019310CF4FFC001E0C01600E1D00600E074
:10A59000E00600E0F0060CF473C08091D403882339
:10A5A00009F46AC0D701C601F7FE07C088279927BA
:10A5B000DC018C199D09AE09BF099C01AD01B7FFF3
:10A5C00004C021503E4F4F4F5F4F09E055954795CE
:10A5D000379527950A95D1F78091D0039091D103B3
:10A5E000820F931F9093D1038093D003D701C601AC
:10A5F000F7FE03C00796A11DB11D13E0B595A79501
:10A60000979587951A95D1F78093C8039093C903BE
:10A61000A093CA03B093CB0389589341A040B040A4
:10A6200064F088E893E1A0E0B0E08093C8039093E1
:10A63000C903A093CA03B093CB032091C803309100
:10A64000C9034091CA035091CB0357FF04C0215066
:10A650003F4F4F4F5F4F232F342F452F552747FD37
:10A660005A9580910D0390910E03820F931F909342
:10A670000E0380930D0306C081E08093D40302C0D3
:10A680001092D40320E0C21620EFD2062FEFE2068C
:10A690002FEFF2060CF073C08091D503882309F4E4
:10A6A0006AC0D701C601F7FE07C088279927DC01D9
:10A6B0008C199D09AE09BF099C01AD01B7FF04C00B
:10A6C00021503E4F4F4F5F4FE9E0559547953795E5
:10A6D0002795EA95D1F78091D0039091D103820F0D
:10A6E000931F9093D1038093D003D701C601F7FE47
:10A6F00003C00796A11DB11D73E0B595A795979569
:10A7000087957A95D1F78093C8039093C903A09356
:10A71000CA03B093CB0388579C4EAF4FBF4F64F42E
:10A7200088E79CEEAFEFBFEF8093C8039093C90317
:10A73000A093CA03B093CB032091C8033091C903FF
:10A740004091CA035091CB0357FF04C021503F4FA3
:10A750004F4F5F4F232F342F452F552747FD5A95D5
:10A7600080910D0390910E03820F931F90930E031F
:10A7700080930D0311C081E08093D5030DC010922A
:10A78000D5030AC01092D1031092D00388EE93E053
:10A790009093DA018093D9014C85242F332780913F
:10A7A000D0039091D1032817390724F43093D103B3
:10A7B0002093D00380919B08882379F0282F33279A
:10A7C00027FD30958091D0039091D1032817390748
:10A7D00024F43093D1032093D0034091B9035091D6
:10A7E000BA036091BB037091BC0341385105610508
:10A7F000710574F080918803909189032091D003B2
:10A800003091D103820F931F909389038093880323
:10A8100040585F4F6F4F7F4FCCF4809188039091E9
:10A8200089032091D0033091D103821B930B909325
:10A830008903809388030AC010920E0310920D03BF
:10A8400010920C0310920B0310922D038091F307CA
:10A85000882341F410920E0310920D0310920C0302
:10A8600010920B038091E1079091E207A091E3071A
:10A87000B091E4078093D6039093D703A093D803B5
:10A88000B093D9038091EB079091EC07A091ED076D
:10A89000B091EE078093DA039093DB03A093DC037F
:10A8A000B093DD0310926503109266031092670364
:10A8B0001092680310926103109262031092630376
:10A8C0001092640310925D0310925E0310925F0376
:10A8D000109260031092E1071092E2071092E307D2
:10A8E0001092E4071092EB071092EC071092ED071C
:10A8F0001092EE071092D8071092D9071092DA073B
:10A900001092DB071092C8071092C9071092CA076D
:10A910001092CB071092380210923702E0901B037E
:10A92000F0901C03C701F7FE04C0882799278E19F1
:10A930009F0940976CF088EE93E09093DA01809342
:10A94000D90180912C0684FD03C081E08093C3036C
:10A9500010913806A12EBB24CC24DD24B701882712
:10A9600077FD8095982F9701F7FE04C022273327A3
:10A970002E193F09442737FD4095542F0E945077E8
:10A980009B01AC01C601B5010E94507797FF04C03E
:10A9900061507E4F8F4F9F4F59E0959587957795E2
:10A9A00067955A95D1F79B01812F99278E9DD001EC
:10A9B0008F9DB00D9E9DB00D1124CD01B7FD039666
:10A9C0009595879595958795280F391F442737FDCD
:10A9D0004095542F2093A9033093AA034093AB03CF
:10A9E0005093AC038091450390914603A091470397
:10A9F000B0914803821B930BA40BB50B80934503C6
:10AA000090934603A0934703B09348038155934C1A
:10AA1000A040B04064F080E593ECA0E0B0E080930B
:10AA2000450390934603A0934703B0934803809156
:10AA3000450390914603A0914703B0914803805B82
:10AA40009C43AF4FBF4F64F480EB9CE3AFEFBFEF8D
:10AA50008093450390934603A0934703B093480324
:10AA600040903303509034034114510409F478C1E9
:10AA700080912C0683FF74C18091750390917603B9
:10AA8000A0917703B0917803B7FF04C081509E4F27
:10AA9000AF4FBF4F39E0B595A795979587953A95F4
:10AAA000D1F76C0197FF04C0D094C194D108D3941E
:10AAB00080916D0390916E03A0916F03B09170032C
:10AAC000B7FF04C081509E4FAF4FBF4F29E0B595EF
:10AAD000A795979587952A95D1F7BC0197FF03C055
:10AAE000709561957F4FC616D7060CF46B01B601C1
:10AAF000D7FE02C0695F7F4F3B0183E07594679486
:10AB00008A95E1F702E0E02EF12C6E0C7F1C0CE13F
:10AB100012E0400E511E72010027F7FC0095102F25
:10AB200024EE3DEF420E531E809126089091270897
:10AB3000A0912808B09129088090960190909701E3
:10AB4000A0909801B0909901BC01CD01A50194019C
:10AB50000E94C477E21AF30A040B150BC801B7016F
:10AB600028E631E040E050E00E94C477DC01CB01F0
:10AB70001CE4E12E1FEFF12EE80EF91E0091D90121
:10AB80001091DA010115110589F539E1C316D104D7
:10AB90006CF580912B0390912C038E0D9F1D90934B
:10ABA0002C0380932B038091C3038823F9F0C20107
:10ABB000AA2797FDA095BA2FBC01CD01A50194014C
:10ABC0000E945077DC01CB018093260890932708E0
:10ABD000A0932808B0932908BC01CD010E94C47736
:10ABE00030933203209331031092C303C701B4E0C2
:10ABF000880F991FBA95E1F7B3010E948F77CB01B7
:10AC0000AA2797FDA095BA2F2091260830912708F2
:10AC10004091280850912908280F391F4A1F5B1FAF
:10AC2000209326083093270840932808509329083A
:10AC3000F090CA016F2D7727C69EC001C79E900D68
:10AC4000D69E900D112497FD4F966C01A5E0D594EA
:10AC5000C794AA95E1F76C197D096B0177FD7AC05D
:10AC60000115110509F06FC00091F2021091F30275
:10AC70008091F0029091F102080F191F17FF02C096
:10AC8000095F1F4FF3E015950795FA95E1F7005C12
:10AC90001F4FCA01B901A50194010E94C477DA01CE
:10ACA000C9012091310330913203442737FD40958B
:10ACB000542F821B930BA40BB50B845E9D4FAF4F9B
:10ACC000BF4FBC01CD0128E631E040E050E00E94DA
:10ACD000C477DC01CB01845B90408C9DA0018D9DED
:10ACE000500D9C9D500D1124CA01B8010E948F7710
:10ACF00083E0F89E60011124C616D70614F4B6014D
:10AD000008C0882799278C199D09681779070CF4C2
:10AD1000BC019B01442737FD4095542F809145038A
:10AD200090914603A0914703B0914803820F931F6F
:10AD3000A41FB51F8093450390934603A093470338
:10AD4000B09348030DC0015010401093DA010093F6
:10AD5000D90106C084EF91E09093DA018093D90184
:10AD600080912D03882381F01092390310923A03C9
:10AD700010923B0310923C0310923D0310923E034D
:10AD800010923F0310924003F0900803FF20F1F46B
:10AD90008091F307282F3327442755278091750387
:10ADA00090917603A0917703B0917803BC01CD0117
:10ADB0000E945077DC01CB01BC01CD0128EF3AE2C3
:10ADC00040E050E00E94C477390102C06624772435
:10ADD000E0900703EE20F1F48091F307282F33274A
:10ADE0004427552780916D0390916E03A0916F03C6
:10ADF000B0917003BC01CD010E945077DC01CB0102
:10AE0000BC01CD0128EF3AE240E050E00E94C47757
:10AE1000290102C0442455248091C1079091C207A2
:10AE2000893C91051CF088EC90E005C088539F4F49
:10AE300034F488E39FEF9093C2078093C107809119
:10AE4000CD079091CE07893C91051CF088EC90E0ED
:10AE500005C088539F4F34F488E39FEF9093CE074B
:10AE60008093CD078091D0079091D107AA2797FDB5
:10AE7000A095BA2F20912408A22EBB24CC24DD2437
:10AE8000BC01CD01A60195010E9450779B01AC0148
:10AE90008091C1079091C207AA2797FDA095BA2F6C
:10AEA000E7E0880F991FAA1FBB1FEA95D1F7280F6B
:10AEB000391F4A1F5B1F57FF04C0215C3F4F4F4F94
:10AEC0005F4F76E055954795379527957A95D1F759
:10AED0008301020F131F1093D1070093D0078091B5
:10AEE000BE079091BF07AA2797FDA095BA2FBC0176
:10AEF000CD01A60195010E9450779B01AC01809184
:10AF0000CD079091CE07AA2797FDA095BA2F67E0AD
:10AF1000880F991FAA1FBB1F6A95D1F7280F391FE9
:10AF20004A1F5B1F57FF04C0215C3F4F4F4F5F4FCD
:10AF300096E055954795379527959A95D1F7420113
:10AF4000820E931E9092BF078092BE0780911F08C9
:10AF500090912008880F991FAA2797FDA095BA2FD6
:10AF60002091C707332744275527BC01CD010E94F4
:10AF700050775B016C0197FF08C08FE390E0A0E081
:10AF8000B0E0A80EB91ECA1EDB1E86E0D594C79499
:10AF9000B794A7948A95D1F78091DE07282F33279D
:10AFA000442755278091590390915A03A0915B0340
:10AFB000B0915C03BC01CD010E945077DC01CB0154
:10AFC000BC01CD0120EF35E540E050E00E94C477A0
:10AFD000B501620F731F7093200860931F08015022
:10AFE000104134F080E090E19093D1078093D00736
:10AFF0008091D0079091D1078050904F34F480E039
:10B0000090EF9093D1078093D007B1E08B16B0E119
:10B010009B0634F080E090E19093BF078093BE07D9
:10B020008091BE079091BF078050904F34F480E02C
:10B0300090EF9093BF078093BE076150704134F04A
:10B0400080E090E19093200880931F0880911F0872
:10B05000909120088050904F34F480E090EF9093CE
:10B06000200880931F0880910001482F5527809168
:10B070001E0190911F014817590794F420911E0159
:10B0800030911F0169817A81649FC001659F900D95
:10B09000749F900D1124B9010E947B777A83698394
:10B0A00089819A81880F991F880F991F9A838983B4
:10B0B00040912C0640FFBDC6EE2009F0BAC6FF2025
:10B0C00009F0B7C6AA24BB244501809109039091D9
:10B0D0000A039093F5058093F40520918C03309139
:10B0E0008D032115310509F03FC080911401909125
:10B0F00015018959934058F087B5853F20F4809118
:10B100003B02815011C081E08093E9034EC08091E1
:10B110001401909115018436910508F587B58B309F
:10B12000D0F080913B028F5F80933B029AE08902CE
:10B130009001112480911B06821B87BD8CE291E057
:10B1400090932902809328028EE591E090938D03DD
:10B1500080938C032AC081E08093E80326C0F0929C
:10B16000E803F092E90321C0809113039091140346
:10B17000A0911503B091160314E0880F991FAA1F20
:10B18000BB1F1A95D1F780933C0290933D02A09388
:10B190003E02B0933F02B0923A02A092390221508F
:10B1A000304030938D0320938C032091CD0141FFDB
:10B1B00024C02233D8F48091E30181508093E301CD
:10B1C0008F3FD9F510922E038091130390911403B1
:10B1D000A0911503B091160380930F039093100371
:10B1E000A0931103B093120381E004C081E0809327
:10B1F0002E0388EC8093E30120C080919A01909106
:10B200009B01820F911D209131063327829FF0010F
:10B21000839FF00D929FF00D1124CF01AA2797FD77
:10B22000A095BA2F80930F0390931003A09311035E
:10B23000B093120381E080932E0380917503909167
:10B240007603A0917703B0917803E0909601F09097
:10B2500097010091980110919901BC01CD01A801BD
:10B2600097010E94C47759016A0180916D03909102
:10B270006E03A0916F03B0917003BC01CD01A801D2
:10B2800097010E94C477B901C5010E947A6E8C01B2
:10B29000CC9714F00CE310E0C8010E941A6A8C01EC
:10B2A00080E28093950180912E03882309F447C49E
:10B2B0008091ED0299279C012071307084FD3FC47C
:10B2C0006091850660FD04C080912C0681FD0CC054
:10B2D000C980DA803093DF032093DE038091ED0292
:10B2E000806C8093ED0299C18091ED0281FF6BC16A
:10B2F0004091DF015091E001CA010F96209119039E
:10B3000030911A0382179307BCF58091E8038823D4
:10B3100099F58091ED0287FF15C08091ED028F773E
:10B320008093ED028091130390911403A091150373
:10B33000B091160380930F0390931003A093110311
:10B34000B09312038091ED0280648093ED02241B80
:10B35000350B2F50304037FF03C0309521953F4FBC
:10B360008091DE039091DF03820F931F9093DF03A0
:10B370008093DE038BE26EC0CA010F97281739074E
:10B38000BCF58091E903882399F58091ED0286FF51
:10B3900015C08091ED028F7B8093ED0280911303A5
:10B3A00090911403A0911503B091160380930F039D
:10B3B00090931003A0931103B09312038091ED02B8
:10B3C00080688093ED02241B350B215F3F4F37FFD0
:10B3D00003C0309521953F4F8091DE039091DF03AC
:10B3E000821B930B9093DF038093DE038DE232C0C8
:10B3F0008091ED02807C69F18091ED028F738093E2
:10B40000ED021092DF031092DE03209113033091BE
:10B410001403409115035091160320930F033093AA
:10B420001003409311035093120361FF06C084EF91
:10B4300091E090932902809328028091170388233A
:10B4400041F423333105410551051CF081E080931F
:10B4500017038DE3809395012091DE033091DF0384
:10B46000C90137FF04C088279927821B930B81509D
:10B4700092400CF491C0809131069927289F700169
:10B48000299FF00C389FF00C1124C70160E075E093
:10B490000E948F77CB01AA2797FDA095BA2F209104
:10B4A0000F03309110034091110350911203280FA4
:10B4B000391F4A1F5B1F20930F03309310034093E3
:10B4C0001103509312031092DF031092DE03C09019
:10B4D0001303D0901403E0901503F0901603D701E6
:10B4E000C60180509440A040B04082179307A40743
:10B4F000B5075CF4D701C60180509C4FAF4FBF4FDA
:10B50000281739074A075B0744F080930F0390938D
:10B510001003A0931103B09312038091850681FF5D
:10B5200006C084E690E090932902809328028091DF
:10B530003506882389F54091090350910A0357FF86
:10B5400002C04D5F5F4F5595479555954795809142
:10B550001E0190911F01209100013327489FB001E7
:10B56000499F700D589F700D1124CB01B9010E94A5
:10B570008F777093E0016093DF01663471051CF4EE
:10B5800086E490E005C06739710534F086E990E003
:10B590009093E0018093DF0180918C0390918D0363
:10B5A000892BB9F18091130390911403A091150395
:10B5B000B091160380930F0390931003A09311038F
:10B5C000B093120326C08091130390911403A091AD
:10B5D0001503B091160380599140A040B04080936C
:10B5E0000F0390931003A0931103B0931203809163
:10B5F0003506882311F0992702C088E790E09093E0
:10B60000E0018093DF0189819A8190930A038093FE
:10B610000903C0900903D0900A03209113033091CD
:10B62000140340911503509116032B8B3C8B4D8BCB
:10B630005E8B20910F0330911003409111035091C4
:10B6400012036B897C898D899E89261737074807E5
:10B65000590724F08091850680FDB8C280918C0343
:10B6600090918D03892B39F0C0900903D0900A0383
:10B67000AA24BB24D9C08B899C89AD89BE89821B31
:10B68000930BA40BB50B8093AD039093AE03A093E3
:10B69000AF03B093B003823070E897077FEFA7073E
:10B6A0007FEFB7072CF481E090E8AFEFBFEF09C060
:10B6B0008F5F9F47A040B04064F08FEF9FE7A0E00E
:10B6C000B0E08093AD039093AE03A093AF03B0932B
:10B6D000B003A090AD03B090AE038091CC01282FB1
:10B6E0003327442755278091AD039091AE03A09155
:10B6F000AF03B091B003BC01CD010E94507797FF1A
:10B7000004C0615E7F4F8F4F9F4FA5E09595879551
:10B7100077956795AA95D1F76093AD037093AE03C3
:10B720008093AF039093B0036530FEEF7F07FFEF88
:10B730008F07FFEF9F072CF484E09EEFAFEFBFEF82
:10B7400009C0605074408040904064F080E094E014
:10B75000A0E0B0E08093AD039093AE03A093AF035D
:10B76000B093B0038090AD039090AE032091390266
:10B7700030913A0237FF02C0295F3F4FF3E0359521
:10B780002795FA95E1F74FEF223834071CF421E8AA
:10B790003FEF05C02038310514F020E830E0C90142
:10B7A000AA2797FDA095BA2F2091CE0133274427D1
:10B7B0005527BC01CD010E94507797FF04C06D5FF3
:10B7C0007F4F8F4F9F4FE2E09595879577956795CF
:10B7D000EA95D1F79B015FEF613075071CF420E01B
:10B7E0003FEF06C06F3F710519F014F020E031E023
:10B7F0008091ED02807C49F0C90137FD03969C01E0
:10B8000035952795359527950DC08091850680FF44
:10B8100009C0C90137FD07969C0143E0359527957E
:10B820004A95E1F7820E931E2091CB01222309F461
:10B8300054C0609135037091360380913703909125
:10B84000380397FF04C061587F4F8F4F9F4F37E0F9
:10B8500095958795779567953A95D1F7332744273E
:10B8600055270E94507797FF04C0615E7F4F8F4F2E
:10B870009F4FB5E09595879577956795BA95D1F7E0
:10B880006093AD037093AE038093AF039093B003C6
:10B890006138AFEF7A07AFEF8A07AFEF9A072CF462
:10B8A00080E89FEFAFEFBFEF0AC06F3F71058105E2
:10B8B000910569F064F080E091E0A0E0B0E0809351
:10B8C000AD039093AE03A093AF03B093B003809108
:10B8D000AD039091AE03880E991E8091C901282F67
:10B8E000332780919E08992787FD9095289FF00126
:10B8F000299FF00D389FF00D11249F01F7FF02C022
:10B9000021583F4F220F232F221F330BFFEF2138E7
:10B910003F071CF420E83FEF06C02F3F310519F028
:10B9200014F020E031E0820E931EC401AA2797FD97
:10B93000A095BA2FE0900903F0900A0397014427DD
:10B9400037FD4095542FBC01CD010E94507797FFE1
:10B9500004C061507E4F8F4F9F4FF9E095958795BA
:10B9600077956795FA95D1F7C61AD70A8091DE03C5
:10B970009091DF03892B09F060C01E141F040CF0A6
:10B980005CC09501B7FE03C0309521953F4F2D3324
:10B99000310540F48091E2039091E3038C159D05FD
:10B9A00074F526C02C533040E5E036952795EA958E
:10B9B000E1F72031310510F02FE030E04091E20353
:10B9C0005091E3031A141B04E4F480E190E0821B1D
:10B9D000930B489F9001499F300D589F300D1124C3
:10B9E00074E0369527957A95E1F72C153D0520F5FD
:10B9F0008091E1019091E201C816D906F4F06C0142
:10BA00001CC0205F3F4F8091E1019091E201829F35
:10BA1000B001839F700D929F700D11249B0164E013
:10BA2000369527956A95E1F74C155D0514F06A0186
:10BA300004C0C216D30608F06901C601AA2797FD03
:10BA4000A095BA2F2DE0880F991FAA1FBB1F2A951A
:10BA5000D1F79801442737FD4095542FBC01CD0103
:10BA60000E94C4772093B1033093B2034093B30391
:10BA70005093B403C090B103D090B2038091E0031F
:10BA80009091E1039C01220F331F280F391F2C0DC9
:10BA90003D1D37FF02C02D5F3F4FA90155954795CA
:10BAA000559547955093E1034093E00380912D060F
:10BAB000282F3327220F331F220F331F2417350758
:10BAC0006CF480911B08282F3327220F331F220F7D
:10BAD000331F205530404217530724F03093E103C1
:10BAE0002093E0038091850680FF14C08091E003DD
:10BAF0009091E103A981BA818A179B0724F0B09342
:10BB0000E103A093E003E091E003F091E103FA8305
:10BB1000E9835CC029813A812E193F0937FF02C0B1
:10BB20002D5F3F4F3595279535952795E090E0039C
:10BB3000F090E103E20EF31EFA82E98247C08091A1
:10BB40003506882301F56091090370910A0377FF98
:10BB500002C06D5F7F4F75956795759567954091AC
:10BB60001E0150911F0180910001282F3327649FEF
:10BB7000C001659F900D749F900D1124B9010E9422
:10BB80008F77CB0101C099279093E0018093DF016B
:10BB90008091DF019091E001873491051CF486E4E7
:10BBA00090E005C08639910534F086E990E09093E5
:10BBB000E0018093DF0129813A813093E1032093F2
:10BBC000E0038091ED02806C8093ED028091ED02A4
:10BBD00099279C012270307081FF1CC18091E40381
:10BBE0009091E503A091E603B091E7030097A105CA
:10BBF000B10521F0809117038130B1F449815A8158
:10BC0000CA01AA2797FDA095BA2F2EE0880F991F89
:10BC1000AA1FBB1F2A95D1F78093E4039093E503F5
:10BC2000A093E603B093E70380911703813019F4E2
:10BC300082E08093170369817A81CB01AA2797FD5F
:10BC4000A095BA2F9801442737FD4095542FBC0189
:10BC5000CD010E945077DC01CB018093B10390931A
:10BC6000B203A093B303B093B403B7FF04C08150F1
:10BC7000904EAF4FBF4F7C018D01FDE015950795AC
:10BC8000F794E794FA95D1F7E092B103F092B203FA
:10BC90000093B3031093B4036091EE027091EF022E
:10BCA0008FE0603A780750F58091E4039091E503C6
:10BCB000A091E603B091E7039C01AD01EAE056953F
:10BCC000479537952795EA95D1F7821B930BA40BDF
:10BCD000B50BA8019701F4E0220F331F441F551F35
:10BCE000FA95D1F7820F931FA41FB51F8093E40329
:10BCF0009093E503A093E603B093E70360547F417C
:10BD000018F58091E4039091E503A091E603B091CA
:10BD1000E7039C01AD01ECE05695479537952795D3
:10BD2000EA95D1F7821B930BA40BB50BA8019701E1
:10BD300072E0220F331F441F551F7A95D1F7820FEF
:10BD4000931FA41FB51F29C08091390290913A0218
:10BD50008091390290913A0297FF03C090958195A6
:10BD60009F4F843691050CF58091E4039091E50393
:10BD7000A091E603B091E7039C01AD016EE05695FA
:10BD80004795379527956A95D1F7821B930BA40B9E
:10BD9000B50B8E0D9F1DA01FB11F8093E4039093E0
:10BDA000E503A093E603B093E7038091E403909149
:10BDB000E503A091E603B091E7031EE0B695A795D1
:10BDC000979587951A95D1F790930A038093090365
:10BDD00040913306442399F055279C01BA010E94F3
:10BDE0008F77C901861B970B9093E3038093E2033F
:10BDF000260F371F3093E2012093E1011FC01092FC
:10BE0000E3031092E2038FEF93E09093E2018093BB
:10BE1000E10114C0109217031092E4031092E5039D
:10BE20001092E6031092E70330930A03209309036C
:10BE300005C08091ED02806C8093ED022090D607C2
:10BE4000222D3327220F331F220F331F285D3F4F30
:10BE5000A981BA812A173B0714F03A8329833090CD
:10BE60001B08832D9927880F991F880F991F8055CC
:10BE70009040E981FA818E179F0714F49A83898391
:10BE800080917102882321F48091A7088F3FA1F04F
:10BE90008091EE029091EF020297C09768F4E980DA
:10BEA000FA801E141F0444F481E090E09093EF02A6
:10BEB0008093EE023A83298309811A811093D90570
:10BEC0000093D8058091A9039091AA03A091AB0398
:10BED000B091AC03F2E0880F991FAA1FBB1FFA951F
:10BEE000D1F700911F0810912008081B190B298118
:10BEF0003A81213A31058CF0C90137FD01969595BB
:10BF00008795801791070CF48C01909581959F4F30
:10BF1000081719076CF48C010BC00135110514F0DA
:10BF200000E510E03FEF003B130714F400EB1FEFB8
:10BF3000232D3327220F331F220F331FC9014981BD
:10BF40005A81841B950B801791070CF48C01698131
:10BF50007A81621B730B061717070CF48B01809113
:10BF6000D0079091D10760911F0370912003861B29
:10BF7000970B9093E0078093DF07D090F307209111
:10BF80003D0330913E0340913F0350914003DD203B
:10BF900041F0661A770AC301AA2797FDA095BA2F28
:10BFA00004C0AA2797FDA095BA2F280F391F4A1F52
:10BFB0005B1F20933D0330933E0340933F03509318
:10BFC000400380913D0390913E03A0913F03B091C7
:10BFD000400381509A4FA040B04064F080E09AEF57
:10BFE000A0E0B0E080933D0390933E03A0933F0315
:10BFF000B093400380913D0390913E03A0913F0395
:10C00000B091400380509640AF4FBF4F64F480E042
:10C0100096E0AFEFBFEF80933D0390933E03A09374
:10C020003F03B0934003C09042062091DF07309158
:10C03000E007F8E0FC1598F08C2D9927829F70019D
:10C04000839FF00C929FF00C1124C701F7FC079618
:10C050007C0163E0F594E7946A95E1F712C08C2DBA
:10C0600086959927829FA001839F500D929F500D26
:10C070001124CA0157FD03967C01F594E794F594C9
:10C08000E794A090CF01B090D0019501442737FDEF
:10C090004095542F80913D0390913E03A0913F0322
:10C0A000B0914003BC01CD010E94C477E20EF31EA3
:10C0B0009090BB01692D772788279927980117FF52
:10C0C00004C022273327201B310B37FF02C02F5F0C
:10C0D0003F4F35952795A981BA812A0F3B1F4427E9
:10C0E00037FD4095542F0E94507797FF04C0615C44
:10C0F0007F4F8F4F9F4F26E0959587957795679552
:10C100002A95D1F79B016E157F050CF47B013095C4
:10C1100021953F4FE216F3060CF479018091BE079A
:10C120009091BF0760911D0370911E03861B970BB2
:10C130009093BD078093BC072091390330913A0357
:10C1400040913B0350913C03DD2041F0461A570AD1
:10C15000C201AA2797FDA095BA2F04C0AA2797FD70
:10C16000A095BA2F280F391F4A1F5B1F2093390350
:10C1700030933A0340933B0350933C03809139033F
:10C1800090913A03A0913B03B0913C0381509A4FA8
:10C19000A040B04064F080E09AEFA0E0B0E080936F
:10C1A000390390933A03A0933B03B0933C038091EF
:10C1B000390390913A03A0913B03B0913C03805026
:10C1C0009640AF4FBF4F64F480E096E0AFEFBFEF13
:10C1D0008093390390933A03A0933B03B0933C03BD
:10C1E0002091BC073091BD0748E04C1598F08C2D8C
:10C1F0009927829FB001839F700D929F700D11242B
:10C20000CB0177FD07966C01B3E0D594C794BA953E
:10C21000E1F712C0C6948C2D9927829FD001839F8D
:10C22000B00D929FB00D1124CD01B7FD03966C01A6
:10C23000D594C794D594C7949501442737FD40956C
:10C24000542F8091390390913A03A0913B03B09110
:10C250003C03BC01CD010E94C477C20ED31E692DE0
:10C26000772788279927980117FF04C022273327AB
:10C27000201B310B37FF02C02F5F3F4F35952795AD
:10C28000E981FA812E0F3F1F442737FD4095542F37
:10C290000E94507797FF04C0615C7F4F8F4F9F4F84
:10C2A000E6E09595879577956795EA95D1F79B0197
:10C2B0006C157D050CF46B01309521953F4FC2162E
:10C2C000D3060CF4690169EE862E66E0962E50EADC
:10C2D000A52E56E0B52E4BE0542E38EF632E37E0F6
:10C2E000732ED5012C9112160CF014C1203429F4B0
:10C2F000E981FA81F88FEF8B1FC049815A81CA0109
:10C30000AA2797FDA095BA2F332727FD3095432FF5
:10C31000532FBC01CD010E94507797FF04C0615C90
:10C320007F4F8F4F9F4F26E095958795779567951F
:10C330002A95D1F7788F6F8BF5012181203439F45C
:10C340002F89388D2E0D3F1D388F2F8B2AC0203C12
:10C3500039F44F89588D4E195F09588F4F8B21C082
:10C36000C701AA2797FDA095BA2F332727FD30953F
:10C37000432F532FBC01CD010E94507797FF04C07B
:10C38000615C7F4F8F4F9F4FB6E09595879577956E
:10C390006795BA95D1F7AF89B88DA60FB71FB88F3B
:10C3A000AF8BF5012281203439F42F89388D2C0D83
:10C3B0003D1D388F2F8B2AC0203C39F44F89588D72
:10C3C0004C195D09588F4F8B21C0C601AA2797FDD4
:10C3D000A095BA2F332727FD3095432F532FBC014B
:10C3E000CD010E94507797FF04C0615C7F4F8F4F53
:10C3F0009F4FA6E09595879577956795AA95D1F774
:10C40000AF89B88DA60FB71FB88FAF8BF501238109
:10C41000203439F42F89388D200F311F388F2F8B1E
:10C420002AC0203C39F44F89588D401B510B588F3E
:10C430004F8B21C0C801AA2797FDA095BA2F33279B
:10C4400027FD3095432F532FBC01CD010E9450771B
:10C4500097FF04C0615C7F4F8F4F9F4FF6E095952B
:10C46000879577956795FA95D1F7AF89B88DA60F1F
:10C47000B71FB88FAF8BF301808191812F89388DE1
:10C480008217930764F4B901680F791F77FF02C020
:10C490006F5F7F4F75956795788F6F8B08C04F8959
:10C4A000588D440F551F481B590B588F4F8B822DA9
:10C4B0009927880F991F880F991F6F89788D861784
:10C4C00097075CF4832D9927880F991F880F991F70
:10C4D000AF89B88DA817B90714F0988F8F8B8F8903
:10C4E000988D97FD03969595879595958795F40179
:10C4F0008183880F991F880F991F2F89388D281BDA
:10C50000390BC901880F8283EF89F88DD301ED9330
:10C51000FC9303C0F401118212825A9422E030E0AD
:10C52000620E731E44E050E0A40EB51E68E070E099
:10C53000860E971E57FED5CEE2E1C85E0C94FB77BF
:10C540008091F6039091F703A091F803B091F9035D
:10C550008093EE039093EF03A093F003B093F10365
:10C560008091F2039091F303A091F403B091F5034D
:10C570008093EA039093EB03A093EC03B093ED0355
:10C58000089510920104109200041092FF0310927B
:10C59000FE03089584B1806A84B93D9A82E58CBD1A
:10C5A0001DBC459A81E0809332088AEA8093430853
:10C5B00083E8809344088AE08093450810924708F6
:10C5C00010924608109249081092480810929D084F
:10C5D00010926508089530913208332309F085C020
:10C5E0000DB407FE82C084E080932702459A2EB5E1
:10C5F0008091050499278130910589F08230910559
:10C600001CF4892B21F03EC00297B9F03BC0309357
:10C610006408209306042138A9F581E008C0253577
:10C6200049F480910604820F8093060482E080938F
:10C63000050428C03093050425C080916408E82FC4
:10C64000FF27E058F74F20838F5F80936408909115
:10C6500006048A31A0F0291769F48AE1A0E8B8E05D
:10C66000E6E6F8E00D9001928A95E1F781E080938B
:10C67000650802C0309365081092050403C0920F4C
:10C680009093060420914208203208F028C0459873
:10C69000000000000000000000000000000000009A
:10C6A000000000000000000000000000000000008A
:10C6B000000000000000000000000000000000007A
:10C6C000E0913B08F0913C08E20FF11D80818EBDA6
:10C6D000809162089081890F8093620803C081E095
:10C6E000809332082F5F209342080895EF92FF92C3
:10C6F0000F931F9380913B069927880F991F880FEE
:10C70000991F7C010027F7FC0095102F809175037D
:10C7100090917603A0917703B0917803BC01CD018D
:10C72000A80197010E94C4773093470820934608D8
:10C7300080916D0390916E03A0916F03B09170038F
:10C74000BC01CD01A80197010E94C477309349082C
:10C750002093480820912608309127084091280806
:10C7600050912908DA01C901E3E0880F991FAA1F37
:10C77000BB1FEA95D1F7820F931FA41FB51F820F2D
:10C78000931FA41FB51F20919601309197014091EE
:10C79000980150919901BC01CD010E94C47730935A
:10C7A0004F0820934E088091860390918703209133
:10C7B000470230914802821B930B90935508809357
:10C7C0005408E0917C03F0917D038091E8079091FB
:10C7D000E907BF010E948F77CB019B01220F331F16
:10C7E000220F331F280F391F280F391F37FF02C0B0
:10C7F0002D5F3F4F359527953595279530934B08FD
:10C8000020934A088091220890912308BF010E943A
:10C810008F779B01220F331F220F331F260F371FE5
:10C82000260F371F37FF02C02D5F3F4F35952795E5
:10C830003595279530934D0820934C0810927D0331
:10C8400010927C031092E9071092E80710922308D7
:10C85000109222088091450899278D30910509F49E
:10C8600066C08E3091055CF48B30910509F48EC062
:10C870008C3091050CF00FC10A9761F0ADC18F307B
:10C88000910509F481C18F3091050CF45CC140978A
:10C8900099F1A2C18091020380935608809101030F
:10C8A0008093570880910003809358088091FF027D
:10C8B000809359088091FE0280935A088091FD026E
:10C8C00080935B088091FC0280935C088091FB025E
:10C8D00080935D088091ED0280935E088091ED0267
:10C8E000837F8093ED020E94A22D80935F08809148
:10C8F00079038093600870C180919F089091A0088F
:10C9000090935708809356088091A3089091A408AB
:10C91000909359088093580880911E0190911F01AF
:10C9200080935A088091000180935B0855C18091E3
:10C930006F06809356088091700680935708809107
:10C9400071068093580880917206809359088091EF
:10C95000730680935A088091770680935B088091D4
:10C96000780680935C088091790680935D088091B9
:10C970007C0680935E0880917A0680935F088091A0
:10C980007B068093600880917D06DAC0F8948091E0
:10C990002206E82FFF27EE0FFF1FE65BF84F0190FE
:10C9A000F081E02DE038F1051CF0EFE7F0E006C083
:10C9B0002FEFE138F20714F4E1E8FFEFE0935608B7
:10C9C00080912306E82FFF27EE0FFF1FE65BF84F4D
:10C9D0000190F081E02DE038F1051CF0EFE7F0E088
:10C9E00006C06FEFE138F60714F4E1E8FFEFE093DB
:10C9F000570880912106E82FFF27EE0FFF1FE65B07
:10CA0000F84F0190F081E02DE038F1051CF0EFE7E0
:10CA1000F0E006C08FEFE138F80714F4E1E8FFEF2B
:10CA2000E093580880912006E82FFF27EE0FFF1FA4
:10CA3000E65BF84F0190F081E02DE038F1051CF045
:10CA4000EFE7F0E006C02FEFE138F20714F4E1E879
:10CA5000FFEF7894E09359088091220380935A085D
:10CA60008091230380935B088091240380935C086A
:10CA70008091250380935D088091260380935E0852
:10CA80008091270380935F0880912803809360083A
:10CA90008091290355C080916304863018F010926C
:10CAA000630485E08093560880917E068093570842
:10CAB0008091130390911403A0911503B091160374
:10CAC000BC01CD0125E030E040E050E00E94C47799
:10CAD000309359082093580880910F0390911003C8
:10CAE000A0911103B0911203BC01CD0125E030E00B
:10CAF00040E050E00E94C47730935B0820935A08CE
:10CB00008091740680935C088091750680935D081F
:10CB10008091760680935E088091210380935F0860
:10CB200080914A0790914B07809360088091D805C7
:10CB30009091D90597FD039695958795959587953D
:10CB40008093610849C01092560882E58093570887
:10CB50001092580880E180935908809102018093D7
:10CB60005A088091480480935B088091490480931F
:10CB70005C0880914A0480935D0880914B04809307
:10CB80005E0880914C0426C080915406809356081C
:10CB900080918406809357088091C1018093580842
:10CBA00080914D068093590880914E0680935A08D3
:10CBB00080914F0680935B088091C00180935C0850
:10CBC0008091510680935D088091520680935E08A3
:10CBD0008091530680935F0880916508882309F44B
:10CBE000D8C08AEF8093ED014091670850916808A2
:10CBF000CA0181509E4F8F5F9340B0F42091690825
:10CC000030916A08C90181509E4F8F5F934060F454
:10CC100080912C0685FF08C05093010440930004C6
:10CC20003093FF032093FE0380916D0890916E086E
:10CC300021E08936920724F49093340380933303E0
:10CC4000809133039091340320913103309132036A
:10CC5000821B930B845E9D4F68E671E00E948F7784
:10CC6000845B90409093300380932F032091710850
:10CC700030917208809128029091290282179307BF
:10CC800040F480916304882321F430932902209397
:10CC900028028091660899278836910549F18936DE
:10CCA000910524F48736910531F07BC089369105D2
:10CCB00009F445C076C08091730880939A088091EA
:10CCC000740880939C088091750880939B088091DC
:10CCD000760880939D088091770880939E088091C4
:10CCE00078088093EE01809179088093040459C0FC
:10CCF0008091730880933D088091740880933E086A
:10CD00008091750880933F08809176088093400851
:10CD100080917708809341088091C80590917808A8
:10CD2000892B8093C8059091790890930204809193
:10CD3000C90583709C70892B8093C90532C080918E
:10CD4000730880933308809174088093340880912D
:10CD50007508809335088091760880933608809115
:10CD600077089091780890933808809337088091DD
:10CD7000790890917A0890933A08809339088091C5
:10CD80007B08992787FD909590937D0780937C077A
:10CD900008C010920104109200041092FF03109238
:10CDA000FE031F910F91FF90EF900895809132083C
:10CDB000882309F43BC0459883E498E090933C08AD
:10CDC00080933B0890910304E92FFF27EC51FE4F1D
:10CDD0009F5F90930304808180934508993010F001
:10CDE00010920304109232080E94766381E08093CF
:10CDF00042080000000000000000000000000000E9
:10CE00000000000000000000000000000000000022
:10CE10000000000000000000000000000000000012
:10CE2000000080914308809362088EBD089587B109
:10CE30008C6087B9429843981092080480E88093E8
:10CE4000F001109207048093EF01089580910D0482
:10CE5000815080930D048F3F09F0FBC024E02093A4
:10CE60000D048091ED02992780739070892B21F435
:10CE70008091490480FF1CC080916D06882349F091
:10CE800080911004882311F42093080481E080939A
:10CE9000100480916E068823B9F0809111048823D4
:10CEA00019F484E08093070481E0809311040CC09E
:10CEB00010921004109211048091690680930E0460
:10CEC00080916B0680930F0480911004882309F0F1
:10CED00040C080918306282F332724FF07C080910C
:10CEE0001803882319F425FD4DC04EC090916A06A1
:10CEF000983F50F08091EA078D3D30F080910E040C
:10CF000088230CF43FC040C0983F48F08091EA0766
:10CF10008A3028F480910E048823B4F133C08091C4
:10CF200008048150809308048F3F79F58091EA07C7
:10CF30008150809308048091F001813011F480E8E1
:10CF400001C086958093F0018091F00190910E04CC
:10CF500017C0809108048150809308048F3FA9F482
:10CF600089E0809308048091F001813011F480E819
:10CF700001C086958093F0018091F00190916D063B
:10CF8000892311F0429A01C04298809111048823AC
:10CF900009F043C080918306282F332724FF07C060
:10CFA00080911803882319F426FD50C034C0909155
:10CFB0006C06983F50F080911A088D3D30F08091BA
:10CFC0000F0488230CF442C026C0983F48F080919B
:10CFD0001A088A3028F480910F048823E4F036C0C0
:10CFE000809107048150809307048F3F91F58091D1
:10CFF0001A088150809307048091EF01813011F469
:10D0000080E801C086958093EF018091EF019091B7
:10D010000F048923D9F4439808958091070481501F
:10D02000809307048F3FA9F489E0809307048091DF
:10D03000EF01813011F480E801C086958093EF0103
:10D040008091EF0190916E06892311F0439A089523
:10D05000439808954FB724E130E0F8948091C900D7
:10D060008F778093C9008091C9008F7B8093C9001E
:10D070008091C9008F7D8093C9005A9A52985B9A1B
:10D08000539A832F99278093CD002093CC008091D1
:10D09000C80082608093C80080E18093C9008091BD
:10D0A000CA008F778093CA008091CA008F7B8093DB
:10D0B000CA008091CA008F7D8093CA008091CA0007
:10D0C0008F7E8093CA008091CA00877F8093CA00B8
:10D0D0008091C9008B7F8093C9008091CA008460D1
:10D0E0008093CA008091CA0082608093CA008091B8
:10D0F000C80087FF03C08091CE00F9CF8091C9009E
:10D1000080688093C9004FBF0895EF92FF920F93FC
:10D110001F93CF93DF93482F00E010E08091F1013F
:10D12000813061F41092F10184E480931204109232
:10D13000140410921304109215042BC18091120450
:10D14000882319F421E030E001C098019091130484
:10D15000992371F4232B11F081E010C084E48093B3
:10D160001204909314049093130490931504FAC03E
:10D17000913069F4232B09F0EBC082E08093130413
:10D18000809114048F5F8093140483E0E9C092308F
:10D19000D1F4232B09F0DCC083E080931204409388
:10D1A000150490911404923039F41092160447FF3C
:10D1B00003C081E08093160483E0809313049F5F93
:10D1C00090931404CFC0933009F0C2C0232B09F010
:10D1D000BFC09093120482E08093130480911404E2
:10D1E0008F5F8093140420911504822F9927782F44
:10D1F0006627842F9927682B792B809146068130EA
:10D2000049F47370CB018050924063E070E00E945B
:10D210008F7717C0823061F47770CB0180509440D3
:10D2200066E070E00E948F772695269526950BC0C4
:10D23000737068567140CB0177FD0196BC017595FE
:10D24000679526952695022F11270F7010700F5F96
:10D250001F4F0D30110508F074C07801E00EF11E6B
:10D26000F701E65BF84F808191819B01281B390B08
:10D27000C90137FF03C0909581959F4F069794F49D
:10D2800080912103883C30F480912103865F809354
:10D29000210308C088EC8093210380916F008F7D6B
:10D2A00080936F00F701E65BF84F808191819C01CC
:10D2B000220F331F280F391F260F371F37FF02C0D9
:10D2C0002D5F3F4FE901D595C795D595C795CB0102
:10D2D00001968C179D0714F4219706C06150704089
:10D2E000C617D7070CF4219680912103843BD0F018
:10D2F000F701E65BF84F80819181FE01E81BF90B95
:10D30000CF0163E070E00E948F77CB01880F991FF7
:10D31000860F971F2EE737E0E20EF31EF701918389
:10D32000808307C02EE737E0E20EF31EF70111827B
:10D330001082000F111F065B184FF801D183C083C4
:10D3400011C00231110570F081E08093F1010AC033
:10D3500081E08093F101109214041092160484E489
:10D360008093120480911404803198F08091160407
:10D37000882331F48091F101882311F48093940182
:10D3800010921404109216041092130484E48093F3
:10D390001204E6E0CDB7DEB70C940778CF93FC011A
:10D3A00097FF05C0CFEFF095E195FF4F01C0C1E0B9
:10D3B00028E631E0CF01B9010E948F77FC018B355F
:10D3C000910554F08B5590408A35910538F484EBE3
:10D3D00090E08E1B9F0BFC0141E00DC0CF01855BEF
:10D3E00090408A35910518F4E45BF04003C02E1B91
:10D3F0003F0BF9014FEFEE0FFF1FE15DF54F259158
:10D4000034918C2F992787FD9095289FB001299FF3
:10D41000700D389F700D1124842F992787FD9095EA
:10D42000689FA001699F500D789F500D1124CA017B
:10D43000CF9108952AE530E0281B390BC9010E94DD
:10D44000CE690895CF93DF9380E00E946070809151
:10D450001E0190911F016AE070E00E948F779F93F8
:10D460008F9380911E0190911F016AE070E00E94ED
:10D470008F777F936F938DEF9AE09F938F93C3E5A0
:10D48000D0E7DF93CF93E0912F04F091300409951A
:10D490002DB73EB7285F3F4F2DBF8091ED01882308
:10D4A000B9F186E00E946070809137089091380849
:10D4B0006AE070E00E947B777F936F938FED90E03E
:10D4C0009F938F938091260890912708A091280818
:10D4D000B0912908209196013091970140919801CF
:10D4E00050919901BC01CD010E94C4773F932F93C5
:10D4F00086E09BE09F938F93DF93CF93E0912F047F
:10D50000F091300409958DB79EB70A968DBF12C071
:10D5100086E00E94607082E19BE09F938F93DF938F
:10D52000CF93E0912F04F091300409950F900F9064
:10D530000F900F90809102048823C1F086E00E9432
:10D5400060708091020499279F938F9389E19BE0FB
:10D550009F938F93DF93CF93E0912F04F09130044A
:10D5600009952DB73EB72A5F3F4F2DBF80E10E943E
:10D5700060708091F7019091F8016CE370E00E9477
:10D580007B779F938F938091F7019091F8016CE3E3
:10D5900070E00E947B777F936F938091A3089091B6
:10D5A000A4089F938F9384E29BE09F938F93C3E59E
:10D5B000D0E7DF93CF93E0912F04F09130040995E9
:10D5C00080912C062DB73EB7265F3F4F2DBF80FFC1
:10D5D00029C08AE10E9460708091950199279F93EC
:10D5E0008F938091130390911403A0911503B09130
:10D5F0001603BC01CD0124E630E040E050E00E947B
:10D60000C4773F932F9381E39BE09F938F93DF93A6
:10D61000CF93E0912F04F091300409958DB79EB718
:10D6200008968DBFDF91CF910895CF93DF9380E06F
:10D630000E94607080910807992787FD90959F93BD
:10D640008F9380910007992787FD90959F938F93E3
:10D650008091F806992787FD90959F938F938091ED
:10D66000F006992787FD90959F938F9388E39BE021
:10D670009F938F93C3E5D0E7DF93CF93E0912F047F
:10D68000F0913004099580E10E9460702DB73EB79B
:10D69000245F3F4F2DBF80912807992787FD9095E4
:10D6A0009F938F9380912007992787FD90959F9353
:10D6B0008F9380911807992787FD90959F938F935B
:10D6C00080911007992787FD90959F938F9388E409
:10D6D0009BE09F938F93DF93CF93E0912F04F09182
:10D6E0003004099580911E062DB73EB7245F3F4F49
:10D6F0002DBF853098F480E10E94607088E59BE042
:10D700009F938F93DF93CF93E0912F04F091300498
:10D7100009950F900F900F900F9018C08730B0F4BC
:10D7200088E10E9460708FED90E09F938F9389E66F
:10D730009BE09F938F93DF93CF93E0912F04F09121
:10D74000300409958DB79EB706968DBFDF91CF91B6
:10D7500008950F931F9380E00E9460702AE030E0EC
:10D7600080919F089091A008B9010E947B779F93B8
:10D770008F9380919F089091A008B9010E947B77B8
:10D780007F936F9380911E0190911F01B9010E94B8
:10D790008F779F938F9380911E0190911F01B90104
:10D7A0000E948F777F936F9382E79BE09F938F9385
:10D7B00003E510E71F930F93E0912F04F0913004DD
:10D7C000099580E10E9460708DB79EB70C968DBF61
:10D7D0008091A5089091A6089F938F938091A108AE
:10D7E0009091A2089F938F9385E89BE09F938F93DE
:10D7F0001F930F93E0912F04F091300409958DB79A
:10D800009EB708968DBF1F910F9108950F931F9398
:10D81000CF93DF938091ED01C3E5D0E7882309F42E
:10D8200078C080E00E9460708091340899279F93AF
:10D830008F938091360899279F938F9381E99BE07E
:10D840009F938F938E01DF93CF93E0912F04F091FC
:10D85000300409958DB79EB708968DBF8091350825
:10D86000833031F48CE00E94607080EA9BE005C058
:10D870008CE00E94607085EA9BE09F938F93DF931A
:10D88000CF93E0912F04F091300409950F900F9001
:10D890000F900F908091330881FF12C08CE00E949E
:10D8A00060708AEA9BE09F938F931F930F93E091A0
:10D8B0002F04F091300409950F900F900F900F9066
:10D8C00080E10E9460708FED90E09F938F93809134
:10D8D000390890913A089F938F93809137089091DF
:10D8E00038086AE070E00E947B777F936F938FEA3D
:10D8F0009BE09F938F9383E590E79F938F93E091B5
:10D900002F04F091300409958DB79EB70A968DBF0C
:10D9100012C082E00E9460708FEB9BE09F938F9318
:10D92000DF93CF93E0912F04F091300409950F908D
:10D930000F900F900F90DF91CF911F910F9108954D
:10D94000CF93C82F209117042093180499278F3262
:10D95000910509F1803391051CF44F97A1F02CC07B
:10D960008F34910501F18F38910531F5222319F497
:10D9700081E090E038C086E0289FF0011124EB514F
:10D98000F54F849117C086E0289FF0011124EA51D9
:10D99000F54F84910FC086E0289FF0011124E951D2
:10D9A000F54F849107C086E0289FF0011124E851CB
:10D9B000F54F849180931704909117048091180477
:10D9C0009813C0E00E9466709091170486E0989FBB
:10D9D000F0011124E751F54F259134918C2FF90175
:10D9E000099580E090E0CF9108951092A0081092E0
:10D9F0009F081092A4081092A3081092A2081092F7
:10DA0000A1081092A7089091480684E6989FC0014B
:10DA100011249093A6088093A5088AE090E00E94C4
:10DA20001A1790931A04809319040895CF93DF93E3
:10DA30008091190490911A040E942317882309F4F5
:10DA400000C18091190490911A040A9690931A04C7
:10DA500080931904E0E0F0E09F0190E05FEFA9EE11
:10DA6000B6E04BE0ED018B8187FF0BC09F5F8D819E
:10DA7000E80FF11D8981280F311D8E81851708F46B
:10DA8000582F4150189647FFEDCF5093A708232BEE
:10DA900041F520911F0430912004409121045091C0
:10DAA0002204BB27A52F942F832F90931E048093CD
:10DAB0001D04AA27BB27281B390B4A0B5B0BCF0180
:10DAC000AA27BB27280F391F4A1F5B1F20931F045B
:10DAD000309320044093210450932204E5E0F0E0C9
:10DAE00013C020911D0430911E042E173F0718F417
:10DAF000E21BF30B02C0E0E0F0E0892F9927880FCA
:10DB0000991FE80FF91F3596F093A008E0939F083E
:10DB1000EF3FF10578F480911E0190911F018E9FD7
:10DB200090018F9F300D9E9F300D1124C90164E636
:10DB300070E013C0CF0196958795969587952091B3
:10DB40001E0130911F01289FA001299F500D389F71
:10DB5000500D1124CA0169E170E00E947B77709337
:10DB6000A2086093A10820911B0430911C042E0F81
:10DB70003F1F30931C0420931B045EE021313507C6
:10DB800008F45FC08091A3089091A4080196909337
:10DB9000A4088093A30820513E4030931C04209396
:10DBA0001B044091480624E6429F90011124281B43
:10DBB000390B3093A6082093A50812161306B4F16A
:10DBC000C90164E670E00E948F77892B79F54423C0
:10DBD00069F18091ED0280628093ED0280910801ED
:10DBE000909109018F5F9F4F61F5C90164E670E074
:10DBF0000E948F7777FF03C0709561957F4F80ED0E
:10DC000097E0689F9001699F300D789F300D112437
:10DC1000C9018053984F909329028093280280E095
:10DC200094E090930901809308010BC08091280231
:10DC300090912902892B29F48091ED028F7D8093A8
:10DC4000ED02DF91CF910895002422273327442746
:10DC500051E0BB27EE27FF27A0E1660F771F881F43
:10DC6000991F001C221F331F441F660F771F881F38
:10DC7000991F001C221F331F441F2AF4050E2B1F5F
:10DC80003E1F4F1F04C0051A2B0B3E0B4F0B550FA9
:10DC9000BB1FEE1F587F556047FD5250AA95E9F60D
:10DCA000E695B7955795E695B7955795852F9B2F90
:10DCB00008952227332741E0552768E0880F991FF0
:10DCC000221F331F880F991F221F331F1AF4240F9E
:10DCD000351F02C0241B350B440F551F487F45607C
:10DCE00037FD42506A9551F7569547955695479599
:10DCF000842F0895AA2797FF04C0809590958A1FC6
:10DD00009A1F77FF04C0609570956A1F7A1F669FFF
:10DD10009001779FA001679F300D411D5A1F300D64
:10DD2000411D5A1F889FF001999F2E0F3F1F401DD4
:10DD3000511D899F300D411D5A1F300D411D5A1F25
:10DD4000CA01B901112480CF4FB720E430E0F89424
:10DD50008091C9008F778093C9008091C9008F7B23
:10DD60008093C9008091C9008F7D8093C9005A9A21
:10DD700052985B9A539A832F99278093CD002093D2
:10DD8000CC008091C80082608093C80088E18093B5
:10DD9000C9008091CA008F778093CA008091CA0021
:10DDA0008F7B8093CA008091CA008F7D8093CA00C8
:10DDB0008091CA008F7E8093CA008091CA00877FBD
:10DDC0008093CA008091C9008B7F8093C9008091A5
:10DDD000CA0084608093CA008091CA0082608093E8
:10DDE000CA008091C80087FF03C08091CE00F9CFA0
:10DDF0008091C90080688093C9004FBF08950F9338
:10DE00001F93CF93DF93482F4F5F893108F08BC06A
:10DE100080914907841720F44F5F40934907415090
:10DE2000CB0183539B4268E170E00E948F77A42F5F
:10DE3000BB27FD01EA0FFB1FE65BF84F8081918154
:10DE40009B01281B390BC90137FF03C090958195B1
:10DE50009F4F069794F480912103883C30F4809181
:10DE60002103865F8093210308C088EC80932103FF
:10DE700080916F008F7D80936F00FD01EA0FFB1F83
:10DE8000E65BF84F808191819C01220F331F280FA0
:10DE9000391F260F371F37FF02C02D5F3F4FE901A3
:10DEA000D595C795D595C795CB0101968C179D073C
:10DEB00014F4219706C061507040C617D7070CF4C0
:10DEC000219680912103843BD8F08D010A0F1B1FFE
:10DED000F801E65BF84F80819181FE01E81BF90BA8
:10DEE000CF0163E070E00E948F77CB01880F991F0C
:10DEF000860F971F0258184FF8019183808307C03F
:10DF0000AA0FBB1FA258B84F11961C921E92E42F65
:10DF1000FF27EE0FFF1FE65BF84FD183C08344302D
:10DF200011F410929401DF91CF911F910F910895F8
:10DF3000CF93DF932091A808822F9927807F90703C
:10DF4000409709F06CC02F3109F046C08091A908B4
:10DF5000809327042091AB08209329048091AC087A
:10DF600080932804822F992790934B0780934A0728
:10DF7000222309F054C080912006282F3327220F36
:10DF8000331FF901E258F84F118210828091210667
:10DF9000A82FBB27AA0FBB1FFD01E258F84F118223
:10DFA000108280912306E82FFF27EE0FFF1FCF017D
:10DFB0008258984FEC0119821882265B384FE9018C
:10DFC00019821882A65BB84F11961C921E92E65BCE
:10DFD000F84F1182108223C0C22FCF70CA30F8F4DC
:10DFE0008091A9088093D2088091AA088093D108D3
:10DFF0008091AB088093D4088091AC088093D308BB
:10E000006091D1087091D2088C2F0E94FF6E6091B0
:10E01000D3087091D4088C2F8F5F0E94FF6EDF9120
:10E02000CF910895CF93C82F8F3F49F480912A0450
:10E030008F3F29F410922C0410922B0432C02091AF
:10E040002C04222339F4CF3111F485E001C084E09F
:10E0500080932D0480912D0490912B048217A0F4BD
:10E06000892F809580932B048F3F19F48EEF809336
:10E070002B0480912B04C81711F40E94986F109202
:10E080002C0410922B040BC0E22FFF27E855F74F0A
:10E09000C0832F5F20932C049C0F90932B04C0937C
:10E0A0002A04CF91089590912604933240F4E92FE9
:10E0B000FF27E255F74F80839F5F909326040895D2
:10E0C000833218F48D5F80932604089590E2E1EB8B
:10E0D000F8E08FE19193815087FFFCCF0895CF93B3
:10E0E000CFB723E031E0F8948091C9008F77809317
:10E0F000C9008091C9008F7B8093C9008091C900BD
:10E100008F7D8093C9005A9A52985B9A539A832FB5
:10E1100099278093CD002093CC008091C800826025
:10E120008093C80088E18093C9008091CA008F77EE
:10E130008093CA008091CA008F7B8093CA0080912F
:10E14000CA0080628093CA008091CA008061809377
:10E15000CA008091CA0088608093CA008091C9007B
:10E1600084608093C9008091CA0084608093CA0053
:10E170008091CA0082608093CA008091C80087FFA6
:10E1800003C08091CE00F9CF8091C9008068809350
:10E19000C9008091C90080648093C9000E946670A4
:10E1A000CFBFCF910895282F99278F709070892B1A
:10E1B00031F4209580912504822B809325040895C5
:10E1C0008091F401882309F441C08091ED0285FF1C
:10E1D0000AC082E98093AE0883E28093AF0885E5A8
:10E1E0008093B00802C01092AE088091F5018F3084
:10E1F00071F4809125040E94A06C882341F081E98C
:10E200008093AE088093AF0881E38093B0081092AA
:10E21000F4018091C80085FFFCCF8091C9008F7EFA
:10E220008093C9008091C9008E7F8093C90080913E
:10E23000AE08882311F48EEF01C08EE78093CE00E4
:10E24000809125048093F5011092250408951F9272
:10E250000F920FB60F9211248F939F93EF93FF931A
:10E260009091F401992309F040C080912E048823F5
:10E2700061F48091AE08882311F483E003C08139F2
:10E2800099F481E080932E040FC0833099F480913B
:10E29000AE08882349F09093AE088091C9008E7F24
:10E2A0008093C9008EEF1EC08091C9008160809369
:10E2B000C9000EC0833261F48091C9008E7F8093C3
:10E2C000C9008FEF8093CE0081E08093F40114C0E9
:10E2D00080912E04E82FFF27E255F74F8F5F809340
:10E2E0002E0480818093CE0007C010922E0480916E
:10E2F000C90080618093C900FF91EF919F918F9138
:10E300000F900FBE0F901F901895EF92FF920F93F2
:10E310001F93CF93DF937C018B01EA01452B39F0EA
:10E32000F80181918F01F70109952197C9F7E6E07E
:10E33000CDB7DEB70C940778EF92FF920F931F933F
:10E34000CF93DF937C018B01EA01452B41F0F8016B
:10E350000F5F1F4F8491F70109952197C1F7E6E000
:10E36000CDB7DEB70C9407780F931F93CF938C0132
:10E37000C62F161634F480E2F8010995C1501C1618
:10E38000D4F3CF911F910F9108950F931F93CF93C3
:10E390008C01C62F161634F480E3F8010995C1509C
:10E3A0001C16D4F3CF911F910F910895A5E3B0E00F
:10E3B000ECEDF1E70C94DF772E96EEADFFAD2E97E6
:10E3C00088249924540180912404882321F42C96D4
:10E3D0001FAE1EAE2C975EE4452E512C4C0E5D1EDA
:10E3E0006F01B60105C0153239F00894C11CD11C6B
:10E3F000F60114911123B9F7A601461B570B31F012
:10E400002C968EAD9FAD2C970E949C71112309F420
:10E410006AC20894C11CD11CFF24FDA6FCA64FEFC4
:10E42000E42EF9A6F6010894C11CD11C14911537ED
:10E4300021F0812F80628837B1F4F0FE0AC0F2012A
:10E4400024E030E0420E531E80809180A280B38091
:10E450000AC0F20142E050E0440E551E80819181D5
:10E460004C01AA24BB24103221F489A58823D1F6BB
:10E470001DC0133219F458E0F52AD4CF1A3211F026
:10E480001D3291F41A3259F4F20182E090E0480E04
:10E49000591EE081ECA7EE232CF6E195ECA790E164
:10E4A000F92AAFEDFA22BECF1B3211F419A7BACF69
:10E4B0001E32C1F5F6010894C11CD11C14911A3208
:10E4C00079F4F20122E030E0420E531E4081518186
:10E4D0003FEF4F3F530714F44FEF5FEFE42EA2CF0F
:10E4E00040E050E0812F80538A30A0F4CA0133E02D
:10E4F000880F991F3A95E1F7840F951F480F591F10
:10E50000410F511D40535040F6010894C11CD11CCD
:10E510001491E8CF8FEF4F3F580714F44FEF5FEFA0
:10E52000E42E85CF103329F4F4FC7CCF90E2F92A55
:10E5300079CF812F81538930D8F440E050E0CA016F
:10E5400023E0880F991F2A95E1F7840F951F480F44
:10E55000591F410F511D40535040F6010894C11CF2
:10E56000D11C1491812F80538A3048F34CA75FCF80
:10E57000183619F4A4E0FA2A55CF1C3619F4B1E084
:10E58000FB2A50CF133661F43E010894611C711CC4
:10E59000F20122E030E0420E531E808189833CC1AB
:10E5A000143421F0143611F0193651F5143411F4E5
:10E5B00031E0F32AF0FE0AC0F20144E050E0440EDC
:10E5C000551E80809180A280B3800CC0F20182E051
:10E5D00090E0480E591E808191814C01AA2497FC3D
:10E5E000A094BA2CB7FE0AC0B094A09490948094E2
:10E5F000811C911CA11CB11C8DE289A70AE06FC08F
:10E600001F3411F01F3631F41F3411F491E0F92A50
:10E6100008E064C0103779F4F201A2E0B0E04A0EDD
:10E620005B1E808191814C01AA24BB2400E1B0E4EF
:10E63000FB2A18E753C01337C1F5F20122E030E09E
:10E64000420E531E608071806114710489F43E0192
:10E650000894611C711C88E289838EE6F301818332
:10E6600085E78B838CE68C838D8389E28E831F8282
:10E67000E7FC13C08E2D992787FD9095AC0160E0D3
:10E6800070E0C3010E948B76009729F0382E36186F
:10E69000E3140CF0C3C03E2CC1C0F3010190002074
:10E6A000E9F731973E2E3618B9C0153511F01537F8
:10E6B00031F4153511F4F1E0FF2A0AE00FC01835E6
:10E6C00019F0183709F0A0C000E1F3FE07C081146B
:10E6D0009104A104B10411F020E4F22A19A6EDA6D8
:10E6E000E7FC02C03FEDF32289E2682E712C6C0E2C
:10E6F0007D1E81149104A104B10421F44DA544238D
:10E7000009F47BC0802F9927AA27BB278EA79FA734
:10E71000A8ABB9AB202E332490E0891690E099067F
:10E7200091E0A90690E0B90648F0C501B4012EA514
:10E730003FA548A959A90E94A27717C0AFEF8A1632
:10E740009104A104B10449F040F0C401B1010E9458
:10E750007B779B014427552708C0882D602F0E9496
:10E760006F77282F3327442755272AAB3BAB4CAB79
:10E770005DAB0A3059F48AA9880F880F880F9AA9CF
:10E78000990F890F382D381B832F10C0003139F4B1
:10E790008AA98295807F482D481B842F07C08AA9AB
:10E7A000880F880F880F582D581B852F90E02EA5B5
:10E7B0003FA548A959A982169306A406B50608F0F4
:10E7C00091E08AA89BA8ACA8BDA88A3010F4805D0F
:10E7D00004C0895A183509F48F7DD3018E933D0109
:10E7E000992309F099CF083041F4F3FE06C0803335
:10E7F00021F080E3FD0182933F01CE010196382E86
:10E800003618F8E23F0E0BC0112309F46CC03E012C
:10E810000894611C711C1983B1E03B2E19A6032DCD
:10E820002DA4231827FC222489A5882311F00F5F2B
:10E8300002C0F6FC0E5F020DEF2CFF24C7018073AF
:10E840009070892B49F48CA5801B682F2C968EAD77
:10E850009FAD2C970E94B47189A5882331F041E0C7
:10E8600050E0BE01675D7F4F0AC0E6FE0EC080E348
:10E870008AA71BA742E050E0BE01665D7F4F2C9641
:10E880008EAD9FAD2C970E948571C70180739070EB
:10E89000809749F48CA5801B682F2C968EAD9FAD78
:10E8A0002C970E94C571622D2C968EAD9FAD2C9732
:10E8B0000E94C571832D992787FD9095AC01B30106
:10E8C0002C968EAD9FAD2C970E948571E4FE89CD6C
:10E8D0002CA5201B2CA7622F2C968EAD9FAD2C97BC
:10E8E0000E94B4717ECDE2E1CB5C0C94FB772FB734
:10E8F00040E0F894E0E0F0E081E2809357009491EA
:10E90000E2E0F0E0809357003491E4E0F0E080939F
:10E91000570084912FBF9E3199F4363941F48930E4
:10E9200011F441E00DC08A3059F442E009C0373992
:10E9300039F4863011F443E003C0853009F444E033
:10E94000842F992708959FB7F8948091C900877FF5
:10E950008093C9008091C9008F7E8093C900809107
:10E96000C9008F778093C9008091C9008F7B809305
:10E97000C9008091C9008F7D8093C90052985A9A2E
:10E9800053985B9A9FBF08951F93CF93DF93182FDF
:10E9900080912404882309F48DC08091F301181715
:10E9A00009F488C080912304882321F40E9477749D
:10E9B0008093230488EB9CE09F938F93C4EFD2E174
:10E9C000DF93CF93E0912F04F091300409950F90DD
:10E9D0000F900F900F90812F99278230910501F1B0
:10E9E000833091052CF4009761F0019769F024C001
:10E9F00084309105D9F084309105ACF00597C9F0C9
:10EA00001BC088EA9CE002C086E99CE09F938F933C
:10EA1000DF93CF93E0912F04F0913004099518C053
:10EA20008DE79CE0F3CF8AE59CE0F0CF8CE49CE09E
:10EA3000EDCF84E49CE0EACF85EC9CE09F938F933C
:10EA4000DF93CF93E0912F04F0913004099510E00B
:10EA50000F900F900F900F9080912304843011F04D
:10EA6000823099F40E94A374812F8150833018F46E
:10EA70000E942A681DC0143019F40E946F7018C0DB
:10EA80001530B1F40E94A46E13C0112389F08BEDF0
:10EA90009CE09F938F9384EF92E19F938F93E091FB
:10EAA0002F04F091300409950F900F900F900F9064
:10EAB0001093F301DF91CF911F9108950F931F934E
:10EAC00081E0809324044091F201E4EFFBE020E038
:10EAD00030E05FE4849199272F5F3F4F829FB00120
:10EAE000839F700D929F700D1124462751503196CF
:10EAF00057FFF0CF4093F201ECECFBE020E030E078
:10EB000057E2849199272F5F3F4F829FB001839FE7
:10EB1000700D929F700D112446275150319657FF6A
:10EB2000F0CF4093F20180912304882321F40E94C6
:10EB30007774809323048091F201833459F088E143
:10EB400090E029E20FB6F894A895809360000FBE7C
:10EB50002093600086ED91E79093300480932F041A
:10EB600086EF9CE09F938F9304EF12E11F930F9326
:10EB7000E0912F04F091300409950F900F900F90C1
:10EB80000F9081E690E09F938F9382E590E09F93B2
:10EB90008F931F921F92809102016AE00E946F770B
:10EBA000892F99279F938F93809102010E946F77FD
:10EBB00099279F938F938CE19DE09F938F931F9351
:10EBC0000F93E0912F04F0913004099584EF9BE0BE
:10EBD0009F938F931F930F93E0912F04F091300434
:10EBE00009958CEC9BE09F938F931F930F93E0917B
:10EBF0002F04F091300409958DB79EB746968DBFCE
:10EC000080E59DE09F938F931F930F93E0912F04D6
:10EC1000F0913004099583EC8093810080916F001E
:10EC2000806280936F000F900F900F900F901F9154
:10EC30000F91089580912404882361F08091F3015D
:10EC4000843011F40E94E0708091F201833411F05D
:10EC50001092240408951F920F920FB60F92112460
:10EC60002F933F934F935F936F937F938F939F93D4
:10EC7000AF93BF93EF93FF932091CE008091FE015D
:10EC80008823B1F02093C6008091FE01823029F5DF
:10EC90002F3F19F58FEF94E3ACE0B0E0C297A109E4
:10ECA000B109B7FFFBCF809172048093CE0015C0ED
:10ECB0009091F301892F8150833020F4822F0E949C
:10ECC00085680BC0943021F4822F0E94D37005C058
:10ECD000953019F4822F0E941270FF91EF91BF912D
:10ECE000AF919F918F917F916F915F914F913F91E4
:10ECF0002F910F900FBE0F901F901895FB01DC0114
:10ED000040FF05C002C005900D9205900D92425043
:10ED10005040C8F70895FC014150504030F0019038
:10ED20000616D1F73197CF010895882799270895BE
:10ED30005058192E84D001D06AC0BA1762077307E1
:10ED400084079507B1F188F40EF410940B2EBA2FB6
:10ED5000A02D062E622F202D072E732F302D082E6A
:10ED6000842F402D092E952F502DFF275523B9F0C4
:10ED7000591B49F0573E98F0469537952795A7952A
:10ED8000F0405395C9F776F0BA0F621F731F841FC6
:10ED900030F4879577956795B795F040939517FA76
:10EDA0000F2E0895BF1BBB27BA0B620B730B840B8E
:10EDB000F6CFDEF670C097FB4ED09F3738F0FEE9F5
:10EDC000F91B982F872F762F6B2F05C061C0969562
:10EDD000879577956795F150D0F73EF4909580959B
:10EDE000709561957F4F8F4F9F4F0895E89403C0B2
:10EDF00097FB0EF4F3DFB62F672F782F892F9EE94C
:10EE0000002405C09A95BB0F661F771F881F112429
:10EE10009923A1F08823B2F79F3F59F0BB0F48F424
:10EE200021F4002011F460FF04C06F5F7F4F8F4F0B
:10EE30009F4F881F9795879597F9089529C0052EAC
:10EE4000092607FA440F551F5F3F79F0AA27A51737
:10EE500008F051E04795880F991F9F3F31F0BB277D
:10EE6000B91708F091E0879508959F919F9111241B
:10EE700014C097FB880F991F9F3F31F0BB27B9172C
:10EE800008F091E0879508959F919F91112405C006
:10EE9000662777278827992708959FEF80EC0895A4
:10EEA000629FD001739FF001829FE00DF11D649F6E
:10EEB000E00DF11D929FF00D839FF00D749FF00DFA
:10EEC000659FF00D9927729FB00DE11DF91F639F9B
:10EED000B00DE11DF91FBD01CF0111240895991B4B
:10EEE00079E004C0991F961708F0961B881F7A9541
:10EEF000C9F780950895AA1BBB1B51E107C0AA1F43
:10EF0000BB1FA617B70710F0A61BB70B881F991FCA
:10EF10005A95A9F780959095BC01CD01089597FB6E
:10EF2000092E07260AD077FD04D0E5DF06D00020A1
:10EF30001AF4709561957F4F0895F6F79095819535
:10EF40009F4F0895A1E21A2EAA1BBB1BFD010DC005
:10EF5000AA1FBB1FEE1FFF1FA217B307E407F50789
:10EF600020F0A21BB30BE40BF50B661F771F881F65
:10EF7000991F1A9469F760957095809590959B01FB
:10EF8000AC01BD01CF01089597FB092E05260ED0D7
:10EF900057FD04D0D7DF0AD0001C38F450954095B7
:10EFA000309521953F4F4F4F5F4F0895F6F790955D
:10EFB0008095709561957F4F8F4F9F4F08952F9249
:10EFC0003F924F925F926F927F928F929F92AF92F9
:10EFD000BF92CF92DF92EF92FF920F931F93CF9346
:10EFE000DF93CDB7DEB7CA1BDB0B0FB6F894DEBFDD
:10EFF0000FBECDBF09942A88398848885F846E8403
:10F000007D848C849B84AA84B984C884DF80EE804C
:10F01000FD800C811B81AA81B981CE0FD11D0FB655
:10F02000F894DEBF0FBECDBFED010895EE0FFF1FB8
:10F030000590F491E02D0994F999FECFB2BDA1BDE0
:10F04000F89A119600B40895F7DF01921A94E1F747
:10F050000895F2DFE02DF0DFF02D0895F999FECF4D
:10F06000B2BDA1BD00BC11960FB6F894FA9AF99AF8
:10F070000FBE0895F3DF012CF1DF112408950190F4
:08F08000EDDF1A94E1F7089599
:10F088005E010A010164FF01FFFFC01FC01F0101EB
:10F0980001737373FF03007D0000C409C409640091
:10F0A8001148656C6C6F20576F726C64000000002B
:10F0B8000000000000000000000000000000000048
:10F0C8000000000000000000000000000000000038
:10F0D8000000000000000000000000000000000028
:10F0E8000000000000000000000000000000000018
:10F0F8000053706F727400004E6F726D616C000087
:10F10800426567696E6E6572000051756164726F61
:10F118000000640001200B050000ECFF000204065B
:10F12800070808080706040200FEFCFAF9F8F8F8D0
:10F13800F9FAFCFE000204060708086440415A4632
:10F1480064640A02969696960840403A10FB303856
:10F158000190D0030090D00300F40105F9FF057871
:10F1680000FF03640B0A0D0B0C0E0B0F10FA2001A5
:06F17800010170FF010F10
:00000001FF
